:020000040800F2
:1058000060D10020995A0008A1CD000889950008B0
:10581000C5BD0008056700084D6D010800000000C7
:10582000000000000000000000000000AD5900086A
:10583000456A000800000000355A0008855A000833
:10584000B35A000891CE0008B35A0008B35A0008B2
:10585000B35A0008B35A0008B35A0008B35A0008F4
:10586000B35A0008B35A0008B35A0008B35A0008E4
:10587000B35A0008B35A0008B35A0008B35A0008D4
:10588000B35A0008B35A0008B35A0008B35A0008C4
:10589000B35A0008B35A0008B35A0008156C000840
:1058A000B35A0008B35A0008B35A0008B35A0008A4
:1058B000B35A0008B35A0008B35A0008B35A000894
:1058C000B35A0008B35A0008B35A0008B35A000884
:1058D000B35A000851640108596401086164010861
:1058E000B35A000859E70008B35A0008B35A000831
:1058F000B35A0008B35A0008B35A0008B35A000854
:10590000B35A0008B35A0008B35A0008B35A000843
:10591000B35A0008B35A0008B35A0008B35A000833
:10592000B35A0008B35A0008B35A0008B35A000823
:10593000DFF80CD000F000FC00480047918301081C
:1059400060D1002080F309887047EFF30980704729
:10595000684680F3098804480078C00714BF022015
:10596000032080F31488704728970108DFF818C0D7
:10597000EFF305831B0618BF6047EFF31483DB07C3
:1059800008BF604700DF7047C58A0108DFF818C00C
:10599000EFF305831B0618BF6047EFF31483DB07A3
:1059A00008BF604700DF70476D8C0108EFF3098086
:1059B000816911F8021C39BB90E80F10E047EFF342
:1059C000098C194B93E80600914218D059B10CB4D8
:1059D0004FF0010381F826302CE9F00FC1F82CC0FC
:1059E00013F046FB0CBC1A60D2F82CC0BCE8F00FD8
:1059F00092F826308CF309881BB192F82500CCF878
:105A000000006FF0020E704710B5084A126891420C
:105A100009D8074C54F8214090E80F10A047EFF345
:105A2000098C8CE80F0010BDD004002074620008BF
:105A30007462000813F002FA114B93E806009142D9
:105A40001BD00CB44FF0000381F82630EFF3098C23
:105A50002CE9F00FC1F82CC013F00AFB0CBC1A6043
:105A6000D2F82CC0BCE8F00F8CF3098892F82630ED
:105A70001BB192F82530CCF800306FF0020E704761
:105A8000D004002013F0DAFBD6E7000012F01CFD72
:105A900013F0D4FBD0E700000648804706480047D3
:105AA000FEE7FEE7FEE7FEE7FEE7FEE7FEE7FEE7CE
:105AB000FEE7FEE7113401083159000840EA01030E
:105AC0009B0703D009E008C9121F08C0042AFAD2B4
:105AD00003E011F8013B00F8013B521EF9D2704778
:105AE000D2B201E000F8012B491EFBD27047002220
:105AF000F6E710B513460A4604461946FFF7F0FFCD
:105B0000204610BD421E12F8013F002BFBD111F8B8
:105B1000013B02F8013B002BF9D1704730B5054637
:105B20002A460B4612F8010B13F8014B08B1A042AC
:105B3000F8D01CB1002802D06D1CF1E7284630BD1A
:105B400010B5044604E00B7800F8013B03B1491C92
:105B5000521EF8D2204610BD421C10F8011B00292D
:105B6000FBD1801A704710B5002200E0521C835C04
:105B70008C5CA34201D1002BF8D1D8B2E1B2401A1B
:105B800010BD034611F8012B00F8012B002AF9D1B2
:105B90001846704730B505460020034600E05B1C00
:105BA000934205D2EC5CC85C201A01D1002CF6D1DE
:105BB00030BD70B5064612F013F8046805460A2297
:105BC0000021304600F023FA2C6070BD70B5064607
:105BD00012F006F8046805460A220021304600F05B
:105BE00016FA2C6070BD2DE9FE4F804681EA030055
:105BF000C00F0C46009021F0004123F00045B8EBA7
:105C00000200A94105D24046214690461C460B465B
:105C1000024623F00040104347D0270DC7F30A0087
:105C2000C3F30A510290401A019040286BDAC3F383
:105C3000130040F4801B0098924620B10023D2EB61
:105C4000030A63EB0B0B01985946C0F14002504622
:105C500000F0ACF906460D4650465946019A00F050
:105C6000C4F910EB08006141002487EA115284EA6C
:105C7000E7731A4340D0009A62B3019A012A4FEAAF
:105C8000075215DC001B61EB02014FF0004202EAF3
:105C90000752CDE90042001C41F5801132462B46E7
:105CA00000F0FCF903B0BDE8F08F40462146F9E76B
:105CB000001B61EB0201001C41F5801300185B41E1
:105CC0002018A2F5001747EB030140EAD570B6197A
:105CD0006D4111E06D084FEA360645EAC0754FEA9E
:105CE0000752001B61EB0201001C41F580114908BD
:105CF0004FEA30000019514132462B4603B0BDE84F
:105D0000F04F00F0BCB90098012240000023D0EB16
:105D1000020263EBE073009821464FEAE074B8EBAF
:105D2000000061EB0401E9E783F000435BE781F0E9
:105D3000004158E72DE9FE4F81EA030404F00044D6
:105D400021F0004100944FF0000B23F0004350EA93
:105D500001045ED052EA03045BD0C3F30A54C1F3DA
:105D60000A552C44A4F2F3340194A0FB0254C1F36D
:105D7000130141F48011C3F3130343F4801301FBB7
:105D8000024400FB034E840A970A44EA815447EA1E
:105D90008357A4FB076802958D0A05FB07854FEA28
:105DA000932C04FB0C542705029D4FEA065847EA42
:105DB0001637B5EB08056EEB070C870E920E47EA17
:105DC000811742EA8312A7FB0201B6EB0B0164EBD9
:105DD00000042B0D43EA0C335E1844EB1C50DA46EA
:105DE0005146E7FB0201C5F313044FEA0B3343EAC4
:105DF00014534FEA0432019C43EA0603A4F10C0455
:105E00000294009CCDE900B400F048F903B0BDE86D
:105E1000F08F00200146F9E72DE9F04D81EA0304F7
:105E200004F0004B21F0004514464FF0000A23F027
:105E3000004150EA050220D054EA01021DD0C5F30A
:105E40000A570246C5F31303C1F31300C1F30A5600
:105E500040F4801543F48013A7EB0608101BD646C8
:105E600008F2FD3873EB050002D308F1010801E0E8
:105E700092185B41B8F1000F03DA00200146BDE83B
:105E8000F08D00204FF48011064684460EE0171B6B
:105E900073EB050705D3121B63EB050306434CEABE
:105EA000010C49084FEA300092185B4150EA0107A3
:105EB000EDD152EA030012D082EA040083EA050120
:105EC000084305D0101BAB4106D20122002306E097
:105ED00000224FF0004302E06FF0010253101AEB72
:105EE00006004CEB085110EB0A0041EB0B01BDE83A
:105EF000F04D00F0C4B80EB5C10F80EAE070084460
:105F0000CA07002140F233438DE80E000A460B46D3
:105F100000F0C4F803B000BDC1F30A5210B5C1F3DC
:105F2000130140F2FF3341F480119A4201DA00205C
:105F300010BD40F233439A42A2F2334203DC524294
:105F400000F043F810BD904010BD2DE9F05F05460C
:105F5000002092469B4688460646814640241BE028
:105F6000284641464746224600F02FF853465A46F7
:105F7000C01A914110D311461846224600F016F877
:105F80002D1A67EB01084F4622460120002100F040
:105F90000DF817EB00094E41201EA4F10104DFDCCF
:105FA000484631462A464346BDE8F09F202A04DB96
:105FB000203A00FA02F1002070479140C2F120031C
:105FC00020FA03F3194390407047202A04DB203A5B
:105FD00021FA02F00021704721FA02F3D040C2F109
:105FE00020029140084319467047202A06DBCB1750
:105FF000203A41FA02F043EAE07306E041FA02F384
:10600000D040C2F1200291400843194670472DE963
:10601000F04791460F4680460446002614F8015B7F
:106020002DB100F09BF80068405DC007F6D12B2D24
:1060300002D02D2D18D0641E4A463946204600F065
:1060400091F827B13968A14201D1C7F800807105E4
:106050004FF002040BD54042002803DD11F0C0FDD3
:106060000460A007BDE8F08746F48066E4E70028F6
:10607000F8DA11F0B5FD04606FF00040F2E710B5FA
:10608000141E73F1000408DA401C41F1000192185B
:106090005B411A4301D120F0010010BD2DE9F04D04
:1060A00092469B4611B1B1FA81F202E0B0FA80F259
:1060B00020329046FFF77AFF04460F4640EA0A0076
:1060C00041EA0B0153465A46084313D0114653EA9E
:1060D000010019D0C8F140025046FFF776FF05468F
:1060E0000E46504659464246FFF760FF084305D02A
:1060F000012004E020463946BDE8F08D002005432C
:1061000046EAE0762C4337430A986305E40AA0EB9D
:1061100008000022FD0A44EA47540A3002D5002054
:106120000146E9E7010510196941DDE90845001953
:106130006941BDE8F04DA2E7064C074D06E0E06876
:1061400040F0010394E8070098471034AC42F6D3BE
:10615000FFF7F2FBD8B50108F8B501080048704711
:10616000D0B101082DE9F05F82460078002715467E
:106170008B460AF10104B946302801D09DB113E0E5
:1061800014F8010B0127782803D0582801D045B115
:106190000AE00DB1102D07D10027102514F8010BCE
:1061A00002E0082500E00A250026B0460EE005FBC7
:1061B000080005FB06F1012701EB10461FFA80F8E5
:1061C000B6F5803F00D3B94614F8010B294600F01C
:1061D00018F80028EBDABBF1000F05D00FB1641EF0
:1061E00000E05446CBF80040B9F1000F06D011F0A2
:1061F000F7FC02210160C81EBDE8F09F48EA064096
:10620000FAE73A2800D2303820F02002412A01D3A0
:10621000A2F13700884201D34FF0FF30704770B5CC
:106220008C1810F8015B15F0070301D110F8013B41
:106230002A1106D110F8012B03E010F8016B01F8C8
:10624000016B5B1EF9D12B0705D40023521E0DD420
:1062500001F8013BFAE710F8013BCB1A921C03E06E
:1062600013F8015B01F8015B521EF9D5A142D8D3A6
:10627000002070BD0000000000B587B00121480279
:1062800008F0AAF90121082008F0A6F90120ADF8CC
:10629000040048208DF8070001A9194801F006FA0A
:1062A000642000F0D0FB00208DF8070001A91448FD
:1062B00001F0FCF9C82000F0C6FB002002908DF828
:1062C0000C008DF80D004FF4602004900020059024
:1062D00001208DF8180002A90A4800F02DF80023CB
:1062E00001221946074800F04FF80121054800F047
:1062F0000BF80121034800F0A3F807B000BD00002F
:10630000000801400024014021B1826842F00102EE
:10631000826003E0826822F00102826070470146D9
:10632000C86C80B270470246002013680B400BB166
:10633000012000E00020704730B502460020002315
:1063400050680F4C20400D790C6844EA0524204326
:10635000506090680B4C2040D1E902542C434D7999
:1063600044EA450420439060D06A20F470000C7C1D
:10637000641EE4B2234340EA0350D06230BD000003
:10638000FFFEF0FFFDF7F1FFF0B504460D460020DB
:106390000021092D11DDE068A5F10A0606EB46078C
:1063A000072606FA07F18843A5F10A0606EB46061A
:1063B00003FA06F10843E0600CE0206905EB4507AD
:1063C000072606FA07F1884305EB450603FA06F1AE
:1063D00008432061072A0FDA606B561E06EB86071A
:1063E0001F2606FA07F18843561E06EB860605FAB5
:1063F00006F10843606322E00D2A0FDA206BD61FF6
:1064000006EB86071F2606FA07F18843D61F06EB20
:10641000860605FA06F10843206310E0E06AA2F15F
:106420000D0606EB86071F2606FA07F18843A2F140
:106430000D0606EB860605FA06F10843E062F0BD9C
:1064400021B1826842F4A002826003E0826822F4F3
:10645000A00282607047F0B504460A4625460CE06B
:1064600003F00F071E11304600F02FF802F8010B61
:10647000384600F02AF802F8010B15F8013B002B12
:10648000EED100201070F0BD2DE9F04706460C4615
:1064900037464FF0040811E017F8015B05F00F0ACA
:1064A0004FEA2519484600F010F804F8010B504651
:1064B00000F00BF804F8010BA8F10108B8F1000F87
:1064C000EAD100202070BDE8F087002805DB09280C
:1064D00003DC00F13001C8B208E00A2805DB0F2810
:1064E00003DC00F15701C8B200E0FF207047000054
:1064F00030B595B004465022374901A8FFF7DEFABF
:10650000002536A1204606F02AF928B9204601F0D8
:1065100013FA344908605DE033A1204606F01FF904
:10652000002832D104F10800FFF743FB304908701E
:1065300004F10B00FFF73DFB2E49087004F10E003B
:10654000FFF737FB2C49087004F11100FFF731FB0E
:1065500008302A49087008460078182803DB0846E6
:1065600000781838087004F11400FFF722FB244962
:10657000087004F11700FFF71CFB22490870012284
:1065800021A100200CF0CCFD24E022A1204606F041
:10659000E6F830B90120224981F82D030020C871A6
:1065A00018E020A1204606F0DAF898B901AB0322E2
:1065B0002C21204600F04CFF054625B12846FFF768
:1065C000F8FA1A49086019480068072802D104201F
:1065D0001649086015B030BD009C01082B4353518B
:1065E0003A000000480000202B43434C4B3A000087
:1065F000A5040020A6040020A7040020A404002075
:10660000A2040020A30400205570646174655469DD
:106610006D6500002B504F433A53544152540000D3
:10662000FC3100202B434F50530000001801002084
:1066300010B510480078012800D110BD02240E4882
:10664000407800B109240D480078401CC0B20B49C5
:106650000870A0420CDD0AA006F06AF80120DFF8FD
:106660002CC000DF0AA006F063F800200349087080
:1066700000BFE2E7BC000020FC3100202401002024
:1066800041542B4353510D0A00000000198C01089E
:1066900041542B434F50533F0D0A000001490860FD
:1066A0007047000000860D4208B50121052007F063
:1066B00093FF0220ADF8000018208DF8030003209E
:1066C0008DF802006946054800F0F0FF22210720FE
:1066D00008F01CFD00200249086008BD00080140C8
:1066E0003400002010B504462CB102F09DFA402180
:1066F00001A00BF01BFD10BDC9FDBCB6C4A3CABDF3
:1067000000000000044802680448018804A011F059
:106710002FFA00BFFEE70000D8000020D4000020C0
:106720000D0A5B4246485D463D25642C4C3D256480
:106730000000000010B500241B48006800F00800AD
:10674000A0B100BF012219A100200CF0E9FC1648FD
:10675000006800F0080119A011F00AFA0A2000F000
:1067600072F904201B49486100BFFEE710E0601C7D
:106770000446194988420BD30420184908600122B5
:1067800017A100200CF0CCFC04201249086110BDB8
:106790000548006800F008000028E8D0012213A195
:1067A00000200CF0BDFCCDE7080C01400D0A50772D
:1067B000724F6E4661696C65640000004B657950EC
:1067C00077725374617475733D3D3D253031367871
:1067D0000D0A00000010014080841E0014140140C6
:1067E0000D0A5077724F6E4F6B0000000D0A507704
:1067F00072206572726F000010B504463748007849
:10680000002805DD35480078401E3449087023E033
:106810003348007800B3B4F5D87F05DC4FF400416D
:10682000304801F017F8B8B9B4F5D17F11DA10206B
:106830002D4908612D480078401CC0B22B490870D2
:10684000052809DD01202A49087000202749087021
:1068500002E000202549087025480078012804D16D
:1068600023490870102020494861B4F5AC7F21DC31
:10687000204801780078401C1E4A10701E2900DA5A
:1068800010BD00201B49087001221BA10CF048FC20
:106890000120DFF87CC000DF1E484079012801D1CB
:1068A00011F016FC00201B49487104200E49486174
:1068B00000BFFEE7B4F5B07F0ADC17480078401C43
:1068C000C0B2154908701E2805DD0020087002E0DE
:1068D00000201149087000BFD2E700004D030020DE
:1068E0004C0300200008014000100140CC000020B3
:1068F000120100201101002056626174206C6F7734
:106900002173687574646F776E206E6F7721000055
:10691000198C0108FC3100201001002010B504463C
:1069200024B1012C26D0022C6CD147E0012236A1E3
:1069300000200CF0F5FB0A20DFF8D8C000DF364855
:106940000470002240F2255134480FF0E8FD012286
:1069500040F2244131480FF0E2FD002240F225517F
:106960002F480FF0DCFD012240F224412C480FF0AB
:10697000D6FD47E001222BA100200CF0D1FB0A201C
:10698000DFF890C000DF24480470012240F2255156
:1069900022480FF0C4FD002240F224411F480FF0AE
:1069A000BEFD012240F2255121480FF0B8FD002222
:1069B00040F224411E480FF0B2FD23E001221DA148
:1069C00000200CF0ADFB0A20DFF848C000DF1248C1
:1069D0000470012240F2255110480FF0A0FD002262
:1069E00040F224410D480FF09AFD012240F225515A
:1069F0000B480FF094FD002240F2244108480FF0AC
:106A00008EFD00BF00BF10BD434F4D3C2D2D3E4DB0
:106A100043552100198C01087601002000380140FF
:106A200000440040434F4D3C2D2D3E475053210024
:106A300000480040434F4D3C2D2D3E4D6F64656D29
:106A400021000000704710B5024607E0002101E078
:106A50004B1C99B241F270739942F9DB131EA2F1FB
:106A60000104A2B2F2D110BD01461CE000BF00BF7C
:106A700000BF00BF00BF00BF00BF00BF00BF00BF1E
:106A800000BF00BF00BF00BF00BF00BF00BF00BF0E
:106A900000BF00BF00BF00BF00BF00BF00BF00BFFE
:106AA00000BF00BF00BF0A1EA1F1010399B2DDD1F2
:106AB0007047000070B586B002AC02AE4A48C1888B
:106AC0004A4800EB8100006800901022204600999F
:106AD00012F0BCFC9DF80900012812D14348163879
:106AE000808870B1414816388088401E3F49163969
:106AF00088800846808820B90846007820F0010088
:106B000008703A481638408830B1384816384088FE
:106B1000401E364916394880344816380078C0F38C
:106B2000800060B13148163800788008401E2F4937
:106B30001639097860F382012C48163801702B4809
:106B40001638D0F80600009988420FD005AD049899
:106B500000F10C010422284612F0EEFC04AD059869
:106B600000F108010422284612F0E6FC0020019002
:106B7000012201A8009912F0DFFC1C481638D0F859
:106B800006000099884228D018481638D0F8061018
:106B90001022204612F05AFC14481638D0F806008D
:106BA00000F108010422684612F0C6FC049800F1C6
:106BB0000C010422684612F0BFFC009800F10801A5
:106BC000042204A812F0B8FC009800F10C01042281
:106BD0000648103812F0B0FC04E004491639059854
:106BE000C1F8060006B070BD0C2F00200E1C00205E
:106BF00028B10021054A1170054A116004E0012105
:106C0000024A1170024A116070470000180000200B
:106C1000AC01002010B54FF4007000F01DF8012801
:106C200008D1042004490861012004490870400289
:106C300000F006F810BD000000100140B100002077
:106C400001490860704700001404014001490860D0
:106C5000704700001404014001460020034A1268F6
:106C60000A400AB1012000E00020704714040140EE
:106C7000014600200022074B1B6803EA0102054B76
:106C800014331B680B4013B10AB1012000E000204F
:106C9000704700000004014010B50446202113484D
:106CA00000F0D8FD012802D11149087002E000204F
:106CB0000F4908700F4890F900000D490978884283
:106CC00000D194B10C48007801280EDD0848007806
:106CD00040B2084908700648007818B907A005F0C6
:106CE00027FD02E009A005F023FD10BD00100140C2
:106CF000300000203C000020B000002041542B5008
:106D00004F433D36303826320D0A000041542B5097
:106D10004F433D36303826310D0A000010B50020B3
:106D2000164908700CF01CFA0A214FF4936008F021
:106D3000B5FE1420DFF848C000DF0CF011FA0A217C
:106D400040F26E3008F0AAFE1420DFF834C000DFF5
:106D50000CF006FA0A214FF4936008F09FFE012020
:106D60000FF014FD012003F07FFD08200AF008F861
:106D7000012204A100200CF0D3F910BD6001002015
:106D8000198C01085B456E74657254784D6F6465AB
:106D90005D00000010B5002401200FF0ABFC00BF27
:106DA0001BE001220EA100200CF0BAF93220DFF81E
:106DB00040C000DF02F08EFC0E48007801280AD1A6
:106DC00020200DF03DFB05E06420DFF824C000DF4B
:106DD00002F080FCF8E7601CC4B2062CE1DB10BDB9
:106DE00041542B504F433D3530300D0A0000000018
:106DF000198C01086101002010B5002000F0E0FBB3
:106E000006200DF01DFB10BD0149C8607047000051
:106E10000020024030B5044604250F4800F083F8F6
:106E20000546042D16D10D48006940F002000B49BB
:106E3000086108464461006940F040000861064866
:106E400000F071F805460548006941F6FD710840FB
:106E500002490861284630BDFFFF0B0000200240B8
:106E600004200B49C96801F0010109B101200EE0BD
:106E70000749C96801F0040109B1022007E004498B
:106E8000C96801F0100109B1032000E00420704737
:106E9000002002400348006940F080000149086179
:106EA000704700000020024070B504460D460426DD
:106EB000F00200F038F80646042E11D109480069A6
:106EC00040F00100074908612580F00200F02BF82E
:106ED00006460448006941F6FE7108400149086110
:106EE000304670BD00200240024803494860034814
:106EF000486070472301674500200240AB89EFCD11
:106F000000B502460423FFF7ABFF034603E0FFF79B
:106F1000A7FF0346521E012B01D1002AF7D102B967
:106F20000523184600BD00B502460423FFF798FF6D
:106F3000034603E0FFF794FF0346521E012B01D1E5
:106F4000002AF7D102B90523184600BD10B5402428
:106F500003F00EFA5B490860084600685A49884207
:106F600070D058480068594A811A90426BD00CDCA6
:106F70005749084488B3B0F5800F65D0B0F5C00F0D
:106F800070D0B0F5E00F1AD14FE0B1F5802F3FD0AF
:106F900050480844A0B1B0F5767F04D0A0F2DE30AE
:106FA0000028F0D127E0A0B2122350224A2101F09C
:106FB00087FEA0B2012348A24A2102F043FA72E000
:106FC000A0B2122350224A2101F07AFEA0B201237E
:106FD00043A24A2102F036FA65E0FFE7A0B212238D
:106FE00050224A2101F06CFEA0B201233AA24A21AC
:106FF00002F028FA57E0A0B2122350224A2101F0F1
:107000005FFEA0B2012338A24A2102F01BFA4AE037
:10701000A0B2122350224A2101F052FEA0B2012355
:1070200033A24A2102F00EFA3DE0A0B21223502210
:107030004A2101F045FEA0B201232FA24A2102F00D
:1070400001FA30E030E01AE0A0B2122350224A21C7
:1070500001F036FEA0B2012329A24A2102F0F2F982
:1070600021E0FFE7A0B2122350224A2101F028FEBE
:10707000A0B2012324A24A2102F0E4F913E0A0B255
:10708000122350224A2101F01BFEA0B2012320A2AC
:107090004A2102F0D7F96420DFF87CC000DF242009
:1070A0000DF0CEF900BF0BE0A0B2122350224A210E
:1070B00001F006FEA0B2012318A24A2102F0C2F993
:1070C00010BD0000A40200200A04FC000A04F40021
:1070D000F6FB83FFE003F8FFD7F3D2BB000000000C
:1070E000C9CFD2BB00000000D7F3B6FE00000000FD
:1070F000D7F3C8FD00000000D5FDD2BB00000000A2
:10710000D5FDB6FE00000000D5FDC8FD0000000062
:10711000D5FDCBC400000000198C0108CEDE0000B4
:1071200010B51F4800681F49884212D11E480078D8
:1071300018B9012009F024FE02E0002009F020FE29
:107140001948007808B9012000E0002016490870AD
:1071500024E0134800681549884212D1124800788B
:1071600018B9042009F00CFE02E0002009F008FE26
:107170000D48007808B9012000E000200A49087095
:107180000CE0074800680A49884207D100200649F8
:10719000087009F0F5FD24200DF052F910BD000033
:1071A0005C0000200A04BC00A90200200A04DC00E4
:1071B0000A04F40010B5204800682049884204D031
:1071C0001D4800681E4988422AD11E480078401C8C
:1071D000C0B21C490870032801DD0020087019485E
:1071E0000078012804D11848007801F057FD22E00A
:1071F00014480078022804D11448007801F04EFDAC
:1072000019E010480078032804D11148007801F0F3
:1072100045FD10E00B48007868B901F005FD0AE073
:10722000054800680B49884205D1002005490870CF
:1072300024200DF005F910BD5C0000200A04BC00FC
:107240000A04DC00A8020020B3040020B5040020DA
:10725000B40400200A04F40000B585B02D4800688D
:107260002D49884203D124200DF0EAF850E0294846
:1072700000682A4988421BD1294890F82B01401CFC
:1072800040B2274981F82B01142802DDF12081F852
:107290002B01234890F92B3122A21421684610F0CB
:1072A00077FC01236A463821122002F0CBF82FE048
:1072B000184800681F4988421CD1194890F82B01D2
:1072C000401E40B2164981F82B0110F1140F02DA6A
:1072D0000F2081F82B01124890F92B3111A21421B3
:1072E000684610F055FC01236A463821122002F04E
:1072F000A9F80DE0074800680F49884208D10FA09F
:107300000BF0F2F810A007F063FF24200DF098F8BE
:1073100005B000BD5C0000200A04F4000A04BC00B3
:10732000B8250020D0A3D7BCD6B5A3BA2530336486
:10733000000000000A04DC000A04EC00D5FDD4DAE9
:10734000B1A3B4E600000000534156452056424127
:107350005443414C0000000010B500F025F80B48E4
:1073600000680B4988420ED04FF478610748FEF759
:10737000BEFB07480549086006A010F0F9FB00F0C5
:107380001FF8012010BD0020FCE700007C36002023
:10739000F8DEBC8A466F726D61742046696C6520A8
:1073A00053797374656D210010B5044C4FF4786205
:1073B0000021204612F04AF810BD00007C36002063
:1073C00010B5044C4FF478620021204612F0B4F856
:1073D00010BD00007C3600202DE9F04F0146C1F3BE
:1073E000074CC1F3072801F0FF09DFF85CA000207B
:1073F000002224E09300DFF854B01BF8035003F19F
:10740000010E1BF80E6003F1020E1BF80E40A9EBF3
:107410000505002D00DA6D42A8EB0606002E00DA05
:107420007642ACEB0404002C00DA644205EB060B58
:107430000BEB0407574501DABA461046521CFF2AE7
:10744000D8DDBDE8F08F00003F420F00F478002047
:107450002DE9F04705460E46174698464FF00009BD
:10746000C246002410E0285DB04203D109F10100BA
:1074700000F0FF09B94505D1601C05EB000A504634
:10748000BDE8F087601CC4B22846FEF765FBA04249
:10749000E9D80020F4E7000010B502F01BF912480B
:1074A000007800B910BD1148007800B9FAE710481B
:1074B0000078012800D1F5E70E484079012810D165
:1074C0000C48C079401CC0B20A49C871322808DD96
:1074D0000120C87181F82D03012207A100200BF0C3
:1074E0001FFE00BFDEE70000B000002060010020AA
:1074F000B7010020FC3100204D6F64656D5265635B
:107500007654696D656F7574215265736574204D8D
:107510006F64656D21000000F0B585B054239F2293
:107520002C21002001F054FC012042238022322132
:1075300000901D2001F0F5FC00252048D0F80670D1
:1075400001AE00242CE010223946304611F07EFFB7
:107550009DF80400012807D100208DF804000122C5
:107560003946304611F0E8FF049F0A2094FBF0F101
:1075700000FB114008B902F0ADF80A2094FBF0F1CD
:1075800000FB114050B9012005F11D0203464021C6
:107590000090342001F0F1FC681CC5B2601C84B27C
:1075A000B4F57A7FCFDB0020044948808880084604
:1075B000007820F00100087005B0F0BDF81B002035
:1075C00010B58EB0044644B9032309A2322101A8A4
:1075D00010F0DEFA2046FFF70BFB01A805F0A8F833
:1075E000002201A910460BF09BFD0EB010BD00005B
:1075F00041542B544350434C4F53453D25640D0A91
:107600000000000010B588B004461C48007801282E
:1076100010D11B48007868B901201949087001F0A1
:1076200003FB18A21E21684610F0B2FA68460AF061
:107630005BFF20E01148407801281CD110480078F9
:10764000012818D100200D49087001F0EDFA13A2AD
:107650001E21684610F09CFA68460AF045FF642037
:10766000DFF844C000DF0020054908700349487076
:1076700001200CF0E5FE08B010BD00001C01002048
:1076800029000020D5FDD4DAC9FDBCB6504F43D344
:10769000A6D3C3A1A3A1A3A1A3000000C9FDBCB6AA
:1076A000CDEAB3C900000000198C01082DE9F041B2
:1076B000024600250026002000230024002791F820
:1076C00003C00CF00F0591F803C00CF0100CBCF1D6
:1076D000000F03D091F802C04CEA050591F800C0F4
:1076E000BCF1000F31D0146800202BE04FF0010CEA
:1076F0000CFA00F3B1F800C00CEA03069E4220D158
:1077000083004FF00F0C0CFA03F7BC4305FA03FC9F
:107710004CEA040491F803C0BCF1280F06D14FF0E5
:10772000010C0CFA00FCC2F814C00AE091F803C086
:10773000BCF1480F05D14FF0010C0CFA00FCC2F867
:1077400010C0401C0828D1D31460B1F800C0BCF1AF
:10775000FF0F34DD546800202EE000F1080C4FF0DC
:10776000010808FA0CF3B1F800C00CEA03069E42C7
:1077700021D183004FF00F0C0CFA03F7BC4305FA3C
:1077800003FC4CEA040491F803C0BCF1280F05D1B6
:1077900000F1080C08FA0CF8C2F8148091F803C044
:1077A000BCF1480F07D100F1080C4FF0010808FAAE
:1077B0000CF8C2F81080401C0828CED35460BDE8F5
:1077C000F0810000F0B50A460023002400210025C6
:1077D00000F00046B6F1004F02D11D4EF16901E004
:1077E0001B4E7168C0F3034583B200F44016B6F532
:1077F000401F08D121F07061154E766826F0706642
:10780000134F7E6012E000F48016B6F5801F06D19B
:10781000032606FA05F4A14341F0706106E0460D27
:10782000360103FA06F6B14341F0706122B1460D0C
:10783000360103FA06F6314300F00046B6F1004F78
:1078400002D1034EF16101E0014E7160F0BD000014
:10785000000001400246002093680B400BB101205C
:1078600000E00020704741617047016170470000EF
:1078700008B510208DF8030003208DF802000120C8
:10788000ADF8000069460D48FFF710FF01220CA17A
:1078900000200BF045FC0D48007820F001000B495A
:1078A00008700846007820F0020008700020487038
:1078B000012002490861002008BD000000100140BD
:1078C000475053496E69742E2E2E00004C3500200F
:1078D00010B515480078022800D110BD1348006883
:1078E0001349884217D11048007840B90020114947
:1078F00008700D480078401C0B49087012E00D48D4
:10790000007803280EDDFFF709FA07480078401CCD
:107910000549087006E004480078012802D10020DB
:107920000149087000BFD8E7020100205C00002078
:107930000A04D4006100002010B50446A01DFEF723
:1079400038F910BD2DE9F14FA0B00020159004F0DA
:107950000FFA16A9A348FEF797FD00201490002403
:1079600004E016A8005D14A90855641C032CF8DB7C
:1079700014A8FEF71EF982460020119012900024F0
:1079800005E016A9E01C085C11A90855641C062C2A
:10799000F7DB11A8FEF70DF983464FF47A709BFBD5
:1079A000F0F00590FEF7A7FACDE90C0100228E4B0E
:1079B000DDE90C01FEF730FACDE90C014FF47A70E5
:1079C0009BFBF0F100FB11B0C0EB001080000590B4
:1079D000FEF791FACDE90A010022844BDDE90A01A4
:1079E000FEF71AFACDE90A01DDE90A23DDE90C0107
:1079F000FEF7F9F805460E4600227D4B2846314633
:107A0000FEF798F9CDE902017A490AFB01F0FEF789
:107A100072FACDE90001DDE90223FEF7E4F8CDE9D1
:107A20000401FEF779FA7449886615A96D48001FAC
:107A3000FEF72AFD002404E015A8005D13A90855EF
:107A4000641C032CF8DB13A8FEF7B3F8814600246E
:107A500005E015A9E01C085C0FA90855641C062C5C
:107A6000F7DB0FA8FEF7A5F80E904FF47A710E9889
:107A700090FBF1F00590FEF73EFACDE908010022F7
:107A8000594BDDE90801FEF7C7F9CDE908014FF4CC
:107A90007A710E9890FBF1F201FB1200C0EB00101E
:107AA00080000590FEF727FACDE9060100224F4B32
:107AB000DDE90601FEF7B0F9CDE90601DDE90623AF
:107AC000DDE90801FEF78FF8074688460022484B9B
:107AD00038464146FEF72EF9CDE90201454909FB3A
:107AE00001F0FEF708FACDE90001DDE90223FEF717
:107AF0007AF8CDE90401FEF70FFA3F49C8662098ED
:107B000000286CD13DA13E48FEF72DF8002836D163
:107B10000022374B38464146FEF70CF9CDE9020109
:107B2000FEF7FAF90590CDE90090334890F87030EF
:107B300034A21E2118A810F02BF8012318AA18212E
:107B4000002001F07FFC0022294B28463146FEF739
:107B5000F1F8CDE90201FEF7DFF90590CDE900A0CB
:107B6000254890F871302CA21E2118A810F010F8AA
:107B7000012318AA2821002001F064FC2FE0002234
:107B80001B4B38464146FEF7D5F8CDE90201FEF71A
:107B9000C3F905904B4625A21E21009018A80FF0AE
:107BA000F7FF012318AA1821002001F04BFC002246
:107BB0000F4B28463146FEF7BDF8CDE90201FEF72E
:107BC000ABF9059053461EA21E21009018A80FF095
:107BD000DFFF012318AA2821002001F033FC21B087
:107BE000BDE8F08F082E002000004E4040774B414A
:107BF00080842E4140420F004C350020636E00000F
:107C00009826002020CEB3B6C82025633A20252E22
:107C100033642E253036640020BEADB6C8202563FF
:107C20003A2025642E253036640000004C617469CA
:107C3000747564653A20252E33642E253036640031
:107C40004C6F6E6769747564653A2025642E253023
:107C50003664000070B5054600240DE004EB4401D5
:107C600001EBC402084901EB82002946FDF77BFFC6
:107C700008B9204670BD641C034808384068A0421B
:107C8000ECD84FF0FF30F5E7843600200246002A9A
:107C900001DA0020704702EB420000EBC203064805
:107CA00000EB8300416A002902DB0448814201DDC8
:107CB0000020EFE70846EDE784360020FFEF1F00C5
:107CC00070B5A2B004460E460FAA012120460BF063
:107CD000DAFA01220FA900200BF022FA0FA8FDF713
:107CE00068FF2649C8630FAA022120460BF0CBFA91
:107CF0000FA8FDF75EFF21490870012048700FAA08
:107D0000032120460BF0BFFA01220FA900200BF03F
:107D100007FA242119484230FDF7E9FE0FA9174858
:107D20004230FDF72EFF002014498870887101222F
:107D300013A10BF0F5F915480068A0F5AA706421AD
:107D400048435A21B0FBF1F5114800682B4611A2B7
:107D50003221009002A80FF01BFF00201249A1F869
:107D6000010002A804F0E4FC0A20DFF840C000DFB4
:107D70000FA004F0DDFC002022B070BDFC3100201B
:107D80006C6F67696E206F6B00000000D0000020F0
:107D90004800002041542B504F433D3532322625B8
:107DA000642625640D0A0000B0010020198C01082A
:107DB00041542B504F433D3530390D0A000000002F
:107DC00070B594B004460E4601AA022120460BF07D
:107DD0005AFA0546012201A900200BF0A1F901A8D9
:107DE000FDF7E7FE1349C86301AA012120460BF005
:107DF0004AFA054601A8FDF7DCFE0E49087001AA03
:107E0000032120460BF03FFA0546012201A900207C
:107E10000BF086F9242107484230FDF768FE01A9DE
:107E200004484230FDF7ADFE002002498870887199
:107E300014B070BDFC3100202DE9F04704460D461A
:107E400091469A46A02C01DBA02D02DA0020BDE865
:107E5000F087A4F1A000C6B2A5F1A000C7B2BAF1A4
:107E6000000F10D1781E711E5E2202FB010000EB94
:107E700040004FEAC0080B494B461822486841466B
:107E800006F04CFEE3E7781E711E5E2202FB010045
:107E90004FEA401804494B4620224868414606F004
:107EA0003DFED4E7E8780020DC78002010B5DFF84C
:107EB0004CC100DF52490968884201D2002010BD40
:107EC000DFF838C100DF401C4D4908604D4800789C
:107ED000401CC0B24B490870042801DD0020087026
:107EE0004848007820B902F043FA4749086015E095
:107EF00044480078012804D102F03AFA4349086066
:107F00000CE040480078022804D102F031FA4049E0
:107F1000086003E002F02CFA3E4908603A48006825
:107F20003A49096888420BD13848006838490968DD
:107F3000884205D13648006836490968884201D030
:107F40000020BCE7344800682F490968884219D0EE
:107F50002D48006830490860084600682F4988426B
:107F60000BD001202E49087000202E4908702A48A5
:107F700001682DA00FF0FCFD04E0002028490870E6
:107F80002C4908702648007858B32B48007888B1EF
:107F90002A48007822490978884209D02048007888
:107FA000264908701C48006825490860012086E7BA
:107FB000002084E71A48007820490870214800789A
:107FC00040B9114800681E49086050201D490870DA
:107FD000012074E71B480078401E1A4908700020F1
:107FE0006DE70020174908701448007820B1002080
:107FF00012490870401E62E7002060E77D92010888
:108000008C000020720000207C00002080000020F6
:108010008400002088000020780000200A04FC0072
:1080200073000020610000204B45593D256C780D00
:108030000A0000006000002063000020740000209F
:108040005C0000207100002070B594B004460E461C
:1080500001AA022120460BF016F901A8FDF7A9FD9F
:1080600001281CD12F4988702F480078012802D0A0
:10807000012081F8320300222CA110460BF050F8A9
:1080800001AA012120460BF0FEF801A8FDF791FDA1
:1080900004282AD10120234981F82F0325E001A8D3
:1080A000FDF787FD022820D101AA012120460BF00F
:1080B000EAF801A8FDF77DFD012803D10020194948
:1080C00081F82F03174890F82F0310B900201549A5
:1080D00088700020134981F83203002217A110464E
:1080E0000BF01EF8002014B070BD01AA0321204639
:1080F0000BF0C9F801A8FDF75CFD0A49C1F8A4001E
:1081000001AA052120460BF0BEF8054628210548A6
:108110007C30FDF7ECFC01A902487C30FDF731FD15
:108120000020E0E7FC31002041030020BFAACABCC8
:10813000CBB5BBB02D2D2D2D0D0A0000BDE1CAF829
:10814000CBB5BBB02D2D2D2D0D0A00002DE9F0472C
:10815000002600272E4C0020814653E02DA004F07D
:10816000E7FA322544E04FF4A061A01C04F014FDAE
:1081700080B22080002837D0A01CFDF7EDFC80469F
:1081800026A1A01C04F0EBFA002831D1B8F1070FAA
:108190002EDD04F10C012448FDF7F3FC224F01E031
:1081A0007F1C761C38780A28FAD100201E49885591
:1081B000607D552803D101201C49087009E0607DCD
:1081C000432803D102201949087002E00020174912
:1081D0000870012016490870012216A100200AF03B
:1081E0009FFF0120BDE8F0870A20DFF860C000DFB4
:1081F000281EA5F10105B6D1012215A10AF090FFB4
:108200000020EFE7B9F1320FA8DB00BFEAE700007A
:10821000DA7300204154490D0A0000005265766966
:1082200073696F6E00000000E62600206B010020DD
:10823000A00400205B335D474554204D4F44454D1D
:108240002054797065204F4B200D0A00198C0108CD
:108250005B335D474554204D4F44454D2054797064
:1082600065206661696C65640D0A000000B589B01F
:10827000074890F8270107490B5C07A21E2101A8B7
:108280000FF086FC01A804F053FA09B000BD00000D
:10829000B8250020DD01002061742B7A736E7465AF
:1082A0003D25640D0A0000002DE9F74F90B005460A
:1082B000B7484088052802DB4FF0050902E0B448C2
:1082C00090F802904FF0000B002009904FF47A785C
:1082D0000DF1280A1198012812D1AD48D0F80600F6
:1082E000AB49C1F812000846D0F8061010225046DB
:1082F00011F0ACF8A6490C98C1F80E0000201190BE
:1083000000241298642879D173E0A148D0F8127043
:1083100010223946504611F099F8082207F1100151
:108320000EA811F093F89DF8280001284AD1BBF15E
:10833000000F07D10BF1010000F0FF0B94490C98DE
:10834000C1F80E00DDF82A00C0F344400090DDF8CB
:108350002A10C1F383534FF03F0C0CEA916204EBF7
:10836000041C05F1DE010CEB01008AA10FF024FCD6
:1083700004EB041205F1DE0150180EA9FDF7C2FB53
:108380009DF82900012807D1002104EB041205F112
:10839000DE001044017406E0012104EB041205F133
:1083A000DE00104401747A490D98C1F8120001F101
:1083B000160000EB84000760601CC4B24C4508DB6B
:1083C000264617E07248D0F806007149C1F812003D
:1083D0000FE0A8F101001FFA80F8B8F1000F07D1F3
:1083E000012270A100200AF09BFE264602E005E073
:1083F00000BF8AE700BF0020E880B9E06FE0644872
:10840000D0F80E7010223946504611F01FF808229D
:1084100007F110010EA811F019F89DF828000128A5
:1084200049D1099838B90998401CC0B209905849F7
:108430000D98C1F81200DDF82A00C0F34440009006
:10844000DDF82A10C1F383534FF03F0C0CEA916220
:1084500004EB041C05F1DE010CEB010054A10FF04C
:10846000ABFB04EB041205F1DE0150180EA9FDF779
:1084700049FB9DF82900012807D1002104EB0412D3
:1084800005F1DE001044017406E0012104EB041242
:1084900005F1DE00104401743D490C98C1F80E004E
:1084A00001F1160000EB84000760601CC4B24C456B
:1084B00006DB264614E036490C98C1F80E000EE0A3
:1084C000A8F101001FFA80F8B8F1000F06D10122CF
:1084D0003AA100200AF024FE264601E000BF8EE704
:1084E00000BF0DF1100A304606EBD071C1F3470111
:1084F0000391002436E004EB041105F1DE0008448A
:108500000290701E001B00EB001105F1DE00084414
:108510000190122250460299FDF7D0FA1222DDE9AD
:108520000110FDF7CBFA122251460198FDF7C6FA69
:108530001748163000EB84000768701E011B1448B2
:10854000163000EB810001681148163000EB840002
:108550000160701E011B0E48163000EB81000760A1
:10856000601CC4B203988442C5DBA9F10100E88015
:10857000AE80002085F83801B5F83411B5F8360121
:1085800002F06CFB284602F045FF13B0BDE8F08F07
:10859000F81B0020253032642F253032642F25301F
:1085A000326420005B534D535D65727231000000F0
:1085B00025642F25642F2564200000005B534D5354
:1085C0005D657272320000002DE9F04F87B082467F
:1085D0000E4617464FF000090024A3469AF8000003
:1085E00008B1307818B9002007B0BDE8F08F0FE06F
:1085F00058460BF1010B01A901F80080B8F13D0FBD
:1086000002D0B8F13B0F01D10020EDE7761C641CCD
:1086100096F80080B8F1000F01D0142CE8DB3D2261
:108620002046641C01A90A54002008555046FDF755
:1086300075FA0546254405E0287838706D1C7F1CC6
:1086400009F101092878202805DD28783B2802D087
:10865000B9F1500FF0DD002038704846C4E7000043
:108660002DE9F0474FF000080025234C002639E0A3
:1086700022A004F05DF84FF032092DE04FF4A06124
:10868000A01C04F089FA80B2208008B3A01CFDF77A
:1086900063FA07461DA1A01C04F061F8E0B9072F9A
:1086A0001ADDE11D1B48FDF76CFADFF8688002E077
:1086B00008F101086D1C98F800000D28F8D1002081
:1086C0001449485514A00FF053FA0120BDE8F08773
:1086D0000A20DFF85CC000DFB9F10000A9F1010950
:1086E000CCD1761C322EC3DB012212A100200AF06D
:1086F00017FD0020EAE70000DA73002041542B50F8
:108700004F433D3530380D0A000000003E31323015
:10871000260000003C3500205B325D474554205068
:108720004F435F564552204F4B2D2D25730D0A00A8
:10873000198C01085B325D47455420504F435F560A
:108740004552204641494C440D0A00000021064A8A
:1087500000BF05E013780370401C521C4B1CD9B2BB
:108760000C29F7DB70470000E8F7FF1F03460022E3
:108770002BE04D2903D102F10C0082B221E0412906
:1087800005DB5A2903DC02F1080082B219E06129F5
:1087900005DB7A2903DC02F1080082B211E03029FE
:1087A00005DB392903DC02F1080082B209E0202947
:1087B00005DB602903DC02F1080082B201E0901DB4
:1087C00082B29F2A01DD9F2203E013F8011B0029DA
:1087D000CFD100BFD0B27047F0B589B0074617B906
:1087E000002009B0F0BD06A8FFF7B0FF1BA00FF0F6
:1087F000BFF9002406E006A8015D1BA00FF0B8F940
:10880000601C04B20C2CF6DB19A00FF0B1F90524A2
:1088100008E0300240EA15662D0206A8005D054317
:10882000601E04B2002CF4DAB6B22A46334611A018
:108830000FF09EF913A2102102A8CDE900560FF007
:10884000A7F9002404E002A8005D3855601C04B2BA
:108850000F2CF8DB0020F8730120C2E753544D338E
:10886000322049443D3D00002530327800000000B0
:108870000D0A000074656D703D253031356C6C75E6
:108880000D0A0000253031356C6C7500F0B5A1B0D3
:1088900004460F460EAA012120460AF0F4FC0EA859
:1088A000FDF787F9144908610EAA032120460AF052
:1088B000EAFC06460EA8FDF77CF985B22B460FA20E
:1088C000322101A80FF064F9012201A900200AF069
:1088D00027FC0EAA042120460AF0D5FC06460122F8
:1088E0000EA900200AF01CFC0EA903481530FDF764
:1088F00048F9002021B0F0BDFC310020D3D0D0A732
:10890000C8D5C6DACEAAA3BA25642E2E2E2E2E2EB8
:108910002E0000002DE9F04790B04FF4A57A012118
:108920003B48FDF78DFD00BF02213948FDF7FBFCF8
:108930000028F9D03648FDF7F2FC0646642E0ADA24
:10894000B6F5805F07DB33A00FF012F94FF0FF3070
:1089500010B0BDE8F08732483249096840F821601C
:1089600030480068401C2F490860092801DD0020BC
:108970000860002406E02A4850F8240006A941F8BF
:108980002400641C0A2CF6DB00241CE0002001A952
:1089900041F8240000250FE006A850F8250001A9A1
:1089A00051F82410884206DD06A850F8250001A9D8
:1089B00041F824002F466D1C0A2DEDDB002006A98E
:1089C00041F82700641C042CE0DBDDE9020100EB28
:1089D00001080398C82802DA4FF0FF30B8E71248C0
:1089E0000078012802D14FF4A67A08E00E480078FA
:1089F000022802D140F2531A01E04FF4A57A08FB95
:108A00000AF0C11700EB11514FEA213948469FE7A0
:108A10000024014056444143204F56455200000077
:108A2000581B00200C010020E900002070B5002632
:108A30002148816BC163416B8163016B4163C16AF2
:108A40000163006A1C49C862002504E01A482C3002
:108A500050F825406D1C052DF8DB0520B4FBF0F423
:108A6000154884628068401C134988600846007875
:108A7000C0F3400068B11148006850B108468068F2
:108A80008989884205D300200B4988600AF01CFEC2
:108A900001260B480078401CC0B2094908701E2806
:108AA00009DB002008700548006820B9012205A1F3
:108AB00000200AF035FB70BD4C350020AC010020D1
:108AC0005200002047505320636C6F736500000014
:108AD00010B504461CB100202A49086010BD2A4880
:108AE000C078012832D129480068B8B926480078F2
:108AF00020F00100244908700846007820F00200A8
:108B0000087000204870012221A10AF009FB002012
:108B10002449088001202449486114E01A4800785B
:108B200020F00100184908700846007820F0020083
:108B300008700020487001201B49086101221BA118
:108B400000200AF0EDFA00200F49C870154800888F
:108B500028B11A480FF05CFF002012490880DFF8A6
:108B600060C000DF07490968884200D2B6E7DFF835
:108B700050C000DF643003490860FFF757FF00BFB3
:108B8000ACE70000200100204C350020AC010020A3
:108B90004750532020436C6F73652D2D2D2D2D2DA7
:108BA00000000000800100200010014047505320C9
:108BB000206F70656E2D2D2D2D2D2D00D6270020B8
:108BC0007D92010870B5044600252CB90E48007846
:108BD00001280ED101250CE00C480078012808D1AD
:108BE00001250BA003F0A4FD012209A100200AF039
:108BF00097FA45B106E000200949C8716420DFF802
:108C000024C000DFF7E770BD610100206201002091
:108C100041542B504F433D3630350D0A00000000C3
:108C2000FC310020198C010810B5074802784FF478
:108C3000A0410648FCF754FF8023A02200210846EB
:108C400004F05CFA10BD0000B2040020F47C0020A7
:108C500070B5104802784FF4A0410F48FCF740FF70
:108C600000240EE0002508E0002004EB84010A4AFD
:108C700002EB41114855681CC5B2A02DF4DD601C03
:108C8000C4B2132CEEDB8023A0220021084604F09E
:108C900035FA70BDB2040020F47C002010B5044603
:108CA00022464FF4A0410548FCF71AFF8023A0227A
:108CB0000021084604F022FA10BD0000F47C0020D8
:108CC0002DE9F05F04460D4617469846A02C01DAC0
:108CD000802D01DBBDE8F09FE019A02802DBC4F184
:108CE0009F0087B205EB0800802803DBC5F17F00F9
:108CF0001FFA80F800261AE0A8191FFA80FA4FF030
:108D0000000910E004EB09001FFA80FB0D48007811
:108D10000AEB8A010C4A02EB411101F80B0009F140
:108D200001001FFA80F9B945ECDB701C86B246459C
:108D3000E2DB43463A462946204604F0DFF900BF0D
:108D4000C8E70000B2040020F47C00202DE9F05FA9
:108D500004460D4617469846A02C01DA802D01DB0B
:108D6000BDE8F09FE019A02802DBC4F19F0087B2A4
:108D700005EB0800802803DBC5F17F001FFA80F8AF
:108D8000002619E0A8191FFA80FA4FF000090FE039
:108D900004EB09001FFA80FB0AEB8A010B4A02EB85
:108DA00041110A9801F80B0009F101001FFA80F93E
:108DB000B945EDDB701C86B24645E3DB43463A46D7
:108DC0002946204604F09AF900BFC9E7F47C002048
:108DD0002DE9FC5F04460D4616461F46B44201DCF1
:108DE000BD4201DDBDE8FC9FA02E00DB9F26802F49
:108DF00000DB7F27301B401C1FFA80FB781B401CC8
:108E00001FFA80FA4FF000081EE005EB080080B260
:108E100001904FF0000911E004EB090080B20090CE
:108E20000E480178019800EB80000D4A02EB4012D9
:108E30000098115409F101001FFA80F9D945EBDBC4
:108E400008F101001FFA80F8D045DEDB53465A4690
:108E50002946204604F052F900BFC3E7B2040020BF
:108E6000F47C00202DE9FC5F04460D4616461F46A3
:108E7000B44201DCBD4201DDBDE8FC9FA02E00DB59
:108E80009F26802F00DB7F27301B401C1FFA80FBB2
:108E9000781B401C1FFA80FA4FF000081DE005EB1C
:108EA000080080B201904FF0000910E004EB0900C7
:108EB00080B200900021019800EB80000C4A02EB88
:108EC00040120098115409F101001FFA80F9D945A8
:108ED000ECDB08F101001FFA80F8D045DFDB5346D8
:108EE0005A462946204604F009F900BFC4E70000AD
:108EF000F47C0020F8B507460D4616461C4604B91A
:108F0000F8BDBD4200DAFBE7601EC4B2002000904D
:108F1000301983B22A463146384600F049F800BF7E
:108F2000EEE72DE9F84306460C4617461D46DDF8E8
:108F30002080BE4201DCAC4201DDBDE8F88343463F
:108F4000224639463046FFF7D5FF43462A46394682
:108F50003046FFF7CFFF01204346324629460090B6
:108F6000204600F00AF8012043463A462946009080
:108F7000204600F002F800BFDFE72DE9F843054680
:108F80000E4617461C46DDF820800CB9BDE8F88374
:108F9000AE4200DAFAE7601EC4B2381982B2334634
:108FA00029463846CDF8008000F002F800BFEDE712
:108FB0002DE9FC5F04460D4616461F46B44201DC0F
:108FC000BD4201DDBDE8FC9FA02C01DA802D00DB55
:108FD000F8E7A02E00DB9F26802F00DB7F27301BC9
:108FE000401C80B20090781B401C80B201904FF072
:108FF000000847E005EB08001FFA80FABAF17F0F7E
:1090000001DD4FF07F0A4FF0000B34E004EB0B0062
:109010001FFA80F9B9F19F0F01DD4FF09F090C98FD
:10902000012819D0022802D0032814D109E01B48D6
:1090300000780AEB8A011A4A02EB411101F8090093
:1090400014E0184800780AEB8A01154A02EB411136
:1090500001F809000AE000BF134800780AEB8A0112
:109060000F4A02EB411101F8090000BF00BF0BF1EC
:1090700001001FFA80FB00988345C7DB08F101005F
:109080001FFA80F801988045B4DB29462046DDE9C7
:10909000002304F033F800BF94E70000B004002080
:1090A000F47C0020B5040020B104002010B519A004
:1090B00000F082FA18B917A118A00EF059FD1FA0F0
:1090C00000F07AFA18B91DA114A00EF051FD1DA0F0
:1090D00008F0CEF84FF47F026FF07F411C4800F09B
:1090E00099F84FF47F00FEF777F91A490870FF20CE
:1090F000FEF772F9184908704FF47F40FEF76CF9DB
:10910000164908701248FEF767F91549087001F012
:10911000A7F910BD485A4B313600000043616E2755
:10912000742066696E642074686520487A6B4669AD
:109130006C6528257329210D0A000000485A4B311F
:10914000320000006C6F676F2E626D7000000000CF
:10915000D1880200B3040020B4040020B50400202C
:10916000B60400202DE9F05F04460D4691469A466C
:1091700004EB0900A02803DBC4F1A0001FFA80F96A
:1091800005EB0A00802803DBC5F180001FFA80FA96
:1091900000262EE0A81987B24FF0000B25E004EB63
:1091A0000B001FFA80F807EB8700174901EB40100E
:1091B00010F8080015490978884209D11448007848
:1091C00007EB8701104A02EB411101F8080008E0A3
:1091D0000E48007807EB87010B4A02EB411101F8BA
:1091E00008000BF101001FFA80FBCB45D7DB701C98
:1091F00086B25645CEDB53464A462946204603F002
:109200007DFFBDE8F09F0000F47C0020B204002048
:10921000B104002070B506460C4615463046FEF7F0
:10922000DBF8074908702046FEF7D6F805490870B4
:109230002846FEF7D1F8044908700DF015FD70BD01
:10924000B1040020B2040020B00400202DE9F84F42
:1092500005460E461746984608F00F0908F0F00A32
:10926000B9F1010F09D0B9F1020F21D0B9F1030F03
:1092700039D0B9F1040F6CD150E0002415E0012081
:1092800006EB040C1FFA8CF305EB040C1FFA8CF2AE
:10929000A6EB040C1FFA8CF105EB040C00901FFAEE
:1092A0008CF0FFF73EFE601C84B2BC42E7DB51E06D
:1092B000002415E0012006EB040C1FFA8CF3A5EB4B
:1092C000040C1FFA8CF2A6EB040C1FFA8CF1A5EB30
:1092D000040C00901FFA8CF0FFF723FE601C84B290
:1092E000BC42E7DB36E0002415E0012006EB040C6D
:1092F0001FFA8CF305EB040C1FFA8CF206EB040C3E
:109300001FFA8CF1A5EB040C00901FFA8CF0FFF70C
:1093100008FE601C84B2BC42E7DB1BE0002415E0C1
:109320000120A6EB040C1FFA8CF305EB040C1FFACA
:109330008CF2A6EB040C1FFA8CF1A5EB040C009048
:109340001FFA8CF0FFF7EDFD601C84B2BC42E7DB36
:1093500000E000BF00BFBDE8F88F00002DE9F04F2E
:10936000ADB081460F4690464046FEF773FC8346FB
:109370005846FEF78BFC8246BAF1000F02D12DB0A1
:10938000BDE8F08F2CAB02221C21584605F0C6FB2D
:10939000BDF8B000082800D0F1E72BAB0422122161
:1093A000584605F0BBFB2AAB04221621584605F0AF
:1093B000B5FB2B98A02802D82A98802800D9DEE790
:1093C00029AB04220A21584605F0A8FB1C4B4FF498
:1093D00080623621584605F0A1FB2B9800F003046B
:1093E000002C07DD2B9800F00300C0F104002B993E
:1093F000451800E02B9D2A98461E002413E029986A
:1094000005FB060101AB58462B9A05F087FB01A826
:1094100000902B9882B2381981B20123484604F09B
:1094200045F8761E641C2A988442E8D32A9883B2B1
:109430002B9882B23946484603F060FE00BF9EE793
:10944000F47800202DE9FF4F83B0804693461F46F5
:1094500007F0F0000290029820B94FF00C090126A5
:10946000CA4604E04FF0100901264FF0100A5C468E
:10947000002523E020789F280DDD0097637822786F
:1094800008EB050188B2049903F0AAFE05EB090078
:1094900085B2A41C12E00097237808EB050188B27E
:1094A0000022049903F09CFE029818B905EBC6004F
:1094B00085B202E005EBC60085B2641C2078002866
:1094C000D8D153462A464046049903F017FE07B008
:1094D000BDE8F08F2DE9FF4F85B0804693461F46CB
:1094E00007F0F0000490049820B94FF00C09012611
:1094F000CA4604E04FF0100901264FF0100A5C46FE
:1095000000252BE020789F2811DDDDE91210CDE940
:10951000007102906378227808EB050188B2069901
:1095200003F014FF05EB090085B2A41C16E0DDE989
:109530001210CDE900710290237808EB050188B282
:109540000022069903F002FF049818B905EBC60043
:1095500085B202E005EBC60085B2641C20780028C5
:10956000D0D153462A464046069903F0C7FD09B0BC
:10957000BDE8F08F03494A694A640A690A6481F8C0
:109580003C007047C00E002004480268044801886F
:1095900004A00EF0EDFA00BFFEE70000D8000020A6
:1095A000D40000200D0A5B4846485D463D25642CEA
:1095B0004C3D25640000000070B505462C4840680D
:1095C00008B9002070BD2BA12846FCF7CCFA58BB87
:1095D0002A4800210160416081602846FEF73AFB7D
:1095E0000446002C01DA0020ECE710202349087023
:1095F00048700978214A527801FB02F0C11700EB4C
:109600005171C1F3C7011D4A91701046446004EBCB
:10961000440000EBC4011648083000EB8100406AAA
:10962000114688600120CDE715A12846FCF79BFA7A
:10963000D8B9154800210160416081602846FEF7D5
:1096400009FB0446002C01DA0020BBE70E48446009
:1096500004EB440000EBC4010548083000EB810036
:10966000406A094988600120ACE700BFAAE7000012
:109670007C360020485A4B3136000000DC78002050
:10968000485A4B3132000000E878002010B50446FB
:109690000121C80204F090FF7D2005F025F808B1F3
:1096A00004F0AAFF45F2555000F028F8062000F01B
:1096B00019F8A0B200F01CF800F00CF800F002F865
:1096C00010BD00004CF6CC40014908607047000016
:1096D000003000404AF6AA200149086070470000A7
:1096E00000300040014948607047000000300040F1
:1096F000014988607047000000300040014908605F
:1097000070470000003000402DE9F04FADF26C4D85
:1097100082460E4600200090012E01D1804609E0CD
:10972000022E02D14FF4001804E001200DF26C4D1E
:10973000BDE8F08F00250027AB460DF2044001F094
:10974000F9FF00BF24480069401BB0F5806F02D3C9
:109750004FF4806906E02048008A401B1FFA80F918
:109760004FF0010B08EB07014A4601A80FF06EFE0F
:10977000009860B90098401CC0B2009000208DF89D
:1097800004008DF805008DF806008DF807004D44A3
:109790004F444A4601A90DF2044001F0DDFFBBF140
:1097A000000FCFD00DF2044001F05CFF002409E06F
:1097B0001AF804100DF25C40005D814200D003E015
:1097C000601C84B2102CF3DB00BF102C01DA0120E6
:1097D000ACE70020AAE70000C00E002070B58AB0F8
:1097E00004460D4600200C4908702A46214601A86F
:1097F00003F0A4FB0646232E06D9012207A1002070
:1098000009F08EFC0AB070BD324601A9032001F0B8
:10981000BFFE00BFF6E700002400002074786275E8
:1098200066206F766572210010B588B000200B4964
:109830000870684603F0FCFB04461D2C06D9012283
:1098400007A1002009F06CFC08B010BDA2B2694667
:10985000032001F09DFE00BFF6E700002400002079
:109860007478627566206F76657221000021016050
:1098700041608160C160491E0161704709480078FC
:10988000FF2804DA07480078401C0649087006489B
:109890000078FF2804DA04480078401C0249087068
:1098A00070470000600000206100002010B586486D
:1098B000007827280BD1122350224A214020FFF79D
:1098C000FFF9012381A24A214020FFF7BBFD7E481A
:1098D0000078012820D17E48007801281CD17D48DD
:1098E00000687D49884213D07A4800687B498842E5
:1098F0000ED0784800687A49884209D075480068D7
:109900007849884204D0734800687749884203D177
:1099100001207649087010BD6E4800686E49891FA5
:1099200088422AD1012272A1002009F0F9FB774870
:1099300090F83C0318B9002075490870C2E0002077
:109940007449087071498871DFF8CCC100DF1430A8
:1099500072490860724800780028EFD101207149EF
:10996000087071A002F0E4FE01226FA1002009F04E
:10997000D7FB002070490870A4E0564800686F4982
:10998000884225D101226EA1002009F0C9FB0020E8
:10999000694908706E480078022815DA6D48007829
:1099A00008B9012000E000206A49087008460078E4
:1099B000012804D101026848FDF757FF04E04FF485
:1099C00080716548FDF74FFF00206149087079E01C
:1099D000404800684049884207D100205649087035
:1099E00001225EA109F09CFB6CE03A4800686049E6
:1099F000884208D101225FA1002009F091FB0020DC
:109A00006149087087E733480068604988421DD182
:109A100000205F49087008460078022810DA2C48B8
:109A2000007868B928480078012809D15948007899
:109A3000012802D002200AF003FD002055490870D9
:109A4000012255A1002009F06BFB64E72148006862
:109A50002249884207D1002055490870012255A1AA
:109A600009F05EFB57E71B4800681D49884205D195
:109A7000012256A1002009F053FB23E0154800689D
:109A80001849884205D1012255A1002009F048FB60
:109A900018E0104800685849884209D100200D4953
:109AA000086056490870012255A109F039FB09E008
:109AB000084800680C49884204D1012256A10020C0
:109AC00009F02EFB00BF26E741030020CEDE000098
:109AD000C30000205C0000200804FC000A04F4001D
:109AE0000A04BC000A04DC000A04F800C4000020D8
:109AF0005B4B45595F5050542F4B45595F50505464
:109B00005F4D494320467265655D0000FC310020D1
:109B1000C5000020640000207D920108E0000020C4
:109B2000BC000020C900002041542B504F433D355C
:109B3000333826320D0A0000630000200A047C003E
:109B40005B4B45595F494E464F20467265655D0047
:109B5000BE00002003010020000C01405B4B455972
:109B60005F46554E435F503220467265655D00008A
:109B70002A00FC005B4B45595F534F535F4F4B200E
:109B8000467265655D000000BD0000200A04EC001F
:109B9000C2000020C80000205B4B45595F50414E79
:109BA000454C5F4D454E5520467265655D00000091
:109BB000C70000205B4B45595F50414E454C5F4507
:109BC00058495420467265655D0000005B4B45595D
:109BD0005F50414E454C5F555020467265655D00B3
:109BE0005B4B45595F50414E454C5F444F574E20AB
:109BF000467265655D0000000A04D400C1000020C3
:109C00005B4B45595F455849545F444F574E5F473A
:109C10005420467265655D005B4B45595F46554E65
:109C2000435F503320467265655D000008B5012131
:109C3000084604F0D1FC01214348FDF7C3FD012192
:109C40001C2004F0C9FC012003F03CF9002004F0C2
:109C500069FD0020FCF722FD48208DF80300032059
:109C60008DF802000820ADF8000069463748FDF77E
:109C70001DFD2020ADF8000069463548FDF716FDB2
:109C80004020ADF8000069463148FDF70FFD802007
:109C9000ADF8000069462E48FDF708FD0820ADF834
:109CA000000069462A48FDF701FD1020ADF80000CC
:109CB00069462748FDF7FAFC0420ADF80000694624
:109CC0002348FDF7F3FC0220ADF8000069461F4869
:109CD000FDF7ECFC4FF48060ADF8000069461B48CE
:109CE000FDF7E4FC10208DF803000001ADF8000042
:109CF00069461748FDF7DAFC04208DF80300C0021E
:109D0000ADF8000069461148FDF7D0FC04208DF83D
:109D100003002020ADF8000069460C48FDF7C6FCA2
:109D200010208DF803008002ADF800006946074856
:109D3000FDF7BCFCFCF7FEFC002006490870AC21D6
:109D40000E2005F0E3F908BD0002300000100140CC
:109D5000000C01406300002010B58AB00024FA48CE
:109D6000007801281ED1F948007801281AD1F84856
:109D70000068F849884213D0F5480068F6498842DF
:109D80000ED0F3480068F549884209D0F0480068D1
:109D9000F349884204D0EE480068F249884201D174
:109DA0000AB010BDE848007801280DD1E8480068E5
:109DB000E849891F884207D0EB480078012803D181
:109DC0000020E9490870EBE70BF01EFCE048E24A8E
:109DD000083A0168881A914272D01ADCE34AA1EB72
:109DE000020091426DD00DDCE148084400285FD0AC
:109DF000A0F54010203800287ED0DE490844002815
:109E000040D146E1B0F5002F77D0B0F5C01FF7D1B3
:109E1000E3E0D94A811A904270D00BDC08286ED05A
:109E2000A0F58020083800286AD0A0F2244000283D
:109E3000E6D14AE1B1F5767F04D0A1F2DE31002906
:109E4000DED13FE0CD4890F83C0388B9CC4800789B
:109E5000401CC0B2CA490870022823DD0120C9494C
:109E600008700020C649087024200AF0E9FA19E0B9
:109E70000120C5490870DFF814C300DFC449096830
:109E8000884200D25CE1C348007858B9C2480078E3
:109E900010B10020C0490870C0A002F049FCBFA06A
:109EA0000DF066FE0122C1A1002009F039F947E159
:109EB0000020B54908700122C3A109F031F93FE142
:109EC00028E1F2E00122C5A1002009F029F9C848E3
:109ED00090F82D010B281ADAC6480078B8B1C448AA
:109EE00090F82D01401CC24981F82D01084690F8D8
:109EF0002D31C1A21E2104E0EDE0D0E0F1E0A0E0B0
:109F000029E002A80DF044FE02A802F011FCB848B6
:109F100090F82D11BCA00DF02BFEB54890F82D3116
:109F2000C0A21E2102A80DF033FE87480078012848
:109F30000AD1BEA250210520FFF710FA112302AA70
:109F400050211A20FFF77EFA0120AA49087000204C
:109F5000B9490870F4E0A64890F82D01002814DDF6
:109F6000A448007888B1A24890F82D01401EA0496D
:109F700081F82D01084690F82D319FA21E2102A8DC
:109F80000DF006FE02A802F0D3FB994890F82D11BF
:109F90009DA00DF0EDFD964890F82D31A1A21E2157
:109FA00002A80DF0F5FD6848007801280AD19FA2AB
:109FB00050210520FFF7D2F9112302AA50211A20BF
:109FC000FFF740FA01208B49087000209A49087079
:109FD00001229AA109F0A4F8B2E09D480078401C43
:109FE000C0B29B490870022825D16648007810BB92
:109FF00098480078F8B95548007818B100205349BE
:10A00000087002E00120514908705048007801288A
:10A0100005D191A26E214820FFF7A0F90BE00120A5
:10A0200090490870904800787F2359226E21009053
:10A030004820FEF7BDFF01228CA1002009F070F836
:10A040007EE001228FA1002009F06AF89348007891
:10A05000401CC0B291490870022819DD012290A16C
:10A06000002009F05DF891A008F03EFA0120924925
:10A070000860FFF72FFB6420DFF840C200DF0120FB
:10A080008D49091D086004208D49486100BFFEE725
:10A0900056E001228BA1002009F042F850E0012295
:10A0A0008EA1002009F03CF84AE092480078401C5C
:10A0B000C0B290490870032801D1FCF72FFE01229D
:10A0C0008DA1002009F02CF83AE0012291A1002096
:10A0D00009F026F834E0012295A1002009F020F8CB
:10A0E0002EE0012298A1002009F01AF89B48007880
:10A0F000401C9A49087008460078032809D10120BD
:10A100001E4981F82F0396A002F012FB01200AF0ED
:10A1100097F915E0194890F83C0380B91848007881
:10A12000401CC0B216490870022808DD01201549FC
:10A13000087000201249087024200AF081F900BF3D
:10A1400000BF00BF2CE6000041030020C300002038
:10A150005C0000200804FC000A04F4000A04BC00AF
:10A160000A04DC000A04F800C10400200A04D40038
:10A17000F6FB83FF2000F0FF28FC0700FC310020E5
:10A18000C500002062010020630000207D920108CC
:10A19000E0000020BC000020C900002041542B50EA
:10A1A0004F433D35333826310D0A00005B4B45598E
:10A1B0005F5050542F4B45595F5050545F4D4943A9
:10A1C0002050726573735D005B4B45595F494E4685
:10A1D0004F2050726573735D000000005B4B455962
:10A1E0005F46554E435F50322050726573735D0079
:10A1F000B8250020CA00002041542B504F433D3663
:10A2000030372625640D0A0073757450726F6475BB
:10A210006374506172612E566F6C4C763D3D2564BF
:10A220000D0A00002530326400000000766F6C7566
:10A230006D652E626D700000CB0000205B4B4559B0
:10A240005F46554E435F50332050726573735D0017
:10A25000C2000020B70100206C6F636B2E626D702E
:10A2600000000000C8000020B60400205B4B4559E8
:10A270005F50414E454C5F4D454E552050726573C1
:10A28000735D00005B4B45595F50414E454C5F4547
:10A290005849542050726573735D0000C700002058
:10A2A0005077724F66664F6B00000000D5FDD4DA20
:10A2B000B9D8BBFA21000000100C0140198C01082C
:10A2C000001001405B4B45595F50414E454C5F5576
:10A2D000502050726573735D000000005B4B455960
:10A2E0005F50414E454C5F444F574E20507265734E
:10A2F000735D0000C10000205B4B45595F45584924
:10A30000545F444F574E5F47542050726573735DDE
:10A31000000000005B4B45595F50315F50335F5583
:10A3200050444154452050726573735D0000000035
:10A330005B4B45595F4F4B5F444F574E5F47505300
:10A340002050726573735D005B4B45595F534F53EB
:10A350005F4F4B2050726573735D0000BD0000209D
:10A3600041542B504F433D3533390D0A0000000056
:10A370000648016801F0FC0109040548826840F2C2
:10A380000A40024041EA020070470000080C014008
:10A390000010014009490978094A117030B1802143
:10A3A000084A51610121054A117005E08021054AE2
:10A3B00011610021014A117070470000C1040020A2
:10A3C000C20400200010014010B504462146054893
:10A3D00004F0BEFE00BF0221024804F0ADFE0028DA
:10A3E000F9D010BD0038004010B504462046FFF7F4
:10A3F000EBFF10BD2DE9F05F04460D4616461F46E3
:10A40000A046B146AA46BB462A2000F0BFF94FEA53
:10A41000282000F0CFF908F0FF0000F0CBF94FEA58
:10A42000292000F0C7F909F0FF0000F0C3F92B2044
:10A4300000F0ACF94FEA2A2000F0BCF90AF0FF0066
:10A4400000F0B8F94FEA2B2000F0B4F90BF0FF0050
:10A4500000F0B0F92C2000F099F9BDE8F09F000061
:10A4600070B5164800880412144805787F239F228F
:10A4700000210846FFF7BEFF00201149086017E0E1
:10A480000020104908600AE0204600F093F92846B1
:10A4900000F090F90B480068401C0A490860094820
:10A4A0000068A028F0DB06480068401C04490860EA
:10A4B000034800688028E3DB70BD0000C40400206E
:10A4C000C8040020CC04002010B500F0FDF8802066
:10A4D0007C494861402008610120FCF7B4FA402023
:10A4E000784948610120FCF7AEFA402075490861BF
:10A4F0007820FCF7A8FA112000F048F97820FCF742
:10A50000A2FAB12000F042F9052000F053F93C20F6
:10A5100000F050F93C2000F04DF9B22000F036F97F
:10A52000052000F047F93C2000F044F93C2000F001
:10A5300041F9B32000F02AF9052000F03BF93C2056
:10A5400000F038F93C2000F035F9052000F032F930
:10A550003C2000F02FF93C2000F02CF9B42000F052
:10A5600015F9032000F026F9C02000F00FF928208B
:10A5700000F020F9082000F01DF9042000F01AF97D
:10A58000C12000F003F9C02000F014F9C22000F04F
:10A59000FDF80D2000F00EF9002000F00BF9C320AB
:10A5A00000F0F4F88D2000F005F92A2000F002F9FF
:10A5B000C42000F0EBF88D2000F0FCF8EE2000F055
:10A5C000F9F8C52000F0E2F81A2000F0F3F8362080
:10A5D00000F0DCF8A02000F0EDF8E02000F0D6F864
:10A5E000042000F0E7F8222000F0E4F8072000F053
:10A5F000E1F80A2000F0DEF82E2000F0DBF8302031
:10A6000000F0D8F8252000F0D5F82A2000F0D2F884
:10A61000282000F0CFF8262000F0CCF82E2000F003
:10A62000C9F83A2000F0C6F8002000F0C3F8012075
:10A6300000F0C0F8032000F0BDF8132000F0BAF8D5
:10A64000E12000F0A3F8042000F0B4F8162000F098
:10A65000B1F8062000F0AEF80D2000F0ABF82D2088
:10A6600000F0A8F8262000F0A5F8232000F0A2F8BA
:10A67000272000F09FF8272000F09CF8252000F00C
:10A6800099F82D2000F096F83B2000F093F8002078
:10A6900000F090F8012000F08DF8042000F08AF816
:10A6A000132000F087F83A2000F070F8052000F041
:10A6B00081F8292000F06AF84FF6FF71002000F0C1
:10A6C0008DF810BD0010014000B587B001211820A1
:10A6D00003F082FF0121880303F06EFF4FF4A040D6
:10A6E000ADF8040003208DF8060010208DF8070057
:10A6F00001A92348FCF7DAFF4FF42040ADF804002D
:10A7000003208DF8060018208DF8070001A91C48C9
:10A71000FCF7CCFFC020ADF8040010208DF8070036
:10A7200001A91848FCF7C2FF4020164908618020A3
:10A7300008614FF44040ADF808004FF48270ADF866
:10A740000A000020ADF80C000220ADF80E00012038
:10A75000ADF810004002ADF812000020ADF8140072
:10A76000ADF816000720ADF8180002A9064804F05D
:10A77000F1FC0121044804F0D3FC07B000BD000047
:10A78000000C0140001001400038004010B50446A4
:10A790004FF4805006490860800008602046FFF7AB
:10A7A00023FE4FF480500249091F086010BD0000CD
:10A7B000140C014010B504464FF48050064908605F
:10A7C0008000091F08602046FFF70EFE4FF48050FE
:10A7D0000149091F086010BD140C0140024A108095
:10A7E000024A118070470000C6040020C404002003
:10A7F00008B50121084603F0EFFE01211648FCF7D9
:10A80000E1FF01213C2003F0E7FE10208DF803005A
:10A8100003208DF802004FF48050ADF80000694627
:10A820000E48FCF743FF0420ADF8000069460C48D1
:10A83000FCF73CFF4FF48070ADF800006946094812
:10A84000FCF734FF4FF480500449086104200449A8
:10A850001031086008BD0000000230000010014007
:10A8600000140140000C014010B5044696210C2054
:10A8700004F04CFC0CB300206B4908606B49087075
:10A880006B4908706B490870FF206B4908706B4971
:10A89000087000206A4908706A4908706A4908709F
:10A8A000FF206A4908706A4908704FF4805069496E
:10A8B000086104206849086010BDDFF8A0C100DF0E
:10A8C00059490968884200D2F6E7DFF890C100DFF5
:10A8D0000F30554908606248007820B94FF4805025
:10A8E0005C49086149E05F48007820B94FF4805026
:10A8F0005849486141E050480078594909788842F0
:10A9000005D14E48007857490978884219D000206F
:10A91000464908704A49087051480078464908700D
:10A9200050480078454908704D4800784006000EB0
:10A930004049087041480078097801EB40003C49E3
:10A9400008703A480078401CC0B23849087038494D
:10A950000978884202DD00203449087033480078C5
:10A9600034490978884204DA4FF480503949486103
:10A9700003E04FF48050374908613B48007818B92C
:10A9800004203549086048E03848007820B90420A0
:10A990003149091D086040E02C48007832490978A7
:10A9A000884205D12A48007830490978884219D070
:10A9B00000201E490870224908702B48007823495E
:10A9C00008702A4800782249087027480078400615
:10A9D000000E1D4908701E480078097801EB400000
:10A9E0001849087016480078401CC0B21449087015
:10A9F00014490978884202DD002011490870104886
:10AA0000007811490978884204DA04201249091DA6
:10AA1000086002E0042010490860E5210C2004F0E1
:10AA200075FB00BF48E700009C000020A00000204C
:10AA3000A1000020A2000020A3000020A40000200C
:10AA4000A5000020A6000020A7000020A8000020EC
:10AA5000A900002000100140101401407D9201085F
:10AA60009400002095000020960000209700002010
:10AA70002DE9F0470446884691461E46DDF820A0A1
:10AA8000C4F80080002507E0206850F8250007780A
:10AA900007B903E0681CC5B2C82DF5DB00BF681E0E
:10AAA000C5B2681CA080052095FBF0F0608160892C
:10AAB000052190FBF1F201FB120010B16089401CEE
:10AAC00060810025C4F8D8600AE006B90AE0D4F82D
:10AAD000D80050F82500077807B903E0681CC5B214
:10AAE000C82DF2DB00BFA4F8DC5000250EE0A088E2
:10AAF000A84205DD1AF8051004F10D00415503E0E8
:10AB0000002104F10D004155681CC5B2C82DEEDBD3
:10AB100084F80C9000202081E080054890F83003F4
:10AB20000449C880204600F019FABDE8F08700000B
:10AB3000FC3100200C2F00202DE9F05F05468846EF
:10AB400091461E46DDE90AABC5F80080002407E007
:10AB5000286850F82400077807B903E0601CC4B2E5
:10AB6000C82CF5DB00BF601EC4B2601CA8800520A5
:10AB700094FBF0F068816889052190FBF1F201FBFC
:10AB8000120010B16889401C68810024C5F8D860A3
:10AB90000AE006B90AE0D5F8D80050F82400077892
:10ABA00007B903E0601CC4B2C82CF2DB00BFA5F8F3
:10ABB000DC40002416E0A888A0420ADD1BF804103F
:10ABC00005F2391001551AF8041005F10D00015570
:10ABD00006E0002105F23910015505F10D0001557F
:10ABE000601CC4B2C82CE6DB85F80C9000202881DC
:10ABF000284600F0E1FBBDE8F09F2DE9F047044650
:10AC00000F4616469846A4F834710120A4F8360180
:10AC10000020E08084F80C800025C4F8D8600DE0A6
:10AC200006B90DE0D4F8D80050F8250090F800904F
:10AC3000B9F1000F00D103E0681CC5B2C82DEFDBED
:10AC400000BFA4F8DC50642084F8330164220121A1
:10AC50002046FDF729FBBDE8F08700002DE9FF4104
:10AC600006460F460A2E01DA012409E0642E01DAB5
:10AC7000022405E0B6F57A7F01DA032400E004241B
:10AC80000A2F01DA012509E0642F01DA022505E027
:10AC9000B7F57A7F01DA032500E00425334610A2D8
:10ACA0000B2101A800970CF073FF60190E49098869
:10ACB000884208D060190C490880102338220121ED
:10ACC0005020FDF7FDFF6119891CC900C1F1A001E9
:10ACD00088B2012301AA1946FEF7B4FBBDE8FF8143
:10ACE00025647C2564000000AC04002070B5044697
:10ACF000A08810B92548006870BD24480068244920
:10AD0000084418B1B0F5001F3AD11CE0204600F00D
:10AD10007FF9E08818B9A088401EE08002E0E08852
:10AD2000401EE080257AE088052190FBF1F020812B
:10AD30002089A84203D0204600F010F902E0204606
:10AD400000F066F91FE0204600F062F9E088401C40
:10AD5000E080E088A188884201DB0020E080257A3D
:10AD6000E088052190FBF1F020812089A84203D0E2
:10AD7000204600F0F3F802E0204600F049F902E036
:10AD800002480068B8E700BF0020B5E75C0000207B
:10AD9000F6FB43FF70B50446A08810B9254800684B
:10ADA00070BD244800682449084418B1B0F5001F5C
:10ADB0003AD11CE0204600F048F9E08818B9A08894
:10ADC000401EE08002E0E088401EE080257AE088B6
:10ADD000052190FBF1F020812089A84203D0204674
:10ADE00000F0EAFA02E0204600F02FF91FE02046CA
:10ADF00000F02BF9E088401CE080E088A1888842C0
:10AE000001DB0020E080257AE088052190FBF1F04D
:10AE100020812089A84203D0204600F0CDFA02E02C
:10AE2000204600F012F902E002480068B8E700BFCF
:10AE30000020B5E75C000020F6FB43FF10B5044698
:10AE4000A08810B94348006810BD424800684249D4
:10AE5000084430B1B0F5001F39D0B0F5601F72D191
:10AE60006EE0204600F008F9B4F83601401EA4F860
:10AE70003601B4F8360118B9B4F83401A4F8360133
:10AE8000E08880B9B4F83401052808DD7522002176
:10AE90002046FDF709FA012084F8380106E0A08871
:10AEA000401EE08002E0E088401EE08094F8380117
:10AEB00018B1002084F8380102E0204600F0DCF8E8
:10AEC000B4F83411B4F83601FFF7C8FE3EE020466E
:10AED00000F0D2F8E088401CE080B4F83601401C55
:10AEE000A4F83601B4F83601B4F83411884202DD12
:10AEF0000120A4F83601E088A18888420EDBB4F86E
:10AF00003401052808DD642200212046FDF7CCF934
:10AF1000012084F8380101E00020E08094F8380135
:10AF200018B1002084F8380102E0204600F0A4F8AF
:10AF3000B4F83411B4F83601FFF790FE06E002E0F1
:10AF40000448006880E7034800687DE700BF0020F0
:10AF50007AE700005C000020F6FB43FF2DE9F0419A
:10AF60000446A08808B9BDE8F081207A00EB800093
:10AF7000C7B23D4619E0A088A84210DC052095FB29
:10AF8000F0F100FB1150182101EB00101FFA80F8BE
:10AF90001023902241460020FDF792FE03E029464F
:10AFA000204600F080F8681CC5B2781D8542E2DBBF
:10AFB000204600F02DF88F262089002808DD06F1B4
:10AFC000080188B2032308221821FEF73FF905E0A3
:10AFD0000823102218213046FDF772FE4FF0680852
:10AFE00021896089401E814208DA06F1080188B291
:10AFF000042308224146FEF729F907E0A8F10800DA
:10B0000081B2082310223046FDF75AFE00BFAAE79E
:10B010002DE9F04104460026D4F8D80010B106F11D
:10B020001000C6B2E088052190FBF1F201FB12008E
:10B03000C5B2182000EB0510C7B20E237E22394698
:10B040003046FEF78FF8BDE8F0812DE9F041044667
:10B050000027E088052190FBF1F201FB1200C5B248
:10B06000182000EB0510C6B20E23A02231460020A6
:10B07000FEF778F8BDE8F0812DE9F041044600269E
:10B08000D4F8D80010B106F11000C6B2A579182086
:10B0900000EB0510C7B20E237E2239463046FEF77C
:10B0A00061F8BDE8F0812DE9F0438BB004460D4610
:10B0B000052095FBF0F100FB115087B20026182007
:10B0C00000EB07101FFA80F910238E224946304604
:10B0D000FDF7F6FD142106A8FAF709FD207B50B113
:10B0E000206850F82520142106A808F0CAF800208E
:10B0F0008DF82B0009E0206850F82510142206A8CE
:10B10000FAF71EFD00208DF82B00112206A901A8D8
:10B1100008F084F8D4F8D800A0B104F10D0010F8BC
:10B120000580D4F8D80050F8282049463046FEF76C
:10B1300015F906F1100188B2012301AA4946FEF76C
:10B1400081F905E0012301AA49463046FEF77AF964
:10B150000BB0BDE8F08300002DE9F04F9DB0044630
:10B160000D46052095FBF0F100FB11501FFA80F908
:10B170004FF00008182000EB091080B21C9010233B
:10B18000A02240461C99FDF79BFD142117A8FAF751
:10B19000AEFC207B50B1206850F82520142117A860
:10B1A00008F06FF800208DF86F0009E0206850F873
:10B1B0002510142217A8FAF7C3FC00208DF86F00A1
:10B1C0000C2217A912A808F029F812A8FAF7C4FC53
:10B1D00086B212A8FDF7CAFA86B2D4F8D8000028C1
:10B1E0005BD004F10D00475D04F2391010F805A0A2
:10B1F00053462EA20A210FA80CF0CAFC0FA8FAF79A
:10B20000ABFC83465B462AA2322102A800960CF0D2
:10B21000BFFC012202A9002007F082FFD7B9012359
:10B2200012AA40461C99FEF70DF9D4F8D81051F82F
:10B23000272008EB0601491C88B21C99FEF78EF8FE
:10B2400008EB0601213188B201230FAA1C99FEF7F1
:10B25000F9F828E00FA8FAF77FFC0146C6F17B0059
:10B26000A0EBC1001FFA80FB01230FAA58461C99CE
:10B27000FEF7E8F8D4F8D81051F82720C6F17B0182
:10B2800088B21C99FEF76AF8C6F19B0188B20123C7
:10B2900012AA1C99FEF7D6F805E0012312AA40462F
:10B2A0001C99FEF7CFF81DB0BDE8F08F256427008C
:10B2B00074696D65206C656E3D3D3D3D3D3D3D3D98
:10B2C00025642C2C2C2C2C6C656E323D3D3D3D258F
:10B2D000640D0A002DE9F0438BB004460D460520AD
:10B2E00095FBF0F100FB11501FFA80F800271820A1
:10B2F00000EB08101FFA80F910238E2249463846C9
:10B30000FDF7DEFC142106A8FAF7F1FB207B60B103
:10B3100005EB051104F1DE000A18142106A807F058
:10B32000B0FF00208DF82B000BE005EB051204F1B7
:10B33000DE001118142206A8FAF702FC00208DF88E
:10B340002B00112206A901A807F068FFD4F8D80045
:10B3500038B305EB051104F1DE000844007CB4F8B5
:10B36000DC10884206DB012212A1002007F0D8FE83
:10B37000002605E005EB051104F1DE000844067C1B
:10B38000D4F8D80050F8262049463846FDF7E6FFA5
:10B3900007F1100188B2012301AA4946FEF752F8CD
:10B3A00005E0012301AA49463846FEF74BF80BB0E9
:10B3B000BDE8F0834C4231002DE9F0410546A888F4
:10B3C00008B9BDE8F081287A00EB8000C6B23446A7
:10B3D00018E0A888A0420FDC052094FBF0F100FBE8
:10B3E0001140182101EB001087B21023A02239462A
:10B3F0000020FDF765FC03E021462846FFF7ACFE80
:10B40000601CC4B2701D8442E3DB2846FFF71DFEBA
:10B4100000BFD6E72DE9F0410446A08808B9BDE891
:10B42000F081002512E0A088A84209DC182000EB7A
:10B4300005171023902239460020FDF741FC03E058
:10B4400029462046FFF746FF681CC5B2052DEADBFA
:10B4500094F83301752802D1A088401EE080204670
:10B46000FFF70AFE8F26B4F83401052808DD06F13F
:10B47000080188B2032308221821FDF7E7FE05E042
:10B480000823102218213046FDF71AFC6827B4F86B
:10B490003401052808DD06F1080188B204230822DA
:10B4A0003946FDF7D3FE07E0A7F1080081B2082373
:10B4B00010223046FDF704FC00BFB0E700B5A3B092
:10B4C0001548A0F20F1191F80E11A0F20F1292F888
:10B4D0002921A0F20F1393F80D31CDE90532CDE902
:10B4E0000710A0F12C020C38D11ECB1ECDE9013182
:10B4F000CDE903029838C23B08A2642100900AA853
:10B500000CF046FB01220AA9002007F009FE0AA858
:10B5100001F00EF923B000BDC726002041542B5086
:10B520004F433D3530342625732625732625732653
:10B53000257326257326257326256426256426254E
:10B54000642625730D0A000070B586B005460E46C8
:10B5500014462B4608A2142101A800940CF018FBF5
:10B5600001A801F0E5F82146304601F0F0F807A007
:10B5700001F0DEF806B070BD41542B5443505345E2
:10B580004E443D25642C25642C0000000D0A00006B
:10B5900070B504460D461646324629462046FFF74A
:10B5A000D3FF3146284602F0ABFF012C08D10948F1
:10B5B0000078FF2804DA07480078401C0549087025
:10B5C000012C06D10448007820F00400001D024937
:10B5D000087070BDA10400204C35002070B5002516
:10B5E00000240C4804680A2C06D102200A4908707D
:10B5F0000AA00CF0BDFA0BE0052C06D1012006498B
:10B6000008700CA00CF0B4FA02E010A00CF0B0FA34
:10B6100070BD0000E8FF0FE0E90000204D63755F9A
:10B62000547970652069532053542D2D2D2D0D0A0A
:10B63000000000004D63755F5479706520695320E8
:10B64000484B2D2D2D2D0D0A000000004D63755F18
:10B6500054797065202D2D2D554E4B4E4F574E0D64
:10B660000A0000002DE9F04190B0044620680E90D9
:10B6700060680F902088C0F3C507382F02DAC7F141
:10B68000380001E0C7F1780080464246284920464C
:10B6900000F062F80026002518E004F11800E91C0B
:10B6A000405C020604F11800A91C405C42EA00421A
:10B6B00004F11800691C405C42EA002004F1180102
:10B6C000495D08434DF82600761C2D1D0E2EE4D34F
:10B6D000694604F1080008F067F90026002521E01A
:10B6E00004F1080010F8261050304155503830F859
:10B6F0002600C0F3072204F15800691C4254503858
:10B7000050F82600C0F3074204F15800A91C425427
:10B71000503850F82600000E04F15801EA1C8854F5
:10B72000761C2D1D042EDBD310B0BDE8F081000087
:10B73000509C010800214160016005498160054A73
:10B74000C260CA430261034AD243426170470000AB
:10B750000123456789ABCDEF2DE9F04391B0044655
:10B760000F4615462088C0F3C509206800EBC500C8
:10B770002168884202D26068401C6060206800EB4B
:10B78000C5002060606800EB5570606033E017F81A
:10B79000012B484609F1010904F118010A54B9F1D5
:10B7A000400F28D14FF0000800261AE004F11800DD
:10B7B000F11C405C020604F11800B11C405C42EA36
:10B7C000004204F11800711C405C42EA002004F1C0
:10B7D0001801895D084301A941F8280008F1010812
:10B7E000361DB8F1100FE1D301A904F1080008F0EB
:10B7F000DBF84FF00009281EA5F10105C7D111B0F3
:10B80000BDE8F08308B54FF4A06001F003FB2520EC
:10B810008DF8000001208DF801008DF802008DF8F0
:10B820000300684601F0BEFA26208DF800000120D2
:10B830008DF801008DF802008DF80300684601F0D4
:10B84000B1FA27208DF8000001208DF801008DF855
:10B8500002008DF80300684601F0A4FA17208DF865
:10B86000000001208DF801008DF802008DF8030022
:10B87000684601F097FA08BD00240020FB490870D3
:10B8800001200AF037FFFEF7D1F9FFF7A7FE03F01A
:10B890009BF94FF4FA70FDF7F9FE07F069FCFDF72C
:10B8A00019FF0BF043FBFBF757FD07F019FDFEF7FF
:10B8B0000BFEEFA00CF05CF9FDF7F8FBFDF70AFFBB
:10B8C000F0A00CF055F9FAF7D7FCFAF7EDFEFFF708
:10B8D00099FFFEF78DFF0BF06BF9FBF7C9FF06F040
:10B8E00091FBED4800686422B0FBF2F1B1F1807F7A
:10B8F00000D31DE021F07F40401E4FF0E022506158
:10B9000050170F22002807DA13071E0EE34B00F032
:10B910000F052D1F5E5503E013071D0EE04B1D5450
:10B9200000BF00204FF0E02290610720106100BFAF
:10B93000DFF870C300DFDC4908604FF45071DB486A
:10B94000FAF7D5F807F00CFC0A20DFF864C300DF33
:10B9500064214FF45E7004F0B3F8032005F0D0F9D1
:10B9600007F0F6FB0122D3A1002007F0D9FBDFF896
:10B9700058C300DF00F54870D44908600023D44A5A
:10B98000D449D548DFF854C300DFD5490860002307
:10B99000D44AD049D448DFF844C300DFD349086013
:10B9A00040F29F41082003F0B1FB09F021FE5CE169
:10B9B000CF480078012803D0CE480078012802D172
:10B9C0000AF012FC16E0CC48007868B9DFF8F8C23B
:10B9D00000DFBE490968884203D8B448407801288E
:10B9E00002D10120C4490870C3480078012801D160
:10B9F0000AF0FAFB0120DFF8B8C200DFBF48008878
:10BA000088B1BF4800783E2803D1BD4802F08CFAC7
:10BA100002E0BB4801F070FD0020B9490870B94947
:10BA20000880B649088040F2BC41082003F06EFB54
:10BA3000B5480078012814D09C48807920B99B48EB
:10BA400090F8320301280CD1AF4800781C2802D0AE
:10BA5000012008F0F5FC0020944981F8320381F8B8
:10BA60003403FCF723FA041E45D0012C3ED10020FC
:10BA7000FEF790FC0020A549A1F80100FEF76CF943
:10BA8000A3A1A548FAF76FF858BB9F480078032890
:10BA900007D09D480078042803D09B4800781E28D2
:10BAA00009D19E4800689E4988421AD09B48006888
:10BAB0009C49884215D0994800689B49884210D01B
:10BAC0009A48007801280CDC07F04AFB9848007877
:10BAD00020B90C214FF4FA7003F0E0FF01209449E3
:10BAE00008700020714981F8330304E0FDF7DEFEA1
:10BAF00000208F4908700020FEF7B6FE0020FBF7FB
:10BB0000CBF8FBF7E5FEDFF8C0C100DF8949096823
:10BB1000884200D2A9E0DFF8B0C100DF6430854977
:10BB2000086085480078032807DA8448007820B147
:10BB300081480078401C8049087002F065FE80480A
:10BB40000078012810D16A48007868B969480078FF
:10BB500050B900207A4908707AA000F0E9FD01226E
:10BB600078A1002007F0DCFAFDF788FE4F488078C6
:10BB700050B94E48807938B9FCF7CCFE754991F937
:10BB80002B110844744908604FF400417348FBF7D7
:10BB900061FE7148006818B16F480068704908601C
:10BBA0006F480068FAF728FEFBF776FC0BF0E6F822
:10BBB0003E4890F83303401CC0B23C4981F833033F
:10BBC0003C2816DD4A480078012812D04948007800
:10BBD00001280ED06348007801280AD04A4800782E
:10BBE000012802D0012008F02BFC00202F4981F809
:10BBF0003303584890F82A015B4931F810000028B7
:10BC000019DD4248B0F80100401C80B23F49A1F85C
:10BC10000100504991F82A11534A32F81110884214
:10BC200009DB00203949A1F80100204840780128AB
:10BC300001D1FEF7AFFB41480078A8B13E4800783B
:10BC4000032811D130480078012805D160239F22B4
:10BC500050210020FDF7BCF844A003F0B9FA002001
:10BC6000364908703449087000BFA1E6E900002099
:10BC70004C6364496E69742E2E2E204F4B210D0AA1
:10BC800000000000477569496E69742E2E2E204F02
:10BC90004B210D0A000000000000002018ED00E01C
:10BCA00000E400E0F9930108AC000020FC31002022
:10BCB000198C01084D61696E205461736B205374B7
:10BCC00061727421000000007D920108E4000020F0
:10BCD000B82100200300040035CB000819930108A7
:10BCE00054010020B81D002085C700085001002025
:10BCF0006101002062010020E80000207A0100209C
:10BD00000E2700207801002041030020B001002010
:10BD10006F70656E00000000D72600205C000020D8
:10BD20000A04EC002A00FC000204FC00BD00002014
:10BD3000C600002008010020CB000020CA0000201F
:10BD4000C900002041542B504F433D353338263233
:10BD50000D0A0000B8250020D00000200008014096
:10BD6000B4000020B70100209A010020766F6C001B
:10BD700010B5124C10212046F9F7B9FE1048C069E1
:10BD8000000E20700E48C069000C60700C48808B5B
:10BD9000000AA0700A48007FE07009488069000E20
:10BDA000207107488069000C60710548008B000A0B
:10BDB000A0710348007EE07110BD0000042E002039
:10BDC0004C350020044802680448018804A00BF0A8
:10BDD000CFFE00BFFEE70000D8000020D400002006
:10BDE0000D0A5B4D4D485D463D25642C4C3D256458
:10BDF000000000002DE9F04104460F4627600025B1
:10BE000000BF206850F8250090F80080B8F1000FBE
:10BE100000D102E0681CC5B2F3E700BF681EC5B2DE
:10BE2000681C2071052095FBF0F0E071E079052198
:10BE300090FBF1F201FB120010B1E079401CE071BF
:10BE4000114800681149884203D011480078012840
:10BE50000CD1104802F076FBC6B2052096FBF0F03C
:10BE6000A071667100200A49087007E00648006862
:10BE70000949884202D10020A0716071204600F07B
:10BE800065F8BDE8F08100005C0000200A04F400C1
:10BE9000AE040020103100200A04EC0070B5044606
:10BEA000274800682749084430B1B0F5001F20D06A
:10BEB000B0F5601F3ED139E0204600F0A0F860796F
:10BEC00018B92079401E607102E06079401E6071EF
:10BED000A5796079052190FBF1F0A071A079A842C5
:10BEE00003D0204600F032F802E0204600F087F848
:10BEF00023E0204600F083F86079401C607160798F
:10BF00002179884201DB00206071A57960790521E3
:10BF100090FBF1F0A071A079A84203D0204600F078
:10BF200015F802E0204600F06AF806E0A07906491C
:10BF3000087100BF0248006870BD00BF0020FBE729
:10BF40005C000020F6FB43FF410300202DE9F04197
:10BF50000446A07900EB800000F0FF0845461BE096
:10BF60002079A84212DC052095FBF0F100FB11506E
:10BF700000EB8000182101EB800087B2781E81B2AF
:10BF8000122378221420FCF79BFE03E0294620466A
:10BF900000F04FF8681CC5B208F105008542DFDBF0
:10BFA000204600F02CF88C26A079002808DD06F148
:10BFB0000A0188B2032308221821FDF747F905E09A
:10BFC0000823122218213046FCF77AFE7C27A1793B
:10BFD000E079401E814208DA06F10A0188B20423A2
:10BFE00008223946FDF732F907E0A7F1080081B2CF
:10BFF000082312223046FCF763FEBDE8F0812DE9EC
:10C00000F041044614256079052190FBF1F201FB13
:10C010001200C7B207EB8700182101EB8000C6B2FF
:10C02000701E81B20E2378222846FDF79BF8BDE8EA
:10C03000F0812DE9F04105460C46052094FBF0F116
:10C0400000FB1140C7B207EB8700182101EB80000D
:10C05000C6B2701E81B2122378221420FCF730FE83
:10C06000296851F82400314606F060F8BDE8F081F7
:10C0700010B50B4800680B49884208D10A4840882F
:10C08000012801DBFAF716FD052008F0D9F904486C
:10C0900000680649884202D1052008F0D1F910BD98
:10C0A0005C0000200A04EC00F81B00200A04F400E5
:10C0B00010B50446D4B1FCF7B7FD01210CA006F081
:10C0C00035F8012314229F210020FCF713FF0BA059
:10C0D00006F00AFA012368229F210020FCF70AFFDC
:10C0E000012309A26E210020FDF7ACF910BD00006C
:10C0F000CFFBCFA2C9BEB3FD00000000C8B7B6A8F1
:10C10000C9BEB3FD3F0000005B4D5DC8B7B6A820B7
:10C11000205B455849545DC8A1CFFB002DE9F04193
:10C1200004460F4615461E462780A5703046F9F78F
:10C1300013FD84F87500102084F87700002084F83F
:10C140007400BDE8F0812DE9F05F044689464FF0A8
:10C15000000A4E4694F802C094F877E00CEB0E0308
:10C16000B4F800C094F876E0F4441FFA8CF2A17899
:10C170002088FCF7A5FD142104F16000F9F7B7FC55
:10C180002088C0F19F0087B23846F91707EB51713C
:10C19000C1F3C70184F87410D0460025AB4644E0D3
:10C1A00030789F2810DD94F87400401B022808DBCB
:10C1B00004F16000284431880180A81CC5B2B61C77
:10C1C00011E04FF0010B0EE094F87400401B0128C1
:10C1D00007DB317804F160004155681CC5B2761C5C
:10C1E00001E04FF0010BBBF1000F1ED04FF0000B30
:10C1F000002104F16000415594F802C04246531CEE
:10C2000003F0FF080CEB02112088012304F1600207
:10C21000FDF718F90AEB05001FFA80FA0025B8F1BE
:10C22000050F02DB5046BDE8F09F30780028B7D1FB
:10C23000002104F16000415594F802C04246531CAD
:10C2400003F0FF080CEB02112088012304F16002C7
:10C25000FDF7F8F80020E6E710B50948006809493D
:10C26000884204D1FBF758F9052008F0E9F80448A2
:10C2700000680549884202D1052008F0E1F810BDA8
:10C280005C0000200A04EC000A04F40010B5044627
:10C29000D4B1FCF7C9FC01210CA005F047FF012334
:10C2A00014229F210020FCF725FE0BA006F01CF9AC
:10C2B000012368229F210020FCF71CFE01230AA213
:10C2C0006E210020FDF7BEF810BD0000CFFBCFA20D
:10C2D000B8F1CABDBBAF0000C8B7B6A8C9BEB3FDB0
:10C2E000CBF9D3D0A3BF00005B4D5DC8B7B6A82083
:10C2F000205B455849545DC8A1CFFB0010B51048DC
:10C30000FFF7CCFD04460F4884420ED10C4840791B
:10C3100010B1012808D103E00F2008F091F803E0E4
:10C32000102008F08DF800BF08E0074800680749B2
:10C33000884203D10649487808F082F810BD000011
:10C34000900100200A04EC005C0000200A04F400C4
:10C350004103002010B504460CB3FCF765FC012135
:10C360000FA005F0E3FE012314229F210020FCF71B
:10C37000C1FD012368229F210020FCF7BBFD0B4972
:10C380000B48FFF737FD012368229F210020FCF7AF
:10C39000B1FD012307A26E210020FDF753F810BD67
:10C3A000CEC4B1BED1A1CFEE0000000040010020FC
:10C3B000900100205B4D5DC8B7B6A820205B4558B2
:10C3C00049545DCDCBB3F60070B5214800682149D2
:10C3D000884203D1052008F033F838E01C48006893
:10C3E0001D49884233D01A4800681C4988422ED122
:10C3F0001B48F9F7B1FB05462A461A4801781AA0EE
:10C400000BF0B6FB1648F9F7A7FB164909788842E6
:10C410001DD96623A02218210020FCF7D9FC104B5F
:10C42000182208211348FFF779FE0D480D4A1278AB
:10C4300081181048FFF787FE04462CB109480078A0
:10C4400020440849087002E000200649087070BDC9
:10C450005C0000200A04F4000A04EC000A04DC007A
:10C46000221C00203C0100206C656E3A25642C25BE
:10C47000640D0A00801B002010B50446002C32D049
:10C4800000201A4908704FF4C8711948F9F72FFBBA
:10C49000FCF7CAFB012117A005F048FE0123142276
:10C4A0009F210020FCF726FD114802F0EFFD104B04
:10C4B000182208211248FFF731FE0D480B4A127866
:10C4C00081180F48FFF73FFE0849087001236822D2
:10C4D0009F210020FCF70EFD01230AA26E210020FF
:10C4E000FCF7B0FF10BD00BFFCE700003C010020DE
:10C4F000221C0020CFFBCFA2D4C4B6C10000000094
:10C50000801B00205BCFC25DB7ADD2B3205B455826
:10C5100049545DB7B5BBD80010B51248408810B17A
:10C520001148FEF78BFC114800681149084450B1CE
:10C53000B0F5002F03D0B0F5402F0FD10AE0022054
:10C5400007F07EFF0BE00748408810B10E2007F08F
:10C5500077FF04E00D2007F073FF00E000BF00BF8D
:10C5600010BD0000F81B00200C2F00205C000020F4
:10C57000F6FB13FF2DE9FE4300251E4CA8460026BE
:10C580002EE0322700251CA000F0D2F81DA20A21BF
:10C5900068460BF0FDFA1DE04FF4A061A01C00F00E
:10C5A000FBFA80B2208088B16946A01C00F0D7F861
:10C5B00080B9E81DA11C085C52280BD105F10900C7
:10C5C000085C412806D10120BDE8FE830120DFF888
:10C5D0003CC000DF381EA7F10101CFB2DCD1761CD0
:10C5E0001E2ECEDB01220AA1002006F099FD0020BC
:10C5F000EAE70000DA73002041542B4350494E3FD4
:10C600000D0A00002B4350494E3A0000198C0108D6
:10C610005B325D4E4F204361726420212121200056
:10C6200010B5A721022002F071FD0AF007F900F011
:10C6300099FB002014490870AB21022002F066FD2E
:10C640004FF4007011490861022011490860C820A8
:10C65000DFF840C000DF02200D49091D08600120FD
:10C66000091F08606420DFF82CC000DF01200849A2
:10C67000091D0860084948710AF0C6FC08B100208D
:10C6800010BD0120FCE70000A104002000100140C3
:10C69000100C0140198C0108FC31002008B5012163
:10C6A0001D2001F099FF002002F03CF810208DF8C9
:10C6B000030003208DF802000220ADF80000694657
:10C6C0001848FAF7F3FF4FF40070ADF80000694620
:10C6D0001548FAF7EBFF0120ADF800006946114854
:10C6E000FAF7E4FF4FF48070ADF8000069460F4898
:10C6F000FAF7DCFF10208DF8030002208DF802000D
:10C700008003ADF8000069460748FAF7CFFF4FF401
:10C7100000400549486101200249143108600220A7
:10C72000086008BD000C01400010014000080140F5
:10C7300070B504462046F9F70FFA85B2262102208B
:10C7400002F0E4FC294620460AF01CFA70BD70B5E0
:10C7500004460D46294620460AF014FA70BD30B54D
:10C7600002460B461946144607E008782578A84289
:10C7700001D0012030BD491C641C08780028F4D188
:10C7800000BFF7E78AB000BF00BFB04C0120B0493E
:10C7900008700122AFA1002006F0C2FC0120FCF7C6
:10C7A00097F90020AF49087006F078FF0020AE49E5
:10C7B00048708870C8700122ACA106F0B1FCFAF78D
:10C7C000E9FA0020FCF7FEF900BF0122ACA100202D
:10C7D00006F0A6FC0020AE4981F82D03C87181F84F
:10C7E0002E03AC4908700420AB490861012240F2D5
:10C7F0002551AA4809F093FEA948B0F8112000235A
:10C80000C11CA8A00BF0B4F96420DFF8B0C200DFAF
:10C8100001209F4981F83C03FFF702FF28B1012264
:10C82000A7A1002006F07CFC17E00120A9490870B0
:10C830000420994908610122A7A1002006F070FC9C
:10C84000FAF76CFAFCF746FF06E000209049C87141
:10C850006420DFF868C200DFF7E7012004F050FA37
:10C860000120FCF7AFF905A801F0D0FEA1A2142128
:10C870006846059B0BF08CF901226946002006F002
:10C880004FFC0120834908700AF08CFC00B19CE742
:10C8900006F066FCFBF7E4FEFBF758FC0AF0E4FA4E
:10C8A00002207C4908700120FAF7F6F9FFF762FED2
:10C8B00070BB0420764981F82E0300BF9148C078F0
:10C8C000012801D1FAF7D4FF0120714981F83D0315
:10C8D0001DE04FF4A061A01C00F05EF980B2208042
:10C8E00000B114E00120DFF8D4C100DF0020684966
:10C8F000C8715748007800B909E08348008828B11A
:10C9000082480CF085F800207F49088000BFE0E7EE
:10C9100001227FA1002006F003FCFEF7CFFD0120DD
:10C920005B4981F83D038FE04948007828BB00202F
:10C930005749C8714FF4A061A01C00F02DF9208068
:10C94000208800280BDD00205149C8710022A11C5D
:10C95000104606F0E5FBA01CF9F7CAFD74E020883C
:10C96000002805DA01226EA1002006F0D9FB6BE059
:10C970000120DFF848C100DF66E04FF4A061A01C91
:10C9800000F00AF920802088002811DD00204049AD
:10C99000C871A0782B2802D0A0785E2803D1A01CF3
:10C9A000F9F7A6FD50E02188A01C0AF0C7FC4BE077
:10C9B0002088002805DA012259A1002006F0B0FBEA
:10C9C00042E00120DFF8F4C000DF3148007818B9F8
:10C9D000012004F095F921E02D488078002803DD3E
:10C9E000052004F08DF919E029488079002803DD3D
:10C9F000062004F085F911E04B480068A0F5AA7004
:10CA0000642148435A21B0FBF1F00F2803D20720DC
:10CA100004F076F902E0042004F072F91C4890F862
:10CA20002D0300B1D1E6DFF804C100DF40490968F9
:10CA3000884200D208E0DFF8F4C000DF64303C49EF
:10CA40000860F9F7F5FD00BF6EE70000DA7300201B
:10CA500060010020506F63205461736B2073746118
:10CA600072742100A1040020400000204D6F646515
:10CA70006D205461736B2073746172742100000027
:10CA80004D6F64656D496E69742E2E2E0000000096
:10CA9000FC310020B00000200010014000480040A0
:10CAA000B82500200D0A25735F5625642E256420C5
:10CAB00053746172742E2E2E0D0A0000198C010819
:10CAC0005B30315D204D6F64656D20496E69742067
:10CAD0004F4B0000E80000205B30315D4661696C1F
:10CAE00065640D0A456E746572204754204D6F646D
:10CAF00065210000436C6F636B3D3D3D25640D0A6D
:10CB0000000000004C35002080010020D6270020C6
:10CB10005B325D436172642072656164790000007C
:10CB20005175657565463100D00000207D92010881
:10CB30007001002000210748DFF81CC000DF07E07B
:10CB40004FF6FF710348DFF814C000DF09F0F0FE74
:10CB5000F6E7000058010020F18F0108319001082C
:10CB6000012207A1002006F0DBFAFAF7D7F806E069
:10CB700000200749C8716420DFF818C000DFF7E71C
:10CB8000676F2047545F4D6F64650D0A0000000019
:10CB9000FC310020198C01082DE9F84380460E462F
:10CBA000304C3148007820B930A00AF0E1FFFFF79F
:10CBB000D7FFA08810B90020BDE8F8836188A01DC8
:10CBC00030F82100ADF800006188A01D00EB810065
:10CBD0004088ADF802000027002522E0B4F8D0001C
:10CBE00000B922E0CE34D4F80A00E18810F80190B0
:10CBF000E088401CE080E08834F8CE19884202DBEF
:10CC00000020A4F8D400B4F8D000401EA4F8D0004E
:10CC1000B74204DA3846791C8FB208F80090681CD5
:10CC200085B2BDF80000A842D8DC00BF6088401C77
:10CC300060806088322801DB00206080A088401E70
:10CC4000A080BDF80000A84202D06FF00100B3E759
:10CC5000BDF80000B04202DD4FF0FF30ACE7BDF898
:10CC60000000A9E7FC6D00206001002053544F50E4
:10CC700020474F2047540D0A0000000030B50346FE
:10CC80000A4612480024048084804480002108E081
:10CC90000025841D04EB81046580841D24F8215047
:10CCA000491C3229F4DBC0F8D830002104E000240C
:10CCB000D0F8D8506C54491C9142F8DB20F8CE2FA4
:10CCC00000248480C4804480CE3830BDFC6D0020B8
:10CCD00070B504460A4622498888322802DB4FF0A4
:10CCE000FF3070BDB1F8D0001044B1F8CE50A8426A
:10CCF00002DD6FF00100F4E7B1F8D2500E88881D14
:10CD000000EB860045800D88881D20F82520002333
:10CD100017E0E05CD231D1F806500E88A85508889B
:10CD2000401C088031F8D209B0F5C05F02DB00205A
:10CD3000A1F8D200B1F8D000401CA1F8D000581CD6
:10CD400083B29342E5DB0888401C088008883228BB
:10CD500001DB002008808888401C88800020C0E714
:10CD6000FC6D002000B54FF4C0510248FFF786FF6C
:10CD700000BD0000FC55002010B50120FAF720FC92
:10CD800048210548F8F7B3FE122000F04DF80020C6
:10CD90000249087010BD0000C00E002024000020D1
:10CDA0007047000070B5002100230F22C47804B33F
:10CDB000154C246804F4E064C4F5E064210AC1F170
:10CDC0000403CA40447804FA03F1847814402143F0
:10CDD00009010E4C0678A155047804F01F050124C2
:10CDE000AC4005786D11AD0005F1E025C5F80041B6
:10CDF00009E0047804F01F050124AC40044D0678D6
:10CE0000761145F8264070BD0CED00E000E400E02E
:10CE100080E100E002490143024A116070470000CE
:10CE20000000FA050CED00E0024948710121014AB9
:10CE300011717047C00E00200B48016801F40070AA
:10CE4000B0F5007F0BD109480078052805DA0748BE
:10CE50000078401C054A107004E001207047002053
:10CE6000024A10700020F9E7080C01400001002080
:10CE700070B50446002506E00120DFF810C000DF91
:10CE8000FCF728FC6D1CA542F6DB70BD198C01086F
:10CE900010B54FF48030F9F7EBFE20B104A00AF092
:10CEA00067FE06F003F94FF48030F9F7CFFE10BDAE
:10CEB000B5E7C1BFB5CD2E2E2E2E2E2E2E2E2E2E08
:10CEC0000D0A0000014908627047000000000E4290
:10CED0000349096841EA8001014A11607047000076
:10CEE0000070004010B5024600200C4B186820F07E
:10CEF0000300104318600A4B1B6843F00403084CFE
:10CF00002360012901D130BF00E020BF044B1B6822
:10CF100023F00403024C236010BD000000700040A9
:10CF200010ED00E001460020034A52680A400AB1B1
:10CF3000012000E000207047007000402DE9FC4710
:10CF4000044688469146002523212046F8F7CFFD68
:10CF5000AB2229466D1C62547A2229466D1C62540C
:10CF6000002229466D1C62541F2229466D1C625402
:10CF70002D48D0F8170001909DF8072029466D1C18
:10CF800062549DF8062029466D1C62549DF80520C8
:10CF900029466D1C62549DF8042029466D1C62547C
:10CFA000002607E02148825D2946681C85B262544C
:10CFB000701C86B2142EF5DBCDF804809DF8072096
:10CFC0002846691C8DB222549DF806202846691C0B
:10CFD0008DB222549DF805202846691C8DB222543A
:10CFE0009DF804202846691C8DB22254CDF800908B
:10CFF0009DF801202846691C8DB222549DF800201E
:10D000002846691C8DB222540027002603E0A05D4B
:10D010004740701C86B2AE42F9DB2846691C8DB2CF
:10D0200027542846BDE8FC87B8250020E80E0020DC
:10D030002DE9FC41044600251D212046F8F757FD47
:10D04000AB2229466D1C62546A2229466D1C62542B
:10D05000002229466D1C6254192229466D1C625417
:10D060002048D0F8170001909DF8072029466D1C34
:10D0700062549DF8062029466D1C62549DF80520D7
:10D0800029466D1C62549DF8042029466D1C62548B
:10D0900014211548F8F72BFD14480088114BDB1CB0
:10D0A00013A21421009010480AF072FD002607E038
:10D0B0000D48825D2846691C8DB22254701C86B2D0
:10D0C000142EF5DB0027002603E0A05D4740701C0E
:10D0D00086B2AE42F9DB2846691C8DB22754284639
:10D0E000BDE8FC81B8250020E80E00201C000020CF
:10D0F00025735F5625642E61707000002DE9F04F96
:10D1000089B004460D4616461F46A02C01DA802D34
:10D1100002DB09B0BDE8F08FA019A02802DDC4F140
:10D120009F0086B2E819802802DDC5F17F0087B232
:10D13000FCF7D0FAE819401E83B2A019401E82B253
:10D1400029462046FDF756F94FF000083FE005EB71
:10D15000080008904FF0000A35E0089800EB8000C6
:10D160001D4901EB401004EB0A01405C0790079851
:10D170004FEA8009194810F809000490174909F18D
:10D180000100085C059009F10200085C0690069811
:10D19000C01003900598801002900498C010019070
:10D1A0000398C102029801EB4011019808441FFA4C
:10D1B00080FB4FEA2B20FDF7FDFA0BF0FF00FDF797
:10D1C000F9FA0AF1010AB245C7DB08F10108B845CE
:10D1D000BDDB00BF9DE70000F47C0020F478002058
:10D1E0002DE9FF4F93B0209800F0F0000F902098A9
:10D1F00000F00F000E900024159810BB0F9838B95E
:10D200004FF00C090C254FF00208484E484F06E03D
:10D210004FF0080910254FF00108464E464F07E031
:10D2200039781698814200D105E07F1C601C84B2D9
:10D2300038780028F4D100BF04FB08F000FB056635
:10D2400024E00F9888B94FF010090C254FF0020820
:10D2500008AE0027002408AA0F9BDDE91501FAF7A4
:10D26000EBFD182812D0354E10E04FF010091025B4
:10D270004FF002086E46002700246A460F9BDDE946
:10D280001501FAF7D9FD202800D02C4E1498284417
:10D29000802802DB17B0BDE8F08F13984844A0281F
:10D2A00000DBF7E74FF0000B3CE01498584480B2E5
:10D2B00012904FF0000A2FE0139800EBCA0080B2E2
:10D2C000119016F8010B109000241FE080202041DF
:10D2D0001099084058B11A480178129800EB800064
:10D2E000184A02EB40121198204411540CE00E9899
:10D2F00050B115480178129800EB8000114A02EBFA
:10D300004012119820441154601C84B2082CDDDBBB
:10D310000AF101001FFA80FAC245CDDB0BF10100D2
:10D320001FFA80FBAB45C0DB00BFB3E75FA301087A
:10D3300003A30108F09C0108909C0108E0A20108E9
:10D34000B1040020F47C0020B20400202DE9FF4F3E
:10D3500093B0209800F0F0000F90209800F00F009C
:10D360000E900024159810BB0F9838B94FF00C0997
:10D370000C254FF00208474E474F06E04FF00809D2
:10D3800010254FF00108454E454F07E039781698B3
:10D39000814200D105E07F1C601C84B238780028EF
:10D3A000F4D100BF04FB08F000FB056624E00F98F1
:10D3B00088B94FF010090C254FF0020808AE00277D
:10D3C000002408AA0F9BDDE91501FAF735FD18289E
:10D3D00012D0344E10E04FF0100910254FF0020823
:10D3E0006E46002700246A460F9BDDE91501FAF717
:10D3F00023FD202800D02B4E14982844802802DBDF
:10D4000017B0BDE8F08F13984844A02800DBF7E779
:10D410004FF0000B3AE01498584480B212904FF04D
:10D42000000A2DE0139800EBCA0080B2119016F8A4
:10D43000010B109000241DE080202041109908402D
:10D4400050B1129901EB8101174A02EB4112119977
:10D450002144219850540BE00E9848B1129800EBEB
:10D460008000114A02EB4012119820442299115475
:10D47000601C84B2082CDFDB0AF101001FFA80FA7D
:10D48000C245CFDB0BF101001FFA80FBAB45C2DBCD
:10D4900000BFB5E75FA3010803A30108F09C0108E2
:10D4A000909C0108E0A20108F47C00202DE9F047DF
:10D4B00004460D46DDF820C0002116E06F1801FB80
:10D4C00002F600200EE006EB00081CF8088007EBCF
:10D4D0008709DFF820A00AEB491904EB000A09F8D4
:10D4E0000A80401C9042EEDB491C9942E6DBBDE815
:10D4F000F0870000F47C00202DE9F04FADF5257D8C
:10D5000006464022FE4995A8F8F7D8FA4FF00008E1
:10D510004FF48771082001F0F9FD00BF404608F183
:10D52000010895A951F8200000780028F6D1A8F14B
:10D53000010840F21111082001F0E8FD002721E068
:10D5400095A850F827A0F01C049000200590834671
:10D550000FE09AF8001004980078814202D0012070
:10D5600005900AE00AF1010A0498401C04900BF1AE
:10D57000010B9AF800000028EBD100BF059800B914
:10D5800002E07F1C4745DBDB00BF40F2251108208D
:10D5900001F0BCFD474503D10DF5257DBDE8F08FB9
:10D5A0000F2F17D2DFE807F008172D316CEFEDECE5
:10D5B000EBEAE9E8E7E6E500092003F0E1FB0122F8
:10D5C000D0A1002005F0ACFD0220F9F7A7F9012059
:10D5D000CF490870EEE3092003F0D2FB0122CDA170
:10D5E000002005F09DFDFAF743F90120CC49C870F1
:10D5F000CC4908600020FBF76BFA0120F9F78EF99F
:10D60000D8E3092003F0BCFBD4E3092003F0B8FB06
:10D61000307A4D2812D1707A43280FD1B07A55282C
:10D620000CD10122C0A1002005F07AFD5520C1498E
:10D630004870C1A001F0CCFD00BFFEE7307A4D2854
:10D640001DD1707A4F281AD1B07A442817D1F07AB8
:10D65000452814D1307B4D2811D10122B9A10020D9
:10D6600005F05EFDBBA0FFF763F807E0FCF732F8BA
:10D67000FFF7E2FB10B10420BB494861F6E799E3EC
:10D680006FAABAA13046FAF79FFF0446012C01DBCE
:10D69000282C05DB0122B6A1002005F041FD89E31D
:10D6A0006FA91AA8F8F76DFA6FAAB7A13046FAF772
:10D6B0008BFF04460CB900250BE0052C05DD01228B
:10D6C000B3A1002005F02CFD74E36FA8F8F771FA00
:10D6D00085B26FAAB5A13046FAF776FF0446012C51
:10D6E00001DB142C05DB0122B2A1002005F018FD9E
:10D6F00060E36FA910A8F8F744FA6FAAB5A1304605
:10D70000FAF762FF0446012C01DB142C05DB012231
:10D71000B3A1002005F004FD4CE36FA906A8F8F7BB
:10D7200030FA06A81AA910ABB5A2CDE900109621CF
:10D730006FA80AF02DFA24A96FA8F8F78CFEB5A0FF
:10D74000FEF7F6FF24A8FEF7F3FFB6A0FEF7F0FF02
:10D7500006A810A91AABB4A2CDE9005102909621F7
:10D760006FA80AF015FA01226FA9002005F0D8FC75
:10D7700020E30DE3DBE2BEE251E243E230E207E206
:10D78000F3E184E0FFE76FAA78A13046FAF71CFFC7
:10D790000446012C01DB282C05DB0122ADA1002071
:10D7A00005F0BEFC06E36FA91AA8F8F7EAF96FAA1C
:10D7B00075A13046FAF708FF04460CB900250BE0C6
:10D7C000052C05DD0122A9A1002005F0A9FCF1E24C
:10D7D0006FA8F8F7EEF985B26FAAABA13046FAF759
:10D7E000F3FE0446012C01DB0A2C05DD0122A7A172
:10D7F000002005F095FCDDE26FA8F8F7E7F9814617
:10D800004C48C0F817901AA91B30F8F7BAF94948E4
:10D81000A0F81350CC30F8F79FF90E2805D201225A
:10D82000A1A1002005F07CFCC4E24248CC301AA93A
:10D83000CDE90010CC38D0F81730A2A296216FA8FD
:10D840000AF0A6F924A96FA8F8F705FEA3A0FEF731
:10D850006FFF24A8FEF76CFF72A0FEF769FFA3A07C
:10D8600001F0B6FC3348D0F817003249B1F8131074
:10D87000304B1B339FA2CDE9001096216FA80AF010
:10D8800087F901226FA9002005F04AFC92E26FAAF5
:10D8900036A13046FAF798FE0446012C01DB282C0D
:10D8A00005DB01229BA1002005F03AFC82E26FA972
:10D8B0001AA8F8F766F96FAA33A13046FAF784FE82
:10D8C00004460CB900250BE0052C05DD012297A1CB
:10D8D000002005F025FC6DE26FA8F8F76AF985B223
:10D8E0001AA914484330F8F74CF91248A0F815501B
:10D8F00095A001F06DFC0F48B0F815000D4B27E125
:10D90000609B010847542B544D3A4F4B00000000D8
:10D91000BC00002047542B54473A4F4B00000000F6
:10D920004C350020AC01002047542B464F54413A5F
:10D930004D435500B8250020434F4D2D464F5441CF
:10D940000000000047542B464F54413A4D4F444588
:10D950004D00000061742B706F633D31303030300A
:10D960003031380D0A00000000100140495000001D
:10D9700047542B5354503A4641494C5B4950204937
:10D980006E76616C69645D00506F72740000000017
:10D9900047542B5354503A4641494C5B506F727474
:10D9A00020496E76616C69645D0000004163636FBD
:10D9B000756E740047542B5354503A4641494C5BA2
:10D9C0004163636F756E7420496E76616C69645D46
:10D9D0000000000050617373776F726400000000F4
:10D9E00047542B5354503A4641494C5B5061737332
:10D9F000776F726420496E76616C69645D00000027
:10DA000069643D25733B69703D25733B7077643DC8
:10DA100025733B0041542B504F433D313230303061
:10DA2000300000000D0A000047542B5354503A496F
:10DA3000503D25733B506F72743D25753B416363C8
:10DA40006F756E743D25733B50617373776F7264AD
:10DA50003D25730047542B534D503A4641494C5B8A
:10DA6000495020496E76616C69645D0047542B53C0
:10DA70004D503A4641494C5B506F727420496E7666
:10DA8000616C69645D00000050534E0047542B5395
:10DA90004D503A4641494C5B50534E20496E766199
:10DAA0006C69645D0000000047542B534D503A46AA
:10DAB00041494C5B4D45494420496E76616C69642F
:10DAC0005D00000069643D256C753B69703D257300
:10DAD0003B7077643D25733B0000000041542B50A0
:10DAE0004F433D303130303030000000434F4D2D3A
:10DAF000534D500047542B534D503A49503D2573D8
:10DB00003B506F72743D25753B50534E3D256C75EF
:10DB10000000000047542B5347503A4641494C5BA4
:10DB2000495020496E76616C69645D0047542B53FF
:10DB300047503A4641494C5B506F727420496E76AB
:10DB4000616C69645D000000434F4D2D53475000E8
:10DB500043339CA2962100906FA80AF019F8012285
:10DB60006FA9002005F0DCFA24E19C4800F1B10126
:10DB7000CDE900101B38D0F8173099A296216FA874
:10DB80000AF006F801226FA9002005F0C9FA11E198
:10DB9000092003F0F5F80122A1A1002005F0C0FA48
:10DBA0000120DFF888C200DF0220F8F7B7FE4FF44B
:10DBB00000709F49486102209E4908600520DFF8F7
:10DBC0006CC200DF02209B49091D086007E0FBF7DB
:10DBD00081FDFFF731F910B1042095494861F6E75E
:10DBE0007E481B38B0F811007C4B183B92A296215E
:10DBF00000906FA809F0CCFF01226FA9002005F06A
:10DC00008FFAD7E0904891A2962103686FA809F097
:10DC1000BFFF01226FA9002005F082FACAE06FAAB7
:10DC2000AFF278213046FAF7CFFC0446012C01DB35
:10DC30001E2C05DD012289A1002005F071FAABE45C
:10DC40006FA910A8F7F79DFF6FAAAFF278213046B1
:10DC5000FAF7BAFC0446012C01DB1E2C05DD01227B
:10DC600086A1002005F05CFA96E45C481B3890F829
:10DC7000CA00032810D18948007801280CD010A9C7
:10DC800056486F30F7F77DFF6FA954488E30F7F78D
:10DC900078FF83A001F09CFA6FA810AB82A24FF42A
:10DCA0009671009024A809F073FF012224A9002096
:10DCB00005F036FA84480068401C10B183480068BB
:10DCC00000B977E0824910A8F7F74DFF30B98049D5
:10DCD0001F316FA8F7F747FF00B96BE010A97C4828
:10DCE000F7F74FFF6FA97A481F30F7F74AFF012077
:10DCF000784908705EE069480078012802D1002761
:10DD0000834602E006274FF0070BCBEB4B10704920
:10DD1000BA394318C7EB471042186FA124A809F07D
:10DD20004BFF012224A9002005F0FAF942E06FAA76
:10DD300071A13046FAF748FC044624B16FA8F7F702
:10DD400038FF074601E040F26E376FAA6BA13046FC
:10DD5000FAF73AFC044624B16FA8F7F72AFF85B218
:10DD600000E0082505F0FCF92946384601F096FE4A
:10DD700005EB850040003B4661A2962100906FA80C
:10DD800009F006FF01226FA9002005F0C9F911E092
:10DD900012481B38B0F81500104B28335CA29621AE
:10DDA00000906FA809F0F4FE01226FA9002005F091
:10DDB000B7F900BF00BF40F22621082001F0A6F904
:10DDC00000BF3CE747542B5347503A49503D257319
:10DDD0003B506F72743D25753B000000D325002039
:10DDE00047542B524D503A50534E3D256C753B4D88
:10DDF0004549443D25733B434E554D3D3030303011
:10DE00003030303030303B55494D49443D30303072
:10DE1000303030303030303B49503D25733B0000CE
:10DE200047542B5053543A4F4B000000198C0108B3
:10DE300000100140100C014047542B5645523A2522
:10DE4000735F562564000000B400002047542B4245
:10DE500041543A20256420560000000047542B41CD
:10DE6000504E3A4641494C5B4163636F756E742076
:10DE7000496E76616C69645D0000000047542B4177
:10DE8000504E3A4641494C5B50617373776F7264F0
:10DE900020496E76616C69645D000000DC01002041
:10DEA000434F4D2D41504E0047542B41504E3A4167
:10DEB00063636F756E743D25733B50617373776F49
:10DEC00072643D25733B0000A8010020D8010020AA
:10DED000CE2E0020DE00002047542B5241504E3AF7
:10DEE0004163636F756E743D25733B506173737747
:10DEF0006F72643D25733B00460000005400000033
:10DF0000424545503D2564487A2C25646D730000D8
:10DF100047542B5247503A49503D25733B504F527E
:10DF2000543D25643B0000002DE9F047A8B00746AA
:10DF30004FF00008C24600250026A946781CF7F7D6
:10DF400038FE64280DD0652814D0662870D0672864
:10DF500006D11420DFF8F8C200DF0420BD49486173
:10DF600072E10122BCA1002005F0DAF80120BE49CF
:10DF7000087069E11EAA0121384605F084F91EA83F
:10DF8000F7F7EAFDC4B2012C01DB282C05DB0122E6
:10DF9000B6A1002005F0C4F856E11EA9B848F7F76D
:10DFA000F0FD1EAA0221384605F06DF91EA8F7F70C
:10DFB000D3FDC4B2012C01DB282C05DB0122B1A169
:10DFC000002005F0ADF83FE11F221EA9AC485030FB
:10DFD000F7F7B6FD1EAA0321384605F054F91EA82E
:10DFE000F7F7BAFDC4B2022C01DB282C05DB0122B5
:10DFF000A9A1002005F094F826E103221EA9A0485B
:10E00000C230F7F79DFD00BF4046411C01F0FF08FC
:10E01000A74951F8200000780028F5D100251DE01F
:10E02000A34850F825600DF178094FF0000A0BE085
:10E03000C2E0307899F80010884202D04FF0010A0F
:10E0400005E0761C09F1010930780028F1D100BF04
:10E05000BAF1000F00D103E0681CC5B24545DFDB13
:10E0600000BF87481B3890F82701A8420FD084488A
:10E070001B3880F8275190F827018E490B5C8EA23F
:10E0800028211EA809F084FD1EA8FEF751FB1EAA38
:10E090000421384605F0F7F81EA8F7F75DFDC4B275
:10E0A000022C01DB282C05DB012287A1002005F0D2
:10E0B00037F8C9E003221EA97148C530F7F740FDC3
:10E0C0001EAA0521384605F0DEF81EA8F7F744FD24
:10E0D000C4B2022C01DB282C05DB012280A1002028
:10E0E00005F01EF8B0E00A221EA96548E830F7F7EF
:10E0F00027FD1EAA0621384605F0C5F81EA8F7F729
:10E100002BFDC4B2022C01DB282C05DB012279A1F6
:10E11000002005F005F897E020221EA95848C830D5
:10E12000F7F70EFD1EAA0721384605F0ACF81EA829
:10E13000F7F73FFD52491B3981F80D011EAA08214E
:10E14000384605F0A0F81EA8F7F733FD4C491B39F7
:10E1500081F829011EAA0921384605F094F81EA865
:10E16000F7F727FD46491B3981F80E011EAA0A213F
:10E17000384605F088F81EA8F7F7EEFCC4B2022C6A
:10E1800001DB282C05DB012260A1002004F0C8FF80
:10E190005AE010221EA93A48F430F7F7D1FC60A0EB
:10E1A00001F016F80A20DFF8A8C000DF00225EA107
:10E1B000104604F0B5FF47E04FF4977230491B3921
:10E1C0005D4800F0E9FC2E49F4315CA009F0D0FC78
:10E1D0004FF497722A491B39604800F0DDFC28494A
:10E1E000F4315FA009F0C4FC2548F430A0F20F110F
:10E1F00091F80E11A0F20F1292F82921A0F20F133C
:10E2000093F80D31CDE90532CDE907102C3800F136
:10E210002001C21EA0F1E30393F82731DFF890C07C
:10E220005CF82330CDE90132CDE903107838144B86
:10E2300052A2502100900AA809F0AAFC00220AA9C3
:10E24000104604F06DFF00BF00BF28B0BDE8F087A6
:10E25000198C01080010014041542B504F433D35AB
:10E2600030310D0A00000000610100204641494C98
:10E270005B495020496E76616C69645D0000000066
:10E28000D32500204641494C5B41504E20496E76D3
:10E29000616C69645D0000004641494C5B4E455429
:10E2A0005F4D4F444520496E76616C69645D0000A6
:10E2B000EC000020DD01002061742B7A736E746520
:10E2C0003D25640D0A0000004641494C5B4C414E1F
:10E2D000475541474520496E76616C69645D000091
:10E2E0004641494C5B4C6F63616C20496E76616CB2
:10E2F00069645D004641494C5B4368616E6E656CC4
:10E3000020496E76616C69645D0000004641494CAD
:10E310005B494D454920496E76616C69645D00003A
:10E32000434F4D2D41504E0041542B504F433D35EE
:10E3300030330D0A0000000000F8010873757450B6
:10E34000726F64756374506172612E4C43445365FF
:10E3500074496E6465783D25730D0A0000F001086C
:10E360006261636B7570506172612E4C43445365FA
:10E3700074496E6465783D25730D0A0041542B5035
:10E380004F433D35303426257326257326257326C5
:10E3900025732625732625732625642625642625C0
:10E3A000642625730D0A000008B501211C2000F029
:10E3B00013F910208DF8030003208DF802000420CB
:10E3C000ADF8000069461248F9F770F904201049C9
:10E3D000486110208DF8030003208DF80200102002
:10E3E000ADF8000069460A48F9F760F904208DF895
:10E3F000030003208DF802004FF40040ADF8000048
:10E4000069460448F9F752F910200149486108BDEE
:10E41000001001400008014010B50446002C29D02E
:10E42000FAF702FC012314229F210020FAF762FD73
:10E430001AA11B48F7F797FB20B9022119A003F096
:10E4400075FE03E002211AA003F070FE13A1144828
:10E45000F7F789FB20B9302118A003F067FE03E02D
:10E46000302119A003F062FE012368229F210020C1
:10E47000FAF740FD09A10A48F7F775FB30B9012307
:10E4800014A26E210020FAF7DDFF05E0012317A298
:10E490006E210020FAF7D6FF10BD0000636E000069
:10E4A00098260020B9D8BBFACCE1CABE0000000013
:10E4B000506F7765724F666600000000C8B7B6A857
:10E4C000B9D8BBFA3F000000506F7765724F66669F
:10E4D0003F000000C8B7B6A8202020202020202020
:10E4E00020202020CDCBB3F6000000005B4D454E30
:10E4F000555D2020202020205B455849545D0000B8
:10E5000070B505460E46314608A009F031FB0024DF
:10E5100005E0295D08A009F02BFB601C84B2B44221
:10E52000F7DB07A009F024FB70BD000044617461B3
:10E530005B25645D3A0D0A0025303278000000004A
:10E540000D0A000070B504462069002805DA07A00E
:10E5500009F00EFB4FF0FF3070BD206954F82050D9
:10E560002069401E20612846F6E70000737461634D
:10E570006B20697320656D7074790D0A00000000CE
:10E5800070B504460D462069042804D106A009F0A0
:10E59000EFFA012070BD2069401C2061206944F819
:10E5A00020500020F6E70000737461636B206675ED
:10E5B0006C6C0D0A0000000029B1064AD2690243C2
:10E5C000044BDA6104E0034AD2698243014BDA6109
:10E5D000704700000010024029B1064A92690243C8
:10E5E000044B9A6104E0034A92698243014B9A61A9
:10E5F00070470000001002400348406A40F08070FD
:10E6000001494862704700000010024030B5002107
:10E610000022002400232D4D6D6805F00C0121B16E
:10E62000042905D0082923D105E0294D056022E001
:10E63000284D05601FE0254D6D6805F47012234DCF
:10E640006D6805F48034022505EB92421CB9224D19
:10E65000554305600BE01D4D6D6805F400351DB197
:10E660001E4D5543056002E01A4D5543056002E01A
:10E67000174D056000BF00BF144D6D6805F0F00137
:10E680000909174D6B5C0568DD4045600F4D6D68ED
:10E6900005F4E061090A124D6B5C4568DD40856058
:10E6A0000A4D6D6805F46051C90A0D4D6B5C4568F3
:10E6B000DD40C560054D6D6805F44041890B094D8D
:10E6C0006B5CC568B5FBF3F5056130BD0010024019
:10E6D00000127A00001BB70000093D00808D5B002E
:10E6E0008C0400209C04002010B501460022002369
:10E6F00000204A11012A02D1094C236806E0022AAF
:10E7000002D1074C236A01E0054C636A01F01F0245
:10E71000012494401C400CB1012000E0002010BDF9
:10E720000010024000210B4A11700A4A203A82F878
:10E730002010012802D0042808D103E00121054A55
:10E74000117004E00521034A117000E000BF00BF12
:10E75000704700002010024010B5012000F034F88E
:10E7600010B1012000F028F8022000F02DF8C0B10F
:10E7700001220CA1002004F0D3FC01200D490870F7
:10E780004004F8F763FA0120FEF7CCFB10B101203A
:10E79000FEF79EFB00F086F8022000F00DF800F076
:10E7A00081F810BD74696D6520636F6D696E670DCA
:10E7B0000A0000003C030020024909888143014A05
:10E7C000118070470428004001460020064A128844
:10E7D0000A40D0B2044A121F12880A4012B108B18E
:10E7E000012000E000207047042800404FF4FA6048
:10E7F0000449088001208870C870002008714871A1
:10E8000088717047780400200E488079401CC0B29F
:10E810000C4988713C2813DB002088710846407938
:10E82000401CC0B248713C280ADB002048710846F1
:10E830000079401CC0B20871182801DB0020087163
:10E8400070470000780400200949098801800849C0
:10E85000897881700649C978C170054909790171C3
:10E8600003494979417102498979817170470000F2
:10E870007804002003B5BDF80000094908809DF820
:10E88000020088709DF80300C8709DF804000871AC
:10E890009DF8050048719DF8060088710CBD0000C8
:10E8A0007804002000BF0348008800F02000002802
:10E8B000F9D070470428004038B5002407E022480A
:10E8C000224941F82400002021490855641C052CE8
:10E8D000F5DD00241FE004EB440000EBC4021D48FA
:10E8E00000EB8200411D1B489338F7F73CF918B93B
:10E8F00001201749085502E002201549085504EB8C
:10E90000440000EBC401134800EB8100401D0F4997
:10E9100041F82400641C0F48A83890F86D00A0420C
:10E92000D9DC0C48A838408928B90BA007490860F1
:10E930000020074908550648084B0022034900906B
:10E940000748FCF795F838BDF8030020B4310020E3
:10E95000F9030020A4320020BFD50000E803002006
:10E960000C2F002038B5002407E02248224941F846
:10E970002400002021490855641C052CF5DD0024E5
:10E980001EE004EB440000EBC4021D4800EB8200D3
:10E99000811D1C48F7F7E7F818B9012017490855F9
:10E9A00002E002201549085504EB440000EBC401C5
:10E9B000134800EB8100801D0F4941F82400641CBE
:10E9C0001048423890F86F00A042DADC0D48423817
:10E9D000808928B90CA0084908600020074908551B
:10E9E00006480A4B0022044900900948FCF740F809
:10E9F00038BD000014040020CC3100201504002094
:10EA0000803300203E320020BFD5000004040020E7
:10EA10000C2F00201CB5002407E03648364941F889
:10EA20002400002035490855641C052CF5DD002420
:10EA30002FE0334890F87100001B401EC0EBC0016E
:10EA400001EB40112F480844807808B9012000E00C
:10EA500000202A4908552A4890F87100001B401EE2
:10EA6000C0EBC00101EB401126480844C01C2249FC
:10EA700041F82400224890F87100001B401EC0EBB2
:10EA8000C00101EB40111F48084440781E49085559
:10EA9000641C1B4890F87100A042CADC1848C08969
:10EAA00038B91AA0144908600020144908551649BD
:10EAB00008551348C08918B900201549C88005E0D9
:10EAC0000F4890F87100401E1149C8801148007825
:10EAD00020B100200E49C8800E4908700A48074935
:10EAE0000D4B0022CDE9001003490948FCF724F83A
:10EAF0001CBD000030040020E4310020310400205F
:10EB0000FC3100205C34002037040020BFD5000019
:10EB10000C2F002040030020200400202DE9F047A6
:10EB200004460D4617469846002C02DA0020BDE840
:10EB3000F08718484068A04201D80020F7E7E9199B
:10EB400004EB440000EBC4021248083000EB8200E2
:10EB5000406A81420AD904EB440000EBC4010D482D
:10EB6000083000EB8100406A461B00E03E4604EBA3
:10EB7000440000EBC4010748083000EB8100806AC4
:10EB800000EB0509B2B2494640460AF05FFC304648
:10EB9000CDE700007C360020F0B505460B46164652
:10EBA000002700240DE0281900F00EFB024638462D
:10EBB0007F1C1A544FEA122C38467F1C03F800C001
:10EBC000A41CB442EFDBF0BD70B5D6B000264FF404
:10EBD0009772DA49DA48FFF7DFFFD84890F82A1130
:10EBE000D8A008F0C5FF4FF497720AA9DD48FFF7D7
:10EBF000D3FF9DF85211DCA008F0BAFF0025E1A177
:10EC0000CE48C01CF6F7AFFF78B9CC48D0F8170053
:10EC1000DD49884209D3C948D0F817000022DB4BF0
:10EC2000181A72EB020100DB01250024D5A10DF1B9
:10EC30002B00F6F798FF68B9DDF83F00D24988420B
:10EC400008D3DDF83F100022D04B591A72EB0200B6
:10EC500000DB0124002D7DD1002CFCD10122CCA1B0
:10EC6000002004F05DFA4FF49771B448F6F73FFFC7
:10EC7000C020B249087088204870C2A1AF48C01CAB
:10EC8000F6F77FFF6B20AD49A1F8110040F26E50FE
:10EC9000A1F81300401DA1F81500BB48C1F81700EA
:10ECA000002081F8CB00BFA1A4481B30F6F769FF14
:10ECB000BCA1A2484330F6F764FFBCA19F486B306B
:10ECC000F6F75FFFBBA19D488A30F6F75AFFB9A15E
:10ECD0009A48A930F6F755FF04209849A1F8C800D2
:10ECE000B6A19648DD30F6F74CFFB5A19348E03069
:10ECF000F6F747FFB3A1B448F6F743FFB3A1B24814
:10ED00002038F6F73EFFB3A1AF480C30F6F739FFD5
:10ED1000B4A1AD481C30F6F734FF0120874981F8D3
:10ED20000D0181F8290181F80E01002081F82501EB
:10ED300081F8260181F8270181F8280181F82A014C
:10ED40009AA17E486B30F6F71CFF00207B4981F8C2
:10ED5000CA0000E004E0082081F82D01012630E01F
:10ED6000012D07D134B90122A0A1002004F0D8F967
:10ED7000022626E075B9012C0CD10122A0A10020A9
:10ED800004F0CEF94FF497720AA96C48F6F796FE94
:10ED9000032616E0012D0FD1012C0DD16748D0F8C4
:10EDA0001700DDF83F10884206D0012299A100200B
:10EDB00004F0B6F9022604E001229BA1002004F031
:10EDC000AFF95E48B0F811006B281CD06B205B498E
:10EDD000A1F8110083A17C481C30F6F7D2FE042074
:10EDE0005649A1F8C800002081F8250181F82601C4
:10EDF00081F8270181F8280181F82A0101260122E2
:10EE00008CA104F08DF94D48B0F8C800052804D352
:10EE100004204A49A1F8C8000126484890F80D018D
:10EE2000012804DD0120454981F80D0101264348F0
:10EE300090F82901012804DD0120404981F82901C9
:10EE400001263E4890F80E01012804DD01203B49CF
:10EE500081F80E010126394890F82501022804DDC9
:10EE60000020364981F80D010126344890F826012A
:10EE7000012804DD0020314981F8260101262F48B0
:10EE800090F82701032804DD00202C4981F8270190
:10EE900001262A4890F82801012804DD002027498E
:10EEA00081F828010126254890F82A01042804DD6C
:10EEB0000020224981F82A010126204890F82D01DE
:10EEC0000B2803DD0B201D4981F82D01012E04D0F4
:10EED000022E03D0032E10D101E000BF00BF334645
:10EEE00058A22821684608F053FE694659A008F048
:10EEF0003FFE684600F06CF900E000BF00BF3248FA
:10EF00003738F9F769FC01280BD12F4B373B53A257
:10EF10002821684608F03CFE01226946002004F0E2
:10EF2000FFF8012251A1002004F0FAF8034890F8FC
:10EF3000CA1052A008F01CFE56B070BDB8250020C3
:10EF400000F8010873757450726F647563745061D2
:10EF500072612E4C4344536574496E6465783D2557
:10EF6000640D0A0000F001086261636B7570506106
:10EF700072612E4C4344536574496E6465783D2537
:10EF8000640D0A004D32310040420F0000EA56FA8B
:10EF90005B315D52737420616C6C20706172612111
:10EFA00000000000302E302E302E300063746E656D
:10EFB00074000000636172640000000034470000C8
:10EFC000636E00006C636E00BB2600203332323566
:10EFD00000000000303030303030303030303030F1
:10EFE000303000006F70656E000000005B325D6DB8
:10EFF00061696E2D2D3E6261636B757000000000CB
:10F000005B335D6261636B75702D2D3E6D61696E62
:10F01000000000005B345D6D61696E2D2D3E626104
:10F02000636B7570000000005B355D4C6F67696352
:10F030004F6B00005B365D5665722D4368616E67ED
:10F0400065640000524541445F504152415F256470
:10F050000000000025730D0A000000005B30315DE8
:10F060006861726449443A25730D0A005061726107
:10F07000526561645F446F6E650D0A0041504E5FDA
:10F08000494E4445583A25640D0A00007FB50446B0
:10F090006D461C48C2881C4800EB8200006800F1E5
:10F0A00010014FF4C87220460AF0D0F91548C28802
:10F0B000154800EB82000168022228460AF0C6F9D2
:10F0C00000208DF801000F48C2880F4800EB820035
:10F0D0000168022228460AF02FFA0B481638808869
:10F0E00070B1094816388088401E07491639888053
:10F0F0000846808820B90846007820F00100087092
:10F100007FBD00000C2F00200E1C0020024A108042
:10F11000024A116070470000D4000020D80000208F
:10F1200021B1028842F04002028004E002884FF6DA
:10F13000BF731A40028070470246002013890B40BB
:10F140000BB1012000E0002070470146888970471C
:10F150008181704710B50022028802F441520B8869
:10F160004C8823438C882343CC8823430C89234336
:10F170004C8923438C892343CC8923431A4302803F
:10F18000838B4FF2FF74234083830B8A038210BD6D
:10F1900010B5044600BF02210A48FFF7CDFF002842
:10F1A000F9D021460748FFF7D3FF00BF01210548EA
:10F1B000FFF7C2FF0028F9D00248FFF7C6FFC0B230
:10F1C00010BD000000300140014608887047000073
:10F1D00010B504460420094908614FF497720849A4
:10F1E000084808F03BF86420F7F72DFC4FF49772BD
:10F1F0000349054808F032F810BD00000010014036
:10F20000B825002000F0010800F801087CB504468C
:10F21000002538A13848F6F7A6FC08B9374D00E0BC
:10F22000374D00200190002C2AD036490880F9F78C
:10F23000FBFC30A13048F6F796FC20B9022132A041
:10F2400002F074FF03E0022131A002F06FFF0123FE
:10F2500014229F210020F9F74DFE012001A92F4A19
:10F260001278885401A82E4B0022294600902D4880
:10F27000FBF7FEFB012368229F210020F9F73AFEED
:10F280002048008890B91BA11B48F6F76CFC30B9E8
:10F29000012325A26E210020FAF7D4F81DE00123F6
:10F2A00027A26E210020FAF7CDF816E01548B0F934
:10F2B0000000C82811D10FA10F48F6F754FC30B94F
:10F2C000012324A26E210020FAF7BCF805E00123F7
:10F2D00026A26E210020FAF7B5F80A480088401CE3
:10F2E00000B208490880B0F5C87F01DB0020088023
:10F2F0007CBD0000636E000098260020FC02002008
:10F3000008030020EC020020555342B5F7CAD40090
:10F31000555342206465627567000000B601002005
:10F32000F00200200C2F00205BC9CF5DD1A1D4F1E9
:10F330002020202020205BCFC25DD1A1D4F100008D
:10F340005B55505D2020202020202020205B444F52
:10F35000574E5D005B4D5DB1A3B4E6202020205BDD
:10F36000455849545DCDCBB3F60000005B53415680
:10F37000455D202020202020205B455849545D0019
:10F3800010B52048FBF7B2FC04461F4884422BD13D
:10F390001EA003F0A9F81B488079204981F8CA0013
:10F3A000084690F8CA004000C0EB40101C4A811883
:10F3B0001A488A30F6F7E5FB184890F8CA00400072
:10F3C000401CC0EB4010164A81181448A930F6F7CB
:10F3D000D8FB14A0FFF7FCFEC820DFF854C000DF04
:10F3E0000120144908700CE01348844203D1132013
:10F3F00005F026F805E01148844202D1062005F008
:10F400001FF810BD0C2F00200A04EC00BCB4BDABEB
:10F41000D6D8C6F4B8FCD0C22E2E2E00B8250020B7
:10F42000142E00204D454E555F535741504E00005D
:10F43000198C0108B10000200A047C000A04F400C1
:10F4400038B50446002C43D02248007801280AD061
:10F4500021A003F049F8C820DFF888C000DF0620AB
:10F4600004F0EEFF38BD2048007801280AD11FA023
:10F4700003F03AF8C820DFF86CC000DF062004F083
:10F48000DFFFEFE7F9F7D0FB02211CA002F04EFEF0
:10F49000012314229F210020F9F72CFD0120194996
:10F4A00091F8CA10184A50541046184B00221849B7
:10F4B00000901848FBF7DCFA012368229F21002006
:10F4C000F9F718FD012314A26E210020F9F7BAFF05
:10F4D00000BFC7E7C0040020BDFBD6B9D0DEB8C46A
:10F4E00000000000198C0108DC010020C5E4D6C32F
:10F4F000CEC4BCFECEDE41504E000000C9E8D6C3EB
:10F5000041504E00B8250020F0010020E401002009
:10F51000B80100200C2F00205B4F4B5DC7D0BBBB58
:10F5200020205B50315DCFEAC7E9000010B588B0FC
:10F530001E48FBF7DBFB04461D4884422DD11B48C7
:10F54000C0881C49097888422DD01C2101A8F6F7F3
:10F55000CEFA164880791749087008460078B8B185
:10F5600015A2192101A808F013FB01A8FDF7E0F886
:10F57000012201A9002003F0D3FD0120DFF848C0DB
:10F5800000DF012011490870062004F059FF0AE04D
:10F590000FA002F0A9FF00BFFEE71048844202D18D
:10F5A000062004F04DFF08B010BD00000C2F002015
:10F5B0000A04EC00B601002061742B7A6164736563
:10F5C000743D640D0A000000198C0108AE0400208F
:10F5D0007265626F6F742E2E2E0000000A04F40014
:10F5E00010B51D4800681D49884212D11C4800789A
:10F5F000401C1B490870084600781A49097888425F
:10F6000002DB0020164908701548007802F0E0FA85
:10F6100021E0114800681449884214D1104800784C
:10F6200018B9104800780E4908700D480078002875
:10F6300004DD0B480078401E09490870084800782E
:10F6400002F0C6FA07E0044800680849884202D17F
:10F65000122004F0F5FE10BD5C0000200A04DC005E
:10F66000CC010020DC0100200A04BC000A04F400E4
:10F6700010B50446F4B1F9F7D7FA02210EA002F052
:10F6800055FD012314229F210020F9F733FC0020AF
:10F690000B4908700846007802F09AFA01236822A4
:10F6A0009F210020F9F726FC012306A26E210020ED
:10F6B000F9F7C8FE10BD000041504ECFEAC7E9007F
:10F6C000CC0100205B455849545DB7B5BBD820201C
:10F6D000202020202020000010B51448FBF706FB56
:10F6E00004461348844219D1124890F826010F4964
:10F6F000C98888420BD00D4880790E4981F82601CF
:10F700000DA0FFF765FD0120DFF83CC000DF012000
:10F710000E490870062004F093FE05E00C48844270
:10F7200002D1062004F08CFE10BD00000C2F00203A
:10F730000A04EC00B82500204D454E555F53657412
:10F74000566F6C756D650000198C0108AE040020C1
:10F750000A04F4007CB50446002525A12548F6F7E7
:10F7600002FA08B9244D00E0244D00200190002C3D
:10F770003CD0F9F759FA1EA11E48F6F7F4F920B962
:10F7800002211FA002F0D2FC03E002211FA002F020
:10F79000CDFC012314229F210020F9F7ABFB0120AF
:10F7A0001449E03991F8261101AA505401A81A4BC6
:10F7B0000022294600901948FBF75AF901236822D4
:10F7C0009F210020F9F796FB09A10A48F6F7CBF92B
:10F7D00030B9012312A26E210020F9F733FE05E0B3
:10F7E000012315A26E210020F9F72CFE7CBD00003C
:10F7F000636E000098260020640200207002002042
:10F80000B9A6B7C5C9E8D6C30000000041774D6F5F
:10F810006465205365740000580200200C2F0020FE
:10F820005BC9CF5DD1A1D4F12020202020205BCF67
:10F83000C25DCDCBB3F600005B55505D202020208B
:10F8400020202020205B444F574E5D0010B588B02B
:10F850002648FBF74BFA0446254884423DD123480D
:10F86000C0882449097888423DD01C2101A8F6F7B8
:10F870003EF91E4880791F49087008460078C8B1D3
:10F880001DA002F031FE4FF400401E4908616420C3
:10F89000DFF874C000DF02201C4908606420DFF834
:10F8A00068C000DF02201949091D086010201549B1
:10F8B00008610EE016A002F017FE4FF40040114957
:10F8C00048613220DFF840C000DF0120134981F891
:10F8D0002D032E2004F0B4FD05E01148844202D12E
:10F8E000062004F0ADFD08B010BD00000C2F002074
:10F8F0000A04EC00B70100207265626F6F742E2E4F
:10F900002E00000000100140198C0108100C01406D
:10F910006E6F726D616C2E2E2E000000FC31002087
:10F920000A04F4007CB50446002538A13848F6F7EF
:10F930001AF908B9374D00E0374D00200190002C2E
:10F940002AD036490880F9F76FF930A13048F6F728
:10F950000AF920B9022132A002F0E8FB03E00221FB
:10F9600032A002F0E3FB012314229F210020F9F7CB
:10F97000C1FA012001A9304A1278885401A82F4BFE
:10F980000022294600902E48FBF772F801236822D6
:10F990009F210020F9F7AEFA2048008890B91BA1FA
:10F9A0001B48F6F7E0F830B9012326A26E210020AB
:10F9B000F9F748FD1DE0012328A26E210020F9F788
:10F9C00041FD16E01548B0F90000C82811D10FA17B
:10F9D0000F48F6F7C8F830B9012325A26E210020A0
:10F9E000F9F730FD05E0012327A26E210020F9F789
:10F9F00029FD0A480088401C00B208490880B0F57B
:10FA0000C87F01DB002008807CBD0000636E000021
:10FA10009826002024030020300300201403002037
:10FA2000B9CCBCFEC9FDBCB600000000424F4F542B
:10FA30002075706461746100B70100201803002014
:10FA40000C2F00205BC9CF5DD1A1D4F12020202054
:10FA500020205BCFC25DD1A1D4F100005B55505D89
:10FA60002020202020202020205B444F574E5D0086
:10FA70005B4D5DB1A3B4E6202020205B455849547E
:10FA80005DCDCBB3F60000005B534156455D2020B1
:10FA900020202020205B455849545D0070B5054664
:10FAA0000C46284608F090FCA0B20121DFF808C0FF
:10FAB00000DF0249086070BD89920108340000200F
:10FAC00070B505460C46284608F07EFC0121054825
:10FAD00003F0CEFCA0B2F6F7B6FF0021014803F018
:10FAE000C7FC70BD000C004043185A00FF2A00DD1F
:10FAF0007047034B1870034B197000BFF8E7000004
:10FB0000960000209700002070B504464025012C87
:10FB100017D1F9F789F801210AA002F007FB0123A8
:10FB200014229F210020F9F7E5F9A8B2012308A2C9
:10FB30003821F9F787FCA8B2012307A24A21F9F777
:10FB400081FC70BDB0B4BCFCB2E2CAD400000000BD
:10FB5000B0B4BCFC00000000CEDE000010B50446CE
:10FB60000CB1F9F761F810BD70B504464025012CC1
:10FB700017D1F9F759F801210AA002F0D7FA0123A9
:10FB800014229F210020F9F7B5F93823A022002183
:10FB900006A002F0E0FA4A23A022002106A002F00B
:10FBA000DAFA70BD4C4544B2E2CAD400BAECB5C62C
:10FBB0002D2DB0B455500000C2CCB5C62D2DB0B41B
:10FBC000444F574E0000000030B585B00446402534
:10FBD000012C50D1F9F728F8012147A002F0A6FA2C
:10FBE000012314229F210020F9F784F9444800786A
:10FBF000022806D1012343A226211220F9F722FC74
:10FC000010E03F480078012806D101233EA22621BA
:10FC10001220F9F717FC05E001233CA2262112204F
:10FC2000F9F710FC3B483CA214210368684607F032
:10FC3000AFFF01236A4626212846F9F703FC37481F
:10FC400090F92B01002808DD344890F92B3134A2BB
:10FC50001421684607F09CFF07E0304890F92B31EB
:10FC60002FA21421684607F093FF01236A4638212A
:10FC70001220F9F7E7FB2E480068C82802D02C486C
:10FC8000006830BB2B48006822490968884210D0C0
:10FC9000204800682749086008461FA2142103680D
:10FCA000684607F075FF01236A4626212846F9F7C2
:10FCB000C9FB20480068B0F5D87F0BD91EA21421DB
:10FCC000684607F065FF01236A465C212846F9F77C
:10FCD000B9FB05E06E23A0225C212846F9F778F8ED
:10FCE00013480068401C12490860B0F5C87F01D372
:10FCF0000020086005B030BDB5E7D1B9D6B5000029
:10FD0000E900002053540000484B0000CEB4D6AAAE
:10FD100000000000B400002025640000B825002089
:10FD2000D0A3D7BCD6B5A3BA2530336400000000F9
:10FD3000AC020020B0020020BACFB8F100000000F1
:10FD400010B51448FAF7D2FF04461348844219D17B
:10FD5000124890F825010F49C98888420BD00D48F8
:10FD600080790E4981F825010DA0FFF731FA0120B5
:10FD7000DFF83CC000DF01200E490870062004F0C7
:10FD80005FFB05E00C48844202D1062004F058FBDA
:10FD900010BD00000C2F00200A04EC00B825002044
:10FDA00053657446617374496E7465720000000097
:10FDB000198C0108AE0400200A04F4007CB5044646
:10FDC000002525A12548F5F7CEFE08B9244D00E011
:10FDD000244D00200190002C3CD0F8F725FF1EA1F7
:10FDE0001E48F5F7C0FE20B902211FA002F09EF9BF
:10FDF00003E0022120A002F099F9012314229F219F
:10FE00000020F9F777F801201449E03991F825111D
:10FE100001AA505401A81C4B0022294600901B48FF
:10FE2000FAF726FE012368229F210020F9F762F8E5
:10FE300009A10A48F5F797FE30B9012314A26E21F3
:10FE40000020F9F7FFFA05E0012317A26E21002038
:10FE5000F9F7F8FA7CBD0000636E000098260020D8
:10FE6000100200201C020020BFECBDDDBDE7C3E690
:10FE7000C9E8D6C30000000046617374496E74651A
:10FE80007266616365000000040200200C2F0020F0
:10FE90005BC9CF5DD1A1D4F12020202020205BCFF1
:10FEA000C25DCDCBB3F600005B55505D2020202015
:10FEB00020202020205B444F574E5D0010B5114894
:10FEC00000681149084448B1B0F5001F07D0B0F5EB
:10FED000401F08D0B0F5601F11D105E00FE00BA066
:10FEE00007F046FE0BE00AE00F48007818B906203C
:10FEF00004F0A6FA02E0242004F0A2FA00BF00BF3A
:10FF000010BD00005C000020F6FB43FF475053206B
:10FF1000444F574E2D2D2D2D2D2D2D2D2D2D2D2D8D
:10FF20002D2D0D0A000000006201002030B589B0BF
:10FF30000546002D70D0F8F777FE844890F83D0311
:10FF4000B8B983480078A0B982A18348F5F70BFEC1
:10FF500018B982A002F0C8FA02E084A002F0C4FA44
:10FF60003220DFF814C200DF012004F069FA09B082
:10FF700030BD7748007800282AD18048007800F00A
:10FF80000100002824D17D4890F8780060B171A16B
:10FF90007148F5F7E8FD18B979A002F0A5FA0FE06D
:10FFA00079A002F0A1FA0BE06AA16B48F5F7DBFD3E
:10FFB00018B978A002F098FA02E078A002F094FA5A
:10FFC0003220DFF8B4C100DF012004F039FACEE7B7
:10FFD00060A16148F5F7C7FDF8B9012172A002F0F0
:10FFE000A5F86648838973A21E2101A807F0D0FDF9
:10FFF000012301AA38210020F9F724FA5F48437D44
:020000040801F1
:1000000071A21E2101A807F0C3FD012301AA4A2104
:100010000020F9F717FA1EE042E001216EA002F07D
:1000200085F8564883896EA21E2101A807F0B0FD0D
:10003000012301AA38210020F9F704FA4F48437D33
:100040006CA21E2101A807F0A3FD012301AA4A21E9
:100050000020F9F7F7F94948407D6B490870012302
:1000600014229F210020F8F745FF0020F7F76AFCD3
:1000700038A13948F5F777FD30B9012363A26E2125
:100080000020F9F7DFF905E0012366A26E210020C8
:10009000F9F7D8F92E48007810B15C2002F074F816
:1000A00036480078C0F340003449097801F0010176
:1000B00040EA012031490978C1F3001140EA810486
:1000C0005D480088A04207D05B4804802048007843
:1000D00010B15C2002F058F858480078401CC0B2BB
:1000E00056490870C8282FDB0020F7F72BFC23485F
:1000F000407D45490978884223D016A11648F5F776
:1001000032FD68B91D48437D2FA21E2101A807F0CA
:100110003FFD012301AA4A210020F9F793F90CE0E1
:100120001648437D33A21E2101A807F031FD0123AB
:1001300001AA4A210020F9F785F91048407D32498B
:10014000087000203D49087000BF10E7FC31002016
:1001500062010020636E000098260020C4A3BFE95E
:10016000B3F5CABCBBAFD6D0000000004D6F6465CC
:100170006D20696E69742100198C01084C350020CE
:10018000CEB4B4F2BFAA00006E6F74206F70656EBB
:1001900021000000B2BBD6A7B3D600006E6F20735B
:1001A0007570706F72742100B1B1B6B7C9E8D6C36B
:1001B0000000000020B1B1B6B7C9CFB4ABCAB1BC22
:1001C000E43A256420C3EB0020D3D0D0A7CEC0D022
:1001D000C73A25642000000047505320536574003F
:1001E00055706C6F61642074696D653A20256420D8
:1001F000530000005374617274204E756D62657215
:100200003A25642000000000F80100202020202072
:100210002020202020205B455849545DCDCBB3F6EB
:10022000000000002020202020202020202020204E
:10023000205B455849545D00F6010020F401002080
:10024000FEB5054600260C24012D4CD1F8F7ECFC38
:1002500070A17148F5F787FC20B901216FA001F06A
:1002600065FF03E0012170A001F060FF012314226B
:100270009F210020F8F73EFE66A16748F5F773FC62
:1002800030B9A0B201236CA23821F9F7DBF805E000
:10029000A0B201236CA23821F9F7D4F85E4B3F33AA
:1002A0006CA20A21684607F073FC6846F5F754FC17
:1002B000C6B204F1500188B201236A463821F9F729
:1002C000C1F8F20004F1500188B20E233821F8F78A
:1002D00049FF012368229F210020F8F70BFE002030
:1002E0005D4908805DE0022D5BD100200090019007
:1002F00002905A480078401C5849087058A1464856
:100300003F30F5F730FCA8B95449087800EBD071BC
:100310004910A0EB410131B153A34EA20A21684616
:1003200007F036FC1BE04EA34AA20A21684607F0FC
:100330002FFC14E04949087800EBD0714910A0EB7C
:10034000410131B146A343A20A21684607F020FCCF
:1003500005E045A33FA20A21684607F019FC68465C
:10036000F5F7FAFBC6B204F1500188B20E23A022C1
:100370003821F8F7A5FC04F1500188B201236A4640
:100380003821F9F75FF8F20004F1500188B20E232A
:100390003821F8F7E7FE012368229F210020F8F7B3
:1003A000A9FD2D48008890B91AA11B48F5F7DBFB81
:1003B00030B901232EA26E210020F9F743F81CE08A
:1003C000012331A26E210020F9F73CF815E0224804
:1003D0000088C82811D10FA10F48F5F7C4FB30B928
:1003E00001232EA26E210020F9F72CF805E001234D
:1003F00030A26E210020F9F725F817480088401C2C
:1004000080B215490880B0F5C87F01DB0020088064
:10041000FEBD0000636E000098260020B0B4BCFC56
:10042000D2F4C9E8D6C300004B6579536F756E648A
:10043000205365740000000020BCFCD2F4BFAAB9B0
:10044000D83A202020200000202053776974636868
:100450003A20200025730000000200200202002044
:100460006F70656E00000000636C6F7365000000C4
:100470005BC9CF5DD1A1D4F12020202020205BCF0B
:10048000C25DD1A1D4F100005B55505D2020202039
:1004900020202020205B444F574E5D005B4D5DB116
:1004A000A3B4E6202020205B455849545DCDCBB352
:1004B000F60000005B534156455D2020202020209F
:1004C000205B455849545D0010B52748006827490E
:1004D000084448B1B0F5001F0FD0B0F5401F15D04B
:1004E000B0F5601F3DD138E021480078401C20491C
:1004F00008700220FFF7A4FE33E01D480078401C7E
:100500001B4908700220FFF79BFE2AE01849087873
:1005100000EBD0714910A0EB410119B9062003F09E
:100520008FFF0DE013A11548F5F71DFB20B914A1AD
:100530001248F5F726FB03E00EA11048F5F721FB62
:1005400011A007F015FB18A0FEF742FE0120194983
:100550000870062003F074FF03E0062003F070FF2C
:1005600000BF00BF10BD00005C000020F6FB43FF91
:10057000030200206F70656E00000000D726002087
:10058000636C6F736500000073746172742073652F
:10059000742D2D2D2D2D2D2D2D2D2D2D2D2D2D2D44
:1005A0002D2D2D2D2D0D0A004D454E555F535747CE
:1005B00050530000AE04002010B504242448006805
:1005C0002449084448B1B0F5001F14D0B0F5401FCD
:1005D00022D0B0F5601F39D134E01F480078401CAC
:1005E000C0B21D490870052801DB002008700220F8
:1005F00000F03CF82AE018480078002805DD16488D
:100600000078401E1449087002E004201249087066
:10061000022000F02BF819E0104890F82A010E494A
:10062000097888420DD001200D4908700A480078E9
:100630000A4981F82A010BA0FEF7CAFD022003F047
:10064000FFFE03E0022003F0FBFE00BF00BF10BD71
:100650005C000020F6FB43FFB0010020B82500201D
:10066000AE0400204C43447061726D0030B585B01B
:1006700005460424012D7DD1804890F82A01804947
:100680000870F8F7D1FA7FA17C48E030F5F76BFAF3
:1006900080B901217CA001F049FD012314229F2192
:1006A0000020F8F727FCA0B2012379A23821F8F73F
:1006B000C9FE0FE001217AA001F038FD01231422C8
:1006C0009F210020F8F716FCA0B2012376A2382162
:1006D000F8F7B8FE6A480078042811D169A1674884
:1006E000E030F5F740FA28B973A20A2102A807F012
:1006F0004FFA17E072A20A2102A807F049FA11E0A6
:100700005F480078704931F8103070A20A2102A8C1
:1007100007F03EFA04F1810188B201236CA238216E
:10072000F8F790FE04F18000C2B23038C1B238232D
:1007300002A801F010FD04F1500188B20E2330220E
:100740003821F8F70FFD4E48037860A2062168466D
:1007500007F01EFA01226946002002F0E1FC0123A5
:1007600068229F210020F8F7C5FB00205949088026
:1007700049E0FFE7022D46D104F1500188B24C2335
:10078000A0223821F8F724FB3D480078042811D135
:100790003CA13A48E030F5F7E6F928B946A20A212B
:1007A00002A807F0F5F917E045A20A2102A807F010
:1007B000EFF911E032480078434931F8103043A294
:1007C0000A2102A807F0E4F904F1810188B20123AB
:1007D0003FA23821F8F736FE04F18000C2B230386B
:1007E000C1B2382302A801F0B6FC04F1500188B26E
:1007F0000E2330223821F8F7B5FC012368229F210F
:100800000020F8F777FB3348008898B91DA11B48F2
:10081000E030F5F7A8F930B901232FA26E210020AE
:10082000F8F710FE1DE0012331A26E210020F8F739
:1008300009FE16E027480088C82812D111A10F48E8
:10084000E030F5F790F930B901232EA26E21002097
:10085000F8F7F8FD05E0012330A26E210020F8F73B
:10086000F1FD1C480088401C80B21A490880B0F590
:10087000C87F01DB0020088005B030BDB82500200E
:10088000B0010020636E00004C4344C9E8D6C300A9
:1008900020B1B3B9E2CAB1BCE43A20202020000064
:1008A0004C434420536574004C6967687454696D07
:1008B000653A202020200000B3A3C1C10000000041
:1008C0004B656570000000009A010020253364002C
:1008D00020530000FA0100205BC9CF5DD1A1D4F103
:1008E0002020202020205BCFC25DD1A1D4F10000C8
:1008F0005B55505D2020202020202020205B444F8D
:10090000574E5D005B4D5DB1A3B4E6202020205B17
:10091000455849545DCDCBB3F60000005B534156BA
:10092000455D202020202020205B455849545D0053
:1009300000B58FB03B4800683B49084448B1B0F56A
:10094000001F0FD0B0F5401F15D0B0F5601F65D166
:100950005DE036480078401C34490870022000F001
:1009600085F85BE031480078401C3049087002206F
:1009700000F07CF852E02D49087800EBD071491066
:10098000A0EB410119B9062003F05AFD1DE000203B
:100990002649087026A12748F5F7E5F888B926A169
:1009A0002448F5F7EEF82348E03890F827010228AC
:1009B0000BDD00201F49E03981F82701F7F756FCCD
:1009C00003E01BA11B48F5F7DCF81CA0FEF700FCB8
:1009D00001201D490870062003F032FD14A11548BE
:1009E000F5F7C1F828B93C2218A16846F5F7A8F830
:1009F00004E03C2219A16846F5F7A2F801226946F5
:100A0000002002F08DFB6846FBF792FE06E0002016
:100A100006490870062003F013FD00BF00BF0FB0A9
:100A200000BD00005C000020F6FB43FFA401002095
:100A3000636E000098260020656E00004D454E55FF
:100A40005F53574750530000AE04002041542B50D1
:100A50004F433D35313226300D0A000041542B50B2
:100A60004F433D35313226310D0A0000FEB50546B3
:100A700000260C24012D57D1F8F7D6F872A173483F
:100A8000F5F771F820B9012171A001F04FFB03E0E7
:100A9000012172A001F04AFB012314229F210020B2
:100AA000F8F728FA68A16948F5F75DF830B9A0B2FF
:100AB00001236EA23821F8F7C5FC05E0A0B201239E
:100AC0006EA23821F8F7BEFC5FA16048F5F74BF83D
:100AD00030B96EA36FA20A21684607F059F805E005
:100AE0006DA36CA20A21684607F052F86846F5F734
:100AF00033F8C6B204F1500188B201236A463821A6
:100B0000F8F7A0FCF20004F1500188B20E2338215E
:100B1000F8F728FB012368229F210020F8F7EAF963
:100B200000205F49088057E0022D55D10020009039
:100B30000190029044A14548F5F715F8A8B9594924
:100B4000087800EBD0714910A0EB410131B152A3FC
:100B500050A20A21684607F01BF81BE04BA34DA2E8
:100B60000A21684607F014F814E04E49087800EBB3
:100B7000D0714910A0EB410131B144A345A20A2133
:100B8000684607F005F805E043A342A20A2168463B
:100B900006F0FEFF6846F4F7DFFFC6B204F150012D
:100BA00088B24823A0223821F8F712F904F1500145
:100BB00088B201236A463821F8F744FCF20004F1B8
:100BC000500188B210233821F8F7CCFA01236822AB
:100BD0009F210020F8F78EF93148008890B91AA1BA
:100BE0001A48F4F7C0FF30B901232FA26E2100206C
:100BF000F8F728FC1CE0012331A26E210020F8F751
:100C000021FC15E026480088C82811D10EA10F4804
:100C1000F4F7A9FF30B901232EA26E210020F8F7C6
:100C200011FC05E0012331A26E210020F8F70AFC37
:100C30001B480088401C80B219490880B0F5C87F65
:100C400001DB00200880FEBD636E000098260020B6
:100C5000D3EFD6D6C9E8D6C3000000004C616E675A
:100C600075616765732053657400000020D3EFD66B
:100C7000D6D1A1D4F13A20202020000020204368C2
:100C80006F6963653A20202020000000D6D0CEC4D2
:100C90000000000025730000456E676C69736800F2
:100CA000FE010020A40100205BC9CF5DD1A1D4F1D9
:100CB0002020202020205BCFC25DD1A1D4F10000F4
:100CC0005B55505D2020202020202020205B444FB9
:100CD000574E5D005B4D5DB1A3B4E6202020205B44
:100CE000455849545DCDCBB3F60000005B534156E7
:100CF000455D202020202020205B455849545D0080
:100D000010B50446082C36D2DFE804F0040B352772
:100D10001219202E002019490870012000F030F827
:100D200029E0012015490870052000F029F822E08B
:100D3000042012490870062000F022F81BE005206C
:100D40000E490870042000F01BF814E006200B493F
:100D50000870012000F014F80DE003200749087026
:100D6000042000F00DF806E0072004490870022076
:100D700000F006F800BF00BF10BD00009900002081
:100D800010B504460A2C60D2DFE804F0050E1720E7
:100D900029323B444D560021084600F00BFC00214F
:100DA0000846FEF7A1FE50E00021012000F002FC01
:100DB00000210846FEF798FE47E00521012000F0DB
:100DC000F9FB00210846FEF78FFE3EE00A210120D4
:100DD00000F0F0FB00210846FEF786FE35E000211A
:100DE000084600F0E7FB00210120FEF77DFE2CE025
:100DF0000021084600F0DEFB01210846FEF774FEE4
:100E000023E00021084600F0D5FB0C210120FEF76D
:100E10006BFE1AE00021012000F0CCFB0021012034
:100E2000FEF762FE11E00121084600F0C3FB01213C
:100E30000846FEF759FE08E00A21012000F0BAFB3F
:100E40000A210120FEF750FE00BF00BF10BD0000C8
:100E50007CB50446002525A12548F4F784FE08B991
:100E6000244D00E0244D00200190002C3CD0F7F7E9
:100E7000DBFE1EA11E48F4F776FE20B902211FA05A
:100E800001F054F903E002211FA001F04FF9012302
:100E900014229F210020F8F72DF801201449E03991
:100EA00091F8281101AA505401A81B4B0022294691
:100EB00000901A48F9F7DCFD012368229F210020E9
:100EC000F8F718F809A10A48F4F74DFE30B90123E4
:100ED00013A26E210020F8F7B5FA05E0012316A24F
:100EE0006E210020F8F7AEFA7CBD0000636E0000B2
:100EF000982600208802002094020020B5CDB9A6D3
:100F0000BAC4C9E8D6C300004C6F77436F6E7375DF
:100F10006D7074696F6E00007C0200200C2F002041
:100F20005BC9CF5DD1A1D4F12020202020205BCF50
:100F3000C25DCDCBB3F600005B55505D2020202074
:100F400020202020205B444F574E5D0010B52A48DA
:100F5000F9F7CCFE04462948844245D1284890F848
:100F600028012549C988884237D0234880792449F7
:100F700081F82801084690F82801D0B9084690F871
:100F8000270120B1012805D0022809D105E0F7F793
:100F90006DF905E0F7F76AF902E0F7F767F900BFC6
:100FA00000BF1E20DFF85CC000DF17A0FBF7C0FB0E
:100FB0000CE00120124981F82701F7F757F91E20AC
:100FC000DFF840C000DF14A0FBF7B2FB16A0FEF76D
:100FD000FFF80120DFF82CC000DF0120164908705F
:100FE000062003F02DFA05E01448844202D10620C1
:100FF00003F026FA10BD00000C2F00200A04EC00BC
:10100000B8250020198C010841542B504F433D3521
:10101000353826300D0A000041542B504F433D35E2
:10102000353826310D0A00004D454E555F53657425
:10103000566F6C756D650000AE0400200A04F40064
:1010400038B50546002407E0E00025FA00F0C0B2FC
:101050000DF80400601CC4B2042CF5DB0422D1049A
:10106000684608F069FA38BD70B500252E48F9F7D2
:101070003DFE04462D4884424DD12D4890F828016C
:1010800001281DD12BA12A48E030F4F76CFD18B9D6
:1010900029A001F029FA02E02CA001F025FA32255E
:1010A00002E00120FBF7E4FE281EA5F10101CDB20C
:1010B000F7D1012029490870062003F0C1F970BD5D
:1010C000194880791A4981F8270125A0FEF780F890
:1010D0000120DFF89CC000DF154890F8270130B1EF
:1010E000012807D0022808D003280CD108E0F7F720
:1010F000BDF808E0F7F7BAF805E0F7F7B7F802E04F
:10110000F7F7B4F800BF00BF0120144908700620AB
:1011100003F096F905E01748844202D1062003F057
:101120008FF900BFCBE700000C2F00200A04EC0071
:10113000B8250020636E0000B5CDB9A6BAC4D6D0DC
:10114000CEDEB7A8C9E8D6C300000000556E6162C4
:101150006C6520746F20736574000000AE0400207D
:101160004D454E555F536574566F6C756D65000047
:10117000198C01080A04F4007CB50446002525A159
:101180002548F4F7F0FC08B9244D00E0244D002078
:101190000190002C3CD0F7F747FD1EA11E48F4F744
:1011A000E2FC20B902211FA000F0C0FF03E00221F1
:1011B0001FA000F0BBFF012314229F210020F7F79E
:1011C00099FE01201449E03991F8271101AA5054E1
:1011D00001A81A4B0022294600901948F9F748FC4B
:1011E000012368229F210020F7F784FE09A10A4805
:1011F000F4F7B9FC30B9012312A26E210020F8F7F0
:1012000021F905E0012315A26E210020F8F71AF953
:101210007CBD0000636E0000982600203402002090
:1012200048020020CDF8C2E7C9E8D6C3000000009C
:101230004E65744D6F64652053657400280200206C
:101240000C2F00205BC9CF5DD1A1D4F1202020203C
:1012500020205BCFC25DCDCBB3F600005B55505D67
:101260002020202020202020205B444F574E5D006E
:10127000F8B504462046F6F7EDFC06463046F6F78C
:1012800005FD054605B9F8BD6B4602221C21304616
:10129000FDF744FCBDF80000082800D0F3E7044B3C
:1012A0004FF4806236213046FDF738FC00BFEAE794
:1012B000F478002010B51A4800681A4988421FD1F6
:1012C000012219A1002001F02BFF1AA001F00CF956
:1012D00001201B490860F8F7FDF96420DFF864C0BD
:1012E00000DF01201649091D0860F8F7F3F9DC203A
:1012F000DFF850C000DF04201349486100BFFEE75B
:10130000074800681149884209D11148007818B986
:10131000012003F095F802E0242003F091F810BDBD
:101320005C0000200A04EC005077724F66664F6B39
:1013300000000000D5FDD4DAB9D8BBFA2E2E2E005D
:10134000100C0140198C0108001001400A04F4003F
:10135000620100207CB50446002500263CA13D48E2
:10136000F4F701FC08B93C4D00E03C4D0020019031
:10137000002C33D03A490880F7F756FC34A13548A1
:10138000F4F7F1FB20B9022136A000F0CFFE03E014
:10139000022138A000F0CAFE012314229F21002060
:1013A000F7F7A8FD2B48E03890F80D012949E039FE
:1013B00091F8291140EA4100C6B2012001A98855DF
:1013C00001A82F4B0022294600902E48F9F750FB28
:1013D000012368229F210020F7F78CFD2048008818
:1013E00090B91BA11B48F4F7BEFB30B9012326A21C
:1013F0006E210020F8F726F81DE0012328A26E21B7
:101400000020F8F71FF816E01548B0F90000C828CA
:1014100011D10FA10F48F4F7A6FB30B9012325A283
:101420006E210020F8F70EF805E0012327A26E21B7
:101430000020F8F707F80A480088401C00B2084965
:101440000880B0F5C87F01DB002008807CBD00006B
:10145000636E000098260020C4020020D8020020FD
:10146000B4020020505454CCE1CABED2F4C9E8D62C
:10147000C3000000507474546F6E6520536574008F
:10148000B80200200C2F00205BC9CF5DD1A1D4F1A0
:101490002020202020205BCFC25DD1A1D4F100000C
:1014A0005B55505D2020202020202020205B444FD1
:1014B000574E5D005B4D5DB1A3B4E6202020205B5C
:1014C000455849545DCDCBB3F60000005B534156FF
:1014D000455D202020202020205B455849545D0098
:1014E00030B589B000242348F9F700FC05462248AE
:1014F000854237D1214890F80D01204991F82911F2
:1015000040EA4100C4B21B48C088A04223D01C213D
:1015100002A8F4F7ECFA1748847904F0010017499F
:1015200081F80D01601081F8290115A0FDF750FE2A
:10153000124890F829010090104890F80D3114A23B
:10154000192102A806F024FB02A8FBF7F1F80120FC
:10155000DFF854C000DF012014490870062002F0B3
:101560006FFF05E01248854202D1062002F068FFB5
:1015700009B030BD0C2F00200A04EC00B825002073
:101580004D454E555F536574507474546F6E6500CD
:1015900041542B504F433D35313126256426256477
:1015A00026310D0A00000000198C0108AE0400204D
:1015B0000A04F40043185A00FF2A00DD7047034B69
:1015C0001870034B197000BFF8E70000940000206A
:1015D0009500002030B587B00546184890FBF5F01F
:1015E00084B2ADF814400320ADF810000020ADF82F
:1015F0001600ADF812008DF8180004A9104801F08B
:10160000FBFF7020ADF80000204604EBD0714910BC
:10161000ADF806100120ADF802000220ADF8080078
:101620006946074801F040FF0821054801F088FF9E
:101630000121034801F01CFF07B030BD002D31012E
:10164000000C004010B51948FAF728FC0446184869
:10165000844223D115484079052818D2DFE800F0EC
:1016600003070B0F13001F2002F0EAFE0FE02A20F1
:1016700002F0E6FE0BE01A2002F0E2FE07E02B206B
:1016800002F0DEFE03E02C2002F0DAFE00BF00BF15
:10169000064841790748FCF773FF05E00648844295
:1016A00002D1022002F0CCFE10BD0000900100200B
:1016B0000A04EC00103100200A04F40010B50446BE
:1016C00034B1F7F7B1FA03A200210846F7F746FE56
:1016D00010BD00007570646174652E626D7000004D
:1016E00010B500F001F810BD0CB50020019000907D
:1016F0003348006840F480303149086000BF30480A
:10170000006800F4003000900198401C019000989F
:1017100020B94FF6FF7101988842F0D1284800683F
:1017200000F4003010B10120009001E00020009092
:101730000098012843D12348006840F01000214957
:1017400008600846006820F003000860084600684A
:1017500040F0010008601A4840681949486008468E
:10176000406848600846406840F480604860084629
:10177000406820F47C1048600846406840F410201F
:1017800048600846006840F08070086000BF0C4860
:10179000006800F000700028F9D00948406820F087
:1017A0000300074948600846406840F0020048606E
:1017B00000BF0348406800F00C000828F9D10CBDB8
:1017C000001002400020024010B50D4800680D498D
:1017D000884201D1F5F710FB0B484078012807D06B
:1017E000F5F70AFB00220949104601F099FC10BDEB
:1017F00001F0D4FC01F0C8FF04F0D2FD00BFF6E711
:101800005C0000200A04F40040000020409701081A
:1018100010B586B0444800684449884223D1192055
:1018200002F00EFE1823A02238210020F7F748FA14
:1018300001233F4A28210420F7F704FE01233D4AF3
:1018400046210420F7F7FEFD01233B4A6E210020CC
:10185000F7F7F8FDF7F73EFFC820DFF8E0C000DF3C
:10186000FBF78AFA5EE0304800683549884203D1C8
:10187000062002F0E5FD55E02B480068314988421A
:1018800004D029480068304988422CD100242648D9
:1018900000682C49884207D12C480088401C2B49FD
:1018A0000880601CC4B20FE01F48006826498842C7
:1018B0000AD1264800886C2806DD24480088401E8E
:1018C00022490880601CC4B244B32048038820A287
:1018D000132101A806F05CF9012301AA442100208C
:1018E000F7F7B0FD1EE0104800681D49884216D188
:1018F0001C48007840B900201B490870194800783E
:10190000401C184908700DE017480078032809DDCD
:101910001A2002F095FD00201249087002E0002014
:101920001049087006B010BD5C0000200A04EC00ED
:1019300086990108AE990108C2990108198C01081D
:101940000A04F4000A04BC000A04DC001C000020A5
:1019500020202020C9FDBCB6B5BD3A562564200024
:101960000A04F800280000206100002010B588B0AB
:101970000446002C33D06C201A490880F7F754F93C
:101980000021194800F0D2FB012314229F210020DE
:10199000F7F7B0FA6B2315A21E21684606F0F8F897
:1019A00001236A462C210020F7F74CFD0D480388DF
:1019B00013A21E21684606F0EBF801236A46442173
:1019C0000020F7F73FFD012368229F210020F7F751
:1019D00091FA01230E4A6E210020F7F733FD08B07B
:1019E00010BD00001C000020D6990108202020B561
:1019F000B1C7B0B0E6B1BE3A205625642020200021
:101A000020202020C9FDBCB6B5BD3A562564200073
:101A1000E399010810B517480068174988421CD19E
:101A200016A11748F4F79FF818B916A000F05CFD4E
:101A300002E018A000F058FD1C480078401C1B492B
:101A4000087008460078022807D10020087018A006
:101A5000FAF76EFE012002F0F3FC0648006819490F
:101A6000884205D1002011490870062002F0E8FCE8
:101A700010BD00005C0000200A04EC00636E000052
:101A800098260020C9FDBCB6D6C1D7EED0C2B0E6BC
:101A9000B1BE3F0055706772616465204E65772066
:101AA00056657273696F6E3F00000000FC010020F4
:101AB00041542B504F433D353432263026300D0AE9
:101AC000000000000A04F40010B50446002C3FD0CA
:101AD000F7F7AAF81FA12048F4F745F820B901212B
:101AE0001EA000F023FB03E0012120A000F01EFB5C
:101AF000012314229F210020F7F7FCF915A11648B5
:101B0000F4F731F830B901231CA238211020F7F77F
:101B100099FC05E001231EA238210020F7F792FC72
:101B2000012368229F210020F7F7E4F909A10A4860
:101B3000F4F719F830B901231AA26E210020F7F743
:101B400081FC05E001231DA26E210020F7F77AFC3D
:101B500010BD0000636E000098260020C9FDBCB6D1
:101B6000B6D4BDB2B0E6B1BE0000000053797374C4
:101B7000656D20557064617465000000C9FDBCB6D8
:101B8000B5BDD7EED0C2B0E6B1BE3F200000000028
:101B900055706772616465204E6577205665727373
:101BA000696F6E005B4D5DC9FDBCB6202020205BD7
:101BB000455849545DCDCBB3F60000005B4F4B5DFB
:101BC00020202020202020205B455849545D000023
:101BD0002DE9F04194B08046002616250E24672397
:101BE0009F2229460020F7F7F3F85748574909780C
:101BF00050F8213056A228210AA805F0C9FF324624
:101C0000761C102000FB025101230AAA1846F7F7A0
:101C100019FC4E4909784900C1EB41114D4A881819
:101C2000F3F79AFFC7B2494800784000C0EB401074
:101C3000484A811822466846F3F740FF00200DF815
:101C400004006B4644A228210AA805F0A1FF3246F1
:101C5000761C102000FB025101230AAA1846F7F750
:101C6000F1FBA7421FDD394800784000C0EB40106F
:101C7000384A104401196846F3F783FF6B4638A2CF
:101C800028210AA805F084FF0020391B0AAA505415
:101C90003046721CD6B2102202FB005101230AAA60
:101CA0001846F7F7CFFB294909784900491CC1EBD1
:101CB0004111284A8818F3F74FFFC7B2234800782C
:101CC0004000401CC0EB4010224A81182246684662
:101CD000F3F7F4FE00200DF804006B4621A2282142
:101CE0000AA805F055FF3046721CD6B2102202FB3E
:101CF000005101230AAA1846F7F7A4FBA74220DDEA
:101D0000124800784000401CC0EB4010114A1044BB
:101D100001196846F3F735FF6B4611A228210AA87E
:101D200005F036FF0020391B0AAA50543046721CB9
:101D3000D6B2102202FB005101230AAA1846F7F777
:101D400081FB14B0BDE8F081B8010020CC01002077
:101D500025733A00142E00204E616D653A257300FC
:101D600025730000506173733A257300F8B5064679
:101D70000F465A248B48007820B30325B6F5D37F4D
:101D800005DC4FF400418848F5F764FDA8B98748A1
:101D9000007870B98648007858B904F1290188B2F2
:101DA00084A20321F7F7DAFA4FF4804085490861ED
:101DB000F8BD4FF48040834948614FF4D2708249A6
:101DC000088008E04FF480407E494861012540F2D8
:101DD00097107D490880B6F5B07F1EDCDFF8ECC1B6
:101DE00000DF7B490968884200D2E1E7DFF8DCC107
:101DF00000DF5030764908607648007830B900201E
:101E0000754908700120734908701FE0002071496E
:101E1000087001207049087018E0B6F5B57F03DA44
:101E200002206D49087011E0B6F5C07F03DC032085
:101E3000694908700AE064480088864203DA042091
:101E40006549087002E0052063490870634890F90D
:101E50000000614991F90010884201D1002F7CD027
:101E6000B6F5B07F12DC4F48007838B104F1290193
:101E700088B25BA20321F7F771FA8CE004F1290123
:101E800088B25AA20321F7F769FA84E0B6F5B57F64
:101E900010DA04F1290188B257A20321F7F75EFA9C
:101EA00004F13E0082B204230C2105200095F7F7CF
:101EB00064F870E0B6F5C07F19DC04F1290188B23E
:101EC0004DA20321F7F74AFA04F1390082B2042344
:101ED0000C2105200095F7F750F804F13E0082B27E
:101EE00004230C2105200095F7F747F853E0364806
:101EF0000088864222DA04F1290188B23EA2032139
:101F0000F7F72CFA04F1340082B204230C210520E7
:101F10000095F7F732F804F1390082B204230C215E
:101F200005200095F7F729F804F13E0082B204235A
:101F30000C2105200095F7F720F82CE004F1290189
:101F400088B22DA20321F7F709FA04F12F0082B21B
:101F500004230C210520009500E021E0F7F70DF89F
:101F600004F1340082B204230C2105200095F7F718
:101F700004F804F1390082B204230C2105200095F5
:101F8000F6F7FBFF04F13E0082B204230C2105208A
:101F90000095F6F7F2FF104890F900000F4908701D
:101FA00000BF05E74C030020000801404D0300205E
:101FB000CC0000204348415247454241542E626DB7
:101FC00070000000001001404C0400207D920108C8
:101FD00044040020480400204A0400204904002052
:101FE00056424154332E626D7000000056424154F7
:101FF000322E626D7000000056424154312E626DE7
:10200000700000002DE9F0411E25222664274FF0C4
:102010003B0880200E49086141000E48F5F723FC7B
:10202000F6F702FE0CA200210846F7F797F9002404
:1020300008E0642094FBF0F100FB114008B9F7F7C9
:1020400049FB641C41F288308442F2DBBDE8F08138
:1020500000100140000C014077656C636F6D652EC8
:10206000626D700030B58BB004460D462B48007889
:1020700098B12A48007814280FD0284800782828DA
:102080000BD0264800783C2807D0244800785028F8
:1020900003D022480078642834D1242220492148E2
:1020A000F3F778FD50B928221D491E48F3F772FD59
:1020B00020B91B487C3890F82C0388B104F11E012C
:1020C00088B212237C222946F6F7FAFD2822144909
:1020D0001448F3F7F3FC002011497C3981F82C03F4
:1020E0002422104902A801F099F8FF200E4909782E
:1020F000CDE9001004F11E0188B21123084A2946D7
:10210000F7F7E8F905480078401CC0B203490870A9
:10211000642801DD002008700BB030BD5903002099
:102120007832002090310020B40400202DE9F041E5
:1021300004460D462046F6F719FB0646C6F1A007F1
:1021400007EBD771C1F34F00012322462946F7F769
:1021500079F9BDE8F0812DE9F04705460C461646B1
:102160001F462846F6F702FB8046311BA1EB080903
:1021700009EBD97104EB610188B201232A46394683
:10218000F7F760F9BDE8F08710B504461223322254
:1021900021462D20F6F766FE1B48007800F001006E
:1021A00030B91223432221462D20F6F75BFE2AE0A8
:1021B00015480078C0F3400080B913480078C0F398
:1021C000001028B911A221462D20F7F7C7F81AE010
:1021D00011A221462D20F7F7C1F814E00A48007833
:1021E000C0F3001028B909A221462D20F7F7B6F850
:1021F00004E009A221462D20F7F7B0F809A2A11C9E
:102200003520F7F7ABF810BD4C350020475053315F
:102210002E626D7000000000475053412E626D70B9
:1022200000000000475053322E626D700000000025
:10223000F0B593B005460C4616468EA103C9CDE90C
:1022400008018EA30FCB04AF0FC790A000680390C6
:1022500000278F4890F82F0301280BD18D4903A840
:10226000F3F781FC08B9002E37D08A480399016042
:10227000012732E0864890F82B0300281FDD86A155
:102280008648F3F770FC68B9824908A8F3F76BFC3D
:1022900000B916B37F48089901609DF824100171B8
:1022A00001271AE07B4904A8F3F75DFC00B9A6B149
:1022B0000E2204A97748F3F701FC01270DE07549C8
:1022C00073484230F3F74FFC00B936B1242270490D
:1022D00042317048F3F7F2FB012771496C48153021
:1022E000F3F741FC00B936B12422694915316C4835
:1022F000F3F7E4FB0127002F7DD004F1130083B234
:10230000A02221462846F6F763FD04F1130083B2AC
:10231000401E81B2A0222846F6F75AFD5C4890F88C
:102320002B0358B95A4890F82F0338B9221D91B29F
:102330006A1D90B25BA2F7F711F813E0544890F8C9
:102340002F03012807D1221D91B26A1D90B258A215
:10235000F7F704F806E0221D91B26A1D90B256A26A
:10236000F6F7FCFF04F1160291B26A1D90B255A275
:10237000F6F7F4FF242247490AA800F04FFF54A1C2
:102380004648F3F7F0FB68B9414890F82F0301285D
:1023900008D1221D91B205F11E0290B211230AAAA2
:1023A000F7F750F83A4890F82B0348B9221D91B23C
:1023B00005F11E0290B211230AAAF7F743F811E0C3
:1023C00024210AA8F3F793FB31497C310AA8F3F7DB
:1023D000D8FB221D91B205F11E0290B211230AAA68
:1023E000F7F730F801220AA9002000F099FE242214
:1023F0002B490AA800E03AE000F010FF04F11602B1
:1024000091B205F11E0290B211230AAAF7F71AF849
:102410001F4890F82B0302281CD11FA11F48F3F777
:10242000A2FB58B92B480078FF2111232AA2CDE93D
:1024300000106F217F20F7F74DF818E0254800784D
:10244000FF21112326A2CDE900106F216920F7F7A3
:1024500041F80CE00E4890F82B0340B91D48007875
:1024600012233C226F2100906420F6F76FFC0027B6
:1024700013B0F0BDB5A5BAF400000000536570615B
:10248000726174652043616C6C000000534F53000F
:10249000FC3100206C310020636E00009826002083
:1024A0004831002047726F7570322E626D700000E7
:1024B000534F532E626D70004F6E6563616C6C2ECE
:1024C000626D700070656F706C65322E626D7000A9
:1024D000656E0000B6040020B9D2B6CF000000003F
:1024E00048616E6755700000F0B593B00546402412
:1024F00004F11403A4F1140081B29F220020F6F726
:1025000067FC012004F112030090A4F1120081B2D3
:102510009D220220F6F705FD1222294601A800F0AF
:102520007DFE01A8F6F722F986B2C6F1A00000EB05
:10253000D071C1F34F07A4F1080081B2012301AAB1
:102540003846F6F77FFF13B0F0BD000038B50446FB
:102550003DA202210020F6F701FF012C01DB632CD4
:1025600006D10E23152204210720F6F77BFC6AE032
:10257000082C0EDA0120022307220E2100900C20E5
:10258000F6F7FBFC0E23152204210B20F6F76AFC5C
:1025900059E0102C16DA0120022307220E210090A8
:1025A0000C20F6F7EAFC012002230B220E210090FA
:1025B0000920F6F7E2FC0E23152204210F20F6F77E
:1025C00051FC40E0162C1EDA0120022307220E21C6
:1025D00000900C20F6F7D1FC012002230B220E21E3
:1025E00000900920F6F7C9FC012002230F220E21DA
:1025F00000900720F6F7C1FC0E23152204211320BA
:10260000F6F730FC1FE00120022307220E21009084
:102610000C20F6F7B2FC012002230B220E210090C1
:102620000920F6F7AAFC012002230F220E210090B8
:102630000720F6F7A2FC0120022313220E210090AE
:102640000420F6F79AFC38BD53696E676C654F4BF2
:102650002E626D700000000070B50446002C39D069
:102660001223A02200210846F6F7FCFB72480068FE
:102670007249086070480068FFF768FF704800689A
:10268000704908600020FFF77FFDE1B26C480068E8
:10269000FFF76CFB012000F001F96B4800686B4903
:1026A00008600846006800F027F96948007830B9EA
:1026B00010237E2203216E20F6F7D4FB04E065A2EE
:1026C00003216E20F6F74AFE6148007840B2634964
:1026D000087070BD5D4800685B490968884207D092
:1026E00059480068594908600846006800F004F934
:1026F0005248006850490968884205D158484078D6
:102700005849097888420BD0554840785549087097
:10271000494800684949086047480068FFF716FFC4
:1027200051480078C0F340004F49097801F0010199
:1027300040EA01204C490978C1F3001140EA8105C3
:102740004A480088A84204D0484805800020FFF786
:102750001BFD002000F0A2F845480078012804D1B4
:1027600044A26E214820F6F7F9FD394800783B492C
:1027700091F90010884213D03548007830B9102301
:102780007E2203216E20F6F76DFB04E031A20321C7
:102790006E20F6F7E3FD2E48007840B22F4908700E
:1027A0004FF400513648F5F755F8364991F90010C5
:1027B00088421DD00520344908704FF48070334999
:1027C00008606420DFF8C8C000DF4FF480702F4934
:1027D000091F08600020F7F7DDFD4FF4005128487D
:1027E000F5F738F840B227490870012029490870E8
:1027F00029488078E8B928488079D0B9114800681C
:102800000F490968884207D10D480068B0F5B07FCC
:1028100002DD2048007860B1094800680949086075
:102820001C48017806480068FFF7A0FA0020194903
:10283000087000BF4DE70000480000205804002049
:10284000B40000205C040020180100206404002073
:10285000300000204561722E626D70006804002017
:1028600040000020620400204C350020600400205D
:10287000C30000206C6F636B2E626D70000000005F
:10288000001001404C0300204D03002014080140BB
:10289000198C010869040020FC31002030B58DB08E
:1028A00004460BA8FBF7D0FF9DF831500E48006896
:1028B000A84200D1ACB10C4805609DF831000090F1
:1028C0009DF8303009A21E2103A805F061F900200F
:1028D000FF21012303AACDE9001005214320F6F7CB
:1028E000F9FD0DB030BD00005004002025303264E9
:1028F0003A253032640000001CB504460CB1022CAD
:102900000AD10020FF2101230DA2CDE900100421EE
:102910001C20F6F7DFFD12E0042C0AD10020FF2175
:10292000012308A2CDE9001004211C20F6F7D2FDF6
:1029300005E012232D2204211C20F6F793FA1CBD7A
:1029400032470000344700002DE9F04F89B080463F
:1029500089464FF0000AD346B8F1000F03D000209B
:102960007149A1F8680071A0F9F7E2FE002201A9FF
:10297000104600F0D5FB4FF47A7600206A4981F8C2
:102980007300888112E0701E86B20120FAF770FA97
:10299000654890F8730000B10AE0C82096FBF0F19A
:1029A00000FB116010B961A0F9F7C2FE002EEAD158
:1029B00000BF5D488089002804DC00205A4981F866
:1029C0006F00AFE058488089052190FBF1F201FBD0
:1029D000120008B98A4608E053488089052190FB17
:1029E000F1F201FB120000F0FF0A4F48B0F9682035
:1029F0002346514651A005F0BBF8B9F1010F0FD1A4
:102A00004948B0F8680085B247488089401B0528CE
:102A100001DB05242FE04448007B401BC4B22AE0C0
:102A20004148B0F8680085B23F48B0F96800052811
:102A300003DA00253C48047B1DE03B488089401BAD
:102A4000504517DC38488089052190FBF1F201FBE5
:102A5000120030B9012248A1002000F061FB0524DA
:102A600009E031488089052190FBF1F201FB120059
:102A7000C4B200E00524052C00DB052400202A490F
:102A800081F86F000846B0F968202346294642A025
:102A900005F06EF82F463AE000BF0020224981F889
:102AA0006E003B4648A21E2101A805F071F801A85E
:102AB000F9F73EFE002201A9104600F031FB322654
:102AC00021E00120FAF7D4F9174890F86E0038B1E8
:102AD000154890F86F00401C134981F86F0013E00F
:102AE000701E80B2061E0DD10BF10100C0B28346EC
:102AF0000A2806DDB346022001F0A2FC09B0BDE8B9
:102B0000F08FCAE700BFDCE700BF781C87B2281946
:102B1000B842C1DCB8F1000F03D000200249A1F88F
:102B2000680000BF00BFE9E7FC31002041542B5092
:102B30004F433D3533320D0A000000002A2A2A2A6D
:102B40002A2A2A2A2A666C61673D3D25642A2A2A98
:102B50002A2A2A2A2A68616E646C65496E6465783F
:102B60003D3D3D3D25642C726561644E756D3D3D76
:102B700025640D0A00000000474F20555055505560
:102B8000502D2D2D2D2D2D2D2D2D2D2D2D2D2D2D52
:102B90002D2D2D2D0D0A0000746869733D3D3D3DBE
:102BA0003D25643D3D3D68616E646C65496E6465BC
:102BB000783D3D3D3D25642C726561644E756D3DEB
:102BC0003D25640D0A00000041542B504F433D3514
:102BD000333426256426310D0A0000002DE9F04724
:102BE00088B0804689464FF0000AB8F1000F03D044
:102BF00000206749A1F8680066A0F9F799FD4FF435
:102C00007A760020624981F87200488112E0701ED5
:102C100086B20120FAF72CF95D4890F8720000B1F5
:102C20000AE0C82096FBF0F100FB116010B959A032
:102C3000F9F77EFD002EEAD100BF554840890028F3
:102C400004DC0020524981F86D009EE05048408924
:102C5000052190FBF1F201FB120018B90520514942
:102C6000087008E04A484089052190FBF1F201FB19
:102C700012004C490870B9F1010F0FD14448B0F867
:102C8000680085B242484089401B052801DB0524C5
:102C90002CE03F48807A401BC4B227E03C48B0F8A3
:102CA000680085B23A48B0F96800052803DA0025C3
:102CB0003748847A1AE036484089401B39490978F8
:102CC000884212DC32484089052190FBF1F201FB79
:102CD000120008B9052409E02D484089052190FB20
:102CE000F1F201FB1200C4B200E00524052C00DB68
:102CF00005240020264981F86D002F463AE000BFE8
:102D00000020234981F86C003B4627A21E2168461B
:102D100004F03EFF6846F9F70BFD002269461046B5
:102D200000F0FEF9322621E00120FAF7A1F8184858
:102D300090F86C0038B1164890F86D00401C1449AA
:102D400081F86D0013E0701E80B2061E0DD10AF1ED
:102D50000100C0B282460A2806DDB246022001F018
:102D60006FFB08B0BDE8F087CAE700BFDCE700BF33
:102D7000781C87B22819B842C1DCB8F1000F03D023
:102D800000200349A1F8680000BF00BFE9E7000088
:102D9000FC31002041542B504F433D3533350D0A53
:102DA00000000000AA04002041542B504F433D3541
:102DB000333726256426310D0A0000002DE9F0473F
:102DC0008AB007468A464FF000091FB100208349A8
:102DD000A1F86A0000208149C8810120DFF800C203
:102DE00000DF00BF00207D4981F8740008467DA205
:102DF0001E21D0F8383302A804F0CAFE774890F8B4
:102E000074107CA004F0B4FE02A8F9F791FC002233
:102E100002A9104600F084F94FF01E0812E00120CC
:102E2000FAF726F86D4890F8740000B10BE0A8F1AD
:102E3000010080B2B0F1000803D175A004F098FE43
:102E4000D0E700BFEBE700BF644890F8741075A0AE
:102E500004F08EFE0020614981F874000846C089A4
:102E6000002805DC002081F8710074A004F080FEC9
:102E70005A48B0F96A005949C989884213DB574852
:102E8000B0F96A3072A21E2102A804F081FE01226C
:102E900002A9002000F044F95048C089401E00B249
:102EA0004E49A1F86A004D48C1896BA004F060FE4C
:102EB0004A48C089052807DC00254848847B21460C
:102EC00069A004F055FE2FE09FB100254348C0895A
:102ED000052190FBF1F201FB120008B9052423E063
:102EE0003E48C089052190FBF1F201FB1200C4B2FB
:102EF0001AE03A48B0F96A00042813DD3748C0895F
:102F0000052190FBF1F201FB120008B9052507E04D
:102F10003248C089052190FBF1F201FB120085B215
:102F2000052401E000250524052C00DB05240020F4
:102F30002A4981F871000120DFF8A4C000DF2E4685
:102F400047E000BF224629464BA004F011FE23486B
:102F5000009650A21E21D0F8383302A804F018FEC3
:102F600002A8F9F7E5FB002202A9104600F0D8F804
:102F70004FF0050829E00320F9F77AFF174890F889
:102F8000700050B1154890F87100401C134981F849
:102F90007100002081F8700018E0A8F1010080B2F3
:102FA000B0F1000810D11AA004F0E2FD09F101000F
:102FB000C0B281460A2806DDC146022001F040FA6F
:102FC0000AB0BDE8F087BDE700BFD4E700BF701CC2
:102FD00086B22819B042B4DC00BFF1E7FC31002012
:102FE000198C010841542B504F433D35353026256F
:102FF000640D0A002A2A2A566F6963654E756D5F53
:103000005570646174653D3D3D25640D0A00000006
:10301000B3ACCAB1C1CB3D3D3D3D3D3D3D3D3D3DE8
:103020003D0D0A00566F6963654E756D5F5570649E
:103030006174653D3D3D25640D0A0000474F544FC6
:103040002D2D2D2D2D2D2D2D2D2D2D2D0000000064
:103050006F7665723A25640073746570303D3D3D4E
:103060003D3D3D25640D0A007374657031203D3D82
:103070003D3D25640D0A0000746869733D3D3D25A2
:103080006420726561646E756D3D3D3D25640D0A79
:103090000000000041542B504F433D35353126256B
:1030A0006426256426310D0A0000000010B50122B7
:1030B00015A1002000F034F84FF480701549086025
:1030C00000F046F880201449486102201149091F88
:1030D000086000021049486101204861000348610E
:1030E00004200E4908600C494861C1020A48F4F7FF
:1030F000B1FB012802D1102007494861012108468F
:10310000F9F7F0FE10BD0000536C656570696E67DD
:1031100000000000140C0140001001401014014098
:103120002DE9F04106460C4617462046F2F714FDFD
:1031300005462946204603F06BFBBDE8F08100B54B
:10314000024612B100F00CF801E000F001F800BDF9
:103150004FF4807001490861704700000010014081
:103160004FF4807001490861704700000010014071
:1031700008B54FF48070ADF8000010208DF8030002
:1031800003208DF8020069460348F4F78FFA002007
:10319000FFF7D5FF08BD00000010014010B51B4827
:1031A000007800B910BD1948007900B9FAE700208D
:1031B0001649087108464079122806D025280AD0F9
:1031C00047280ED058281ED114E01048807908B93D
:1031D000F6F72AFB17E000220D491046FFF7A0FF83
:1031E00011E000220B491046FFF79AFF0220F6F784
:1031F000C1F908E0002208491046FFF791FF0320BB
:10320000F6F7B8F900BF00BF00BFCBE7C00E002043
:103210005C9701082D990108799701082DE9F0477D
:103220000646884614464046F2F796FC8146002141
:10323000601E3154621E41463046F2F781FC601E2A
:1032400048451CDC052C1ADD2E21A01E3154E01E41
:1032500031543546002707E028789F2802DDAD1C51
:10326000BF1C01E06D1C7F1C201FB842F4DCB8427B
:1032700005D128789F2802DD2E21201F3154BDE87A
:10328000F08703467047F0B503460024002500266A
:10329000002715E01878262804D1601C04B28C425F
:1032A00000DD13E08C4208D126B9681C05B22F4618
:1032B00001265B1C187802F8010B5B1C681C05B228
:1032C00018780D2802D018780A28E3D100BF002012
:1032D00002F8010B8C4200DAF0BDF8B2FCE7000006
:1032E00030B5B3B050212148F2F701FC20A0F4F72B
:1032F000B1FC0546681C20B91FA004F039FC33B0AE
:1033000030BD2846F4F7C2FC0446002C03DC20A0A4
:1033100004F02EFCF3E7C82C05D9C822214623A0CF
:1033200004F026FCEBE701AB224600212846FBF720
:10333000F5FB04460D4A24A101A8F5F745F904461A
:1033400034B925A004F014FC002008490870D6E721
:1033500028A10648F9F703FA10B9002003490870BC
:10336000024926A004F004FC00BFC8E7081B0020A7
:103370007379732E696E69007379732E696E692093
:10338000206E6F7420666F756E640D0A0000000079
:103390007379732E696E69206E6F20646174612089
:1033A0006F72206572720D0A000000007379732E2F
:1033B000696E69206C656E3D25642C73686F756C51
:1033C000643C3D25640D0A0048505F564F49434513
:1033D0005F545453000000006E6F207365676D6585
:1033E0006E742048505F564F4943455F5454530D07
:1033F0000A0000004E554C4C000000007379732EFB
:10340000696E69206F6B0D0A25730D0A00000000BC
:1034100010B51248006840F00100104908600846E5
:1034200040680F4908400D494860084600680D494A
:1034300008400A4908600846006820F480200860B7
:103440000846406820F4FE0048604FF41F00886082
:10345000FEF746F904480549086010BD0010024017
:103460000000FFF8FFFFF6FE0058000808ED00E03E
:1034700021B1028842F00102028004E002884FF686
:10348000FE731A400280704731B1B0F8442042F414
:103490000042A0F8442005E0B0F84420C2F30E0238
:1034A000A0F844207047000070B5002400220023DB
:1034B000058C4FF6FE7635400584028C8388048B9C
:1034C0004FF68F752C40B51E2C400D882C43751E71
:1034D0002A400D892A434D882A43144DA8420BD017
:1034E000134DA84208D0134DA84205D0124DA84252
:1034F00002D0124DA84213D14FF6F7752A404D89DC
:103500002A434FF6FB752A408D882A434FF6FF6504
:103510002B404FF6FF552B408D892B43CD892B43F4
:1035200083800483CD888586028470BD002C014091
:103530000034014000400140004401400048014087
:103540000A460021018B4FF6F7731940114301839E
:103550007047000070B5002400220023058C4FF650
:10356000EF7635400584028C8388048B48F6FF751E
:103570002C404FF6FF452C400D884FF6FF7606EAAB
:1035800005252C434FF6DF752A400D8906EA0515FF
:103590002A434D8806EA05152A43154DA84202D054
:1035A000144DA8421DD14FF67F752A404D894FF624
:1035B000FF7606EA05152A434FF6BF752A408D8827
:1035C00006EA05152A434FF6FF352B404FF2FF75EB
:1035D0002B408D8906EA85052B43CD8906EA8505B2
:1035E0002B4383800483CD880587028470BD00004F
:1035F000002C014000340140002202881D4B9842FB
:103600000ED01D4B98420BD0B0F1804F08D01B4B11
:10361000984205D01A4B984202D01A4B984204D1D6
:103620004FF68F731A404B881A43174B984207D0B6
:10363000164B984204D04FF6FF431A40CB881A43EA
:1036400002808B8883850B8803850A4B98420BD0B8
:10365000094B984208D00E4B984205D00D4B98422A
:1036600002D00D4B984201D10B7A0386012383824D
:1036700070470000002C014000340140000400406D
:1036800000080040000C0040001000400014004002
:1036900000400140004401400048014010B5084C82
:1036A0001C212046F2F723FA064C7C212046F2F733
:1036B0001EFA2046007820F010002146087010BD48
:1036C000C83500204C35002030B59FB00120F4F7FC
:1036D00039F9214890F87100572805D11E49886EA4
:1036E00006F016F8044601E01B48846E1A4890F86C
:1036F0007000532805D11849C86E06F009F8054630
:1037000001E01548C56E1448407D1349496A124AC4
:10371000926A114BDB8ACDE90045CDE90232CDE951
:1037200004100D480DA26421436F06A804F030FA7E
:10373000012213490020FFF7F3FC06A8F8F7F8FF71
:10374000012206A90020FFF7EBFC01220D49002011
:10375000FFF7E6FC1FB030BD4C35002041542B5024
:103760004F433D35323526253964262564262564A8
:103770002625642625642625642625640D0A000076
:103780008CB5010840B5010800B58DB0724840887D
:10379000401C80B270494880B0F5FA7F76DD002089
:1037A000488008464079472848D004DC122807D0D2
:1037B00025281FD11FE058285CD0C228F9D166E027
:1037C0006548807998B96448407A401C62494872DB
:1037D0000846407A032803DA1220F9F725FB09E0AE
:1037E00001205D49C872C220F9F71EFB02E01220D9
:1037F000F9F71AFB80E05848807918B91220F9F7D8
:1038000013FB1AE05448807A401C534988720846DA
:10381000807A14280BDA012250A10020FFF780FCE7
:103820004D4948694FF48061F5F7D8FF05E0022063
:103830004949C872C220F9F7F7FA5DE00022022177
:1038400045481830F5F760FF10B1012810D103E0AA
:103850005820F9F7E9FA0BE004203F49C87200222A
:1038600041491046FFF75CFCC220F9F7DDFA00BFC2
:1038700000BF41E03D48FDF7E3FB00223C49104614
:10388000FFF74EFC05F006FC00BFFEE735E0012324
:10389000384A28210420F5F7D5FD2F48C07A0128A1
:1038A00006D002280BD0032810D004281CD114E025
:1038B0000123314A46210420F5F7C4FD14E0012319
:1038C0002E4A46210420F5F7BDFD0DE001232C4AC8
:1038D00046210420F5F7B6FD06E00123294A4621DA
:1038E0000420F5F7AFFD00BF00BFC820DFF898C087
:1038F00000DFF3F781FA00BF00BF24480078401CC6
:1039000022490870084601780078401C1F4A107050
:10391000FE291EDB0020114608701D480078401C5F
:103920001B49087008460078032809DA032319A206
:103930003221684604F02CF96846F8F7F9FE08E0F1
:103940000020134908700448007810B90120F3F7EB
:1039500037FE0DB000BD0000C00E00205265712082
:1039600044617461000000008A970108A9CBED9FB3
:10397000E4970108F79901080C9A0108219A0108B7
:10398000369A01084B9A0108198C0108250000207D
:103990002600002041542B54435053544154555356
:1039A0003D25640D0A000000F0B505460C46286868
:1039B0006968AA68EB6801EA020623EA01073E4348
:1039C00027683E44FE4F3E443044C60146EA5060FC
:1039D000084400EA010622EA00073E4367683E44C5
:1039E000F84F3E4433441E0346EA1353034403EAAC
:1039F000000621EA03073E43A7683E44F24F3E44D7
:103A00003244560446EAD2321A4402EA030620EA55
:103A100002073E43E7683E44EC4F3E4431448E0586
:103A200046EA9121114401EA020623EA01073E43D6
:103A300027693E44E64F3E443044C60146EA5060A2
:103A4000084400EA010622EA00073E4367693E4453
:103A5000E04F3E4433441E0346EA1353034403EA53
:103A6000000621EA03073E43A7693E44DA4F3E447D
:103A70003244560446EAD2321A4402EA030620EAE5
:103A800002073E43E7693E44D44F3E4431448E052D
:103A900046EA9121114401EA020623EA01073E4366
:103AA000276A3E44CE4F3E443044C60146EA506049
:103AB000084400EA010622EA00073E43676A3E44E2
:103AC000C84F3E4433441E0346EA1353034403EAFB
:103AD000000621EA03073E43A76A3E44A6F52446B2
:103AE0004F3E3244560446EAD2321A4402EA0306F2
:103AF00020EA02073E43E76A3E44BB4F3E4431445E
:103B00008E0546EA9121114401EA020623EA0107E3
:103B10003E43276B3E44B54F3E443044C60146EA1F
:103B20005060084400EA010622EA00073E43676B42
:103B30003E44AF4F3E4433441E0346EA135303440E
:103B400003EA000621EA03073E43A76B3E44A94F60
:103B50003E443244560446EAD2321A4402EA03068C
:103B600020EA02073E43E76B3E44A34F3E44314404
:103B70008E0546EA9121114401EA030622EA030771
:103B80003E4367683E449D4F3E443044460146EA0A
:103B9000D060084400EA020621EA02073E43A76912
:103BA0003E44974F3E4433445E0246EAD3530344B7
:103BB00003EA010620EA01073E43E76A3E44914FCB
:103BC0003E443244960346EA92421A4402EA000610
:103BD00023EA00073E4327683E448B4F3E4431446E
:103BE0000E0546EA1131114401EA030622EA0307F1
:103BF0003E4367693E44854F3E443044460146EAB1
:103C0000D060084400EA020621EA02073E43A76AA0
:103C10003E447F4F3E4433445E0246EAD35303445E
:103C200003EA010620EA01073E43E76B3E44794F71
:103C30003E443244960346EA92421A4402EA00069F
:103C400023EA00073E4327693E44734F3E44314414
:103C50000E0546EA1131114401EA030622EA030780
:103C60003E43676A3E446D4F3E443044460146EA57
:103C7000D060084400EA020621EA02073E43A76B2F
:103C80003E44674F3E4433445E0246EAD353034406
:103C900003EA010620EA01073E43E7683E44614F1C
:103CA0003E443244960346EA92421A4402EA00062F
:103CB00023EA00073E43276A3E445B4F3E443144BB
:103CC0000E0546EA1131114401EA030622EA030710
:103CD0003E43676B3E44554F3E443044460146EAFE
:103CE000D060084400EA020621EA02073E43A768C2
:103CF0003E444F4F3E4433445E0246EAD3530344AE
:103D000003EA010620EA01073E43E7693E44494FC2
:103D10003E443244960346EA92421A4402EA0006BE
:103D200023EA00073E43276B3E44434F3E44314461
:103D30000E0546EA1131114481EA02065E406769C8
:103D40003E443E4F3E443044060146EA107008446B
:103D500080EA01065640276A3E44394F3E443344C8
:103D6000DE0246EA5353034483EA00064E40E76A04
:103D70003E44344F3E443244160446EA12421A444A
:103D800082EA03064640A76B3E442F4F3E4431442F
:103D9000CE0546EA5121114481EA02065E40676879
:103DA0003E442A4F3E443044060146EA107008441F
:103DB00080EA0106564027693E44254F3E4449E0CB
:103DC00078A46AD756B7C7E8DB702024EECEBDC111
:103DD000AF0F7CF52AC68747134630A8019546FDEC
:103DE000D8988069AFF7448BBED75C892211906B5D
:103DF000937198FD8E4379A62108B44962251EF679
:103E000040B340C0515A5E26AAC7B6E95D102FD60E
:103E10005314440281E6A1D8C8FBD3E7E6CDE121E3
:103E2000D60737C3870DD5F4ED145A4505E9E3A944
:103E3000F8A3EFFCD9026F678A4C2A8D4239FAFF4A
:103E400081F6718722619D6D0C38E5FD44EABEA4C0
:103E5000A9CFDE4B3344DE0246EA5353034483EAE0
:103E600000064E40E7693E449F4F3E4432441604EC
:103E700046EA12421A4482EA03064640A76A3E44D2
:103E80009A4F3E443144CE0546EA5121114481EA1D
:103E900002065E40676B3E44954F3E443044060147
:103EA00046EA1070084480EA0106564027683E44FE
:103EB000904F3E443344DE0246EA5353034483EAC0
:103EC00000064E40E7683E448B4F3E4432441604A1
:103ED00046EA12421A4482EA03064640A7693E4473
:103EE000864F3E443144CE0546EA5121114481EAD1
:103EF00002065E40676A3E44814F3E4430440601FC
:103F000046EA1070084480EA01065640276B3E449A
:103F10007C4F3E443344DE0246EA5353034483EA73
:103F200000064E40E76B3E44774F3E443244160451
:103F300046EA12421A4482EA03064640A7683E4413
:103F4000724F3E443144CE0546EA5121114461EAA4
:103F50000306564027683E446D4F3E443044860178
:103F600046EA9060084460EA02064E40E7693E4433
:103F7000684F3E4433449E0246EA9353034463EA47
:103F800001064640A76B3E44634F3E443244D6038D
:103F900046EA52421A4462EA00065E4067693E44BD
:103FA0005E4F3E4431444E0546EAD121114461EA58
:103FB00003065640276B3E44594F3E443044860129
:103FC00046EA9060084460EA02064E40E7683E44D4
:103FD000544F3E4433449E0246EA9353034463EAFB
:103FE00001064640A76A3E444F4F3E443244D60342
:103FF00046EA52421A4462EA00065E4067683E445E
:104000004A4F3E4431444E0546EAD121114461EA0B
:1040100003065640276A3E44454F3E4430448601DD
:1040200046EA9060084460EA02064E40E76B3E4470
:10403000404F3E4433449E0246EA9353034463EAAE
:1040400001064640A7693E443B4F3E443244D603F6
:1040500046EA52421A4462EA00065E40676B3E44FA
:10406000364F3E4431444E0546EAD121114461EABF
:104070000306564027693E44314F3E443044860192
:1040800046EA9060084460EA02064E40E76A3E4411
:104090002C4F3E4433449E0246EA9353034463EA62
:1040A00001064640A7683E44274F3E443244D603AB
:1040B00046EA52421A4462EA00065E40676A3E449B
:1040C000224F3E4431444E0546EAD12111442E6828
:1040D00006442E606E680E446E60AE681644AE6094
:1040E000EE681E44EE60F0BD604BBBF670BCBFBE18
:1040F000C67E9B28FA27A1EA8530EFD4051D8804E7
:1041000039D0D4D9E599DBE6F87CA21F6556ACC45A
:10411000442229F497FF2A43A72394AB39A093FCA8
:10412000C3595B6592CC0C8F7DF4EFFFD15D848524
:104130004F7EA86FE0E62CFE144301A3A111084EA8
:10414000827E53F735F23ABDBBD2D72A91D386EBA4
:1041500038B5002440F225513A4802F0B6F900285B
:1041600057D0384802F06CFAC0B200903648007858
:10417000022805D19DF80010344802F066FA3FE0AD
:1041800031480078012805D19DF80010304802F030
:104190005CFA35E02F48008828B100202E490880BD
:1041A0002E49087038BD9DF800102B480288008801
:1041B000401C294B188029488154294800780D2833
:1041C0001ED19DF800000A281AD1244800783E2804
:1041D00007D022480078412803D02048007847289B
:1041E00009D11D4800881B49088000201B491A4A34
:1041F0001288885404E00020174908801749087085
:1042000015480088C72804DB00201349088011499D
:1042100008809DF800001249087040F225510948B5
:1042200002F02BF90821074802F042F9012806D1D3
:10423000044802F005FA0821024802F015F900BF0F
:10424000B0E7000000380140760100200044004043
:10425000004800407A010020780100200E2700204D
:104260008D01002008B540F22551274802F02DF9B4
:1042700000283AD0244802F0E3F9C0B20090234865
:10428000007802280AD19DF80010214802F0DDF9DB
:1042900040F225511C4802F0F0F808BD1D48008886
:1042A000B0F5A06F1CDA9DF800001B491B4A12886C
:1042B00088541A480088401C80B218490880B0F51C
:1042C000A06F01DB0020088012480088401C1149C3
:1042D00008809DF800000A2802D1114804F050F827
:1042E00040F22551084802F0C8F80821064802F0BB
:1042F000DFF8012806D1044802F0A2F9082102489B
:1043000002F0B2F800BFC8E7004400407601002088
:104310000038014086010020022900208801002089
:104320005801002038B5002440F225513D4802F0E4
:10433000CCF8002868D03B4802F082F9C0B2009067
:1043400039480078012805D19DF80010374802F05F
:104350007CF950E036480088002849D19DF80000DB
:104360003449354A1288885408460078242803D0F6
:1043700000203149088004E02F480088401C2E4965
:1043800008802D480088B0F5957F02DD00202A497D
:1043900008802A4800780D282DD19DF800000A28B1
:1043A00029D124484078472807D12248C07852288C
:1043B00003D12048407943280BD01E484078472835
:1043C00012D11C48007947280ED11A48407941285B
:1043D0000AD1002118480088401E164A1154164878
:1043E00000881349088006E000201349088002E095
:1043F00000201149088040F225510A4802F03DF89A
:104400009DF800000D4908700821064802F050F898
:10441000012806D1034802F013F90821014802F0EF
:1044200023F838BD004800407601002000380140E4
:1044300080010020D62700207E0100208F0100206F
:1044400006490978814200D1704704498978034AB6
:1044500051701146887000BFF6E70000410300204C
:1044600070B5044600250A4D84B1F4F7DDFB032145
:1044700008A0FDF75BFE012314229F210020F4F722
:1044800039FD29460648F7F7B5FC70BD00BFFCE7CB
:1044900094030020B9A4B3A7C4A3CABD00000000C0
:1044A0005003002070B50546002D76D0574800789F
:1044B000C8B957A15748F1F756FB18B956A0FEF7EF
:1044C00013F802E059A0FEF70FF8322402E00120B1
:1044D000F8F7CEFC201EA4F101018CB2F7D1012027
:1044E000FFF7AEFF70BD494890F82B03022819D1A1
:1044F00047A14848F1F737FB18B953A0FDF7F4FF7F
:1045000002E055A0FDF7F0FF322402E00120F8F7A9
:10451000AFFC201EA4F101018CB2F7D10120FFF7FE
:104520008FFFDFE701210846FEF70EFA00204E4913
:104530000880F4F779FB36A13648F1F714FB70B91F
:10454000324890F83403012804D1032147A0FDF735
:10455000EDFD12E0032148A0FDF7E8FD0DE02B483A
:1045600090F83403012804D1032146A0FDF7DEFDB5
:1045700003E0032146A0FDF7D9FD012314229F216A
:104580000020F4F7B7FCFAF7EDF9012368229F2128
:104590000020F4F7AFFCA5E7FFE73348008890B9A7
:1045A0001BA11C48F1F7DFFA30B901233CA26E21B0
:1045B0000020F4F747FF1CE001233FA26E210020FA
:1045C000F4F740FF15E028480088C82811D110A151
:1045D0001048F1F7C8FA30B901233CA26E2100203F
:1045E000F4F730FF05E001233EA26E210020F4F72E
:1045F00029FF1D480088401C80B21B490880B0F587
:10460000C87F01DB0020088000BF6BE7FC31002081
:10461000636E0000982600202020C7EBCFC8B5C7E6
:10462000C2BC2E2E2E20202000000000506C6561A0
:104630007365206C6F67696E2066697273742E2EC5
:104640002E20202000000000B5A5BAF4BDFBD6B98D
:10465000B2D9D7F7A3A1000043616E277420646F1D
:104660002074686174000000E4030020C8BAD7E930
:10467000D3EFD2F400000000C8BAD7E9D1A1D4F139
:104680000000000047726F757020566F6963650007
:1046900047726F75702053656C656374696F6E0047
:1046A0005BC9CF5DD1A1D4F12020202020205BCF99
:1046B000C25DD1A1D4F100005B55505D20202020C7
:1046C00020202020205B444F574E5D005B4D5DC88D
:1046D000B7B6A8202020205B455849545DCDCBB308
:1046E000F60000005B4D5D4F4B2020202020202055
:1046F000205B455849545D0070B594B00546C5B17E
:1047000000209E490870F4F78FFA9DA19D48F1F7AB
:104710002AFA20B903219CA0FDF708FD03E003213C
:104720009CA0FDF703FD012314229F210020F4F734
:10473000E1FB0226162445B9994800689949884248
:1047400076D18E4800780028FAD10020944908607C
:104750007F239F222146F4F73BFB89A18948F1F78B
:1047600002FA38B9874BDD3B8FA2322102A803F051
:104770000FFA06E0834BDD3B8EA2322102A803F044
:1047800007FA012302AA21463046F4F75BFE04F142
:10479000140084B27AA17B48F1F7E5F938B9794B76
:1047A0002F3388A2322102A803F0F2F906E0754BFC
:1047B0002F3384A2322102A803F0EAF9012302AACE
:1047C00021463046F4F73EFE04F1140084B26CA199
:1047D0006C48F1F7C8F958B9002000906948E038F2
:1047E000B0F8113079A2322102A803F0D1F90AE021
:1047F000002000906348E038B0F8113077A23221F1
:1048000002A803F0C5F9012302AA21463046F4F7B5
:1048100019FE04F1140084B259A15A48F1F7A3F922
:1048200038B9724B72A2322102A803F0B1F906E046
:104830005AE06E4B71A2322102A803F0A9F90123BC
:1048400002AA21463046F4F7FDFD04F1140084B2BB
:104850003222002102A8F1F743F96B48007880B9B1
:1048600047A14848F1F77FF928B968A2322102A888
:1048700003F08EF92EE069A2322102A803F088F934
:1048800028E061480078012810D13DA13D48F1F7AA
:104890006AF928B965A2322102A803F079F919E072
:1048A00066A2322102A803F073F913E0564800789B
:1048B00002280FD132A13348F1F755F928B962A285
:1048C000322102A803F064F904E063A2322102A8B5
:1048D00003F05EF9012302AA21463046F4F7B2FD47
:1048E00002202649087047E02D4800685D4988424B
:1048F00042D12248007802283ED100202849086091
:104900007F239F222146F4F763FA1DA11D48F1F78A
:104910002AF928B954A2322102A803F039F904E097
:1049200054A2322102A803F033F9012302AA21463E
:104930003046F4F787FD04F1140084B21422514983
:104940000FA8F1F7FDF801230FAA21463046F4F72E
:1049500079FD4C4B13331AA2322102A803F018F947
:1049600004F1140084B2012302AA21463046F4F770
:1049700069FD00200149087014B070BD4204002098
:10498000636E000098260020D6D5B6CBD0C5CFA246
:104990000000000044657669636520496E666F001B
:1049A0005C0000200A04BC00D6D5B6CBD0CDBAC579
:1049B0003A257300446576696365204E616D653AFA
:1049C0002573000049443A2573000000D3A6D3C3E1
:1049D000B0E6B1BE3A5625642E2564004D435520FD
:1049E0005665723A5625642E256400003C35002039
:1049F000B6D4BDB2B0E6B1BE3A257300504F4320E5
:104A00005665723A257300006B010020C4A3BFE90C
:104A1000C0E0D0CD3ACEB4D6AA0000004D6F647588
:104A20006C653A556E6B6E6F776E0000C4A3BFE97C
:104A3000C0E0D0CD3AC3C0B0E60000004D6F647551
:104A40006C653A5553000000C4A3BFE9C0E0D0CD67
:104A50003AC5B7B0E60000004D6F64756C653A4525
:104A6000550000000A04DC00B9CCBCFEB0E6B1BEC3
:104A70003A000000486172645265766973696F6E2E
:104A80003A000000E626002010B50446002C29D08C
:104A9000F4F7CAF8012314A219460020F4F7D2FC57
:104AA000012314229F210020F4F724FA11484088A2
:104AB000012807DB0F48418800230F4A0F48F6F70B
:104AC0009CF803E000210846F6F7C8F801230CA281
:104AD0006E210020F4F7B6FC012368229F210020FC
:104AE000F4F708FA10BD00002020CEC4B1BECFFB01
:104AF000CFA20000F81B0020300100200C2F002066
:104B00005B4D5DB2E9D4C4202020205B535DD1A170
:104B1000CFEE200030B587B00546002D34D0F4F735
:104B200097F84FF0FF30F94908600020F849086015
:104B30002846FDF791FDF7A1F748F1F714F860B9A1
:104B40001123F6A26F210020F4F77CFC1223A0228F
:104B50006E210020F4F706FB0BE01123F4A26F2175
:104B60000120F4F76FFC1223A0226E210020F4F73D
:104B7000F9FAF4480078012804D101221321002019
:104B8000FDF756FB07B030BDEF48007801281ED175
:104B9000E0A1E148F0F7E7FF18B9ECA0FDF7A4FCAD
:104BA00002E0EDA0FDF7A0FC3220DFF8BCC300DF7F
:104BB00054239F222C210020F4F70AF9E1480078C1
:104BC000012804D1012213210020FDF731FB2846E2
:104BD000FDF742FDDB48007808B9002418E0D94809
:104BE000807838B9D748807920B901240020DF497E
:104BF00008600DE0D348807828B9D2488079012830
:104C000001D1022404E0CF488078002800DD03248D
:104C100034B1012C1BD0022C47D0032C16D1A0E0BC
:104C2000BA480068844203D1C748007801280DD1F2
:104C30004E239F2213210020F4F7CAF8CCA213219F
:104C40001E20F4F78BFB0020BF490870A2E0AF489C
:104C50000068844203D1BC480078012824D14E2347
:104C60009F223C212420F4F7B3F8AAA1AA48F0F728
:104C70007AFF58B9C1A23C210520F4F76FFB11233C
:104C8000C1A23C211E20F4F7DDFB0AE0BBA23C21BF
:104C90000520F4F763FB1123BDA23C211E20F4F78D
:104CA000D1FB0020A849087074E09848006884424D
:104CB00003D1A5480078012852D14E239F223C21E0
:104CC0000020F4F785F893A19348F0F74CFF00BB60
:104CD000B1A23C210520F4F741FB9A4890F82F033C
:104CE00058B9FF20AF4909781123AFA2CDE90010D0
:104CF0003C211E20F4F7EEFB2BE0FF20A9490978A8
:104D00001123ACA2CDE900103C211E20F4F7E2FBF8
:104D10001FE0A1A23C210520F4F720FB894890F870
:104D20002F0358B9FF209F4909781123A5A2CDE987
:104D300000103C211E20F4F7CDFB0AE0FF2099492A
:104D400009781123A1A2CDE900103C211E20F4F71F
:104D5000C1FB01207B4981F82C0300207A490870AF
:104D600018E06A480068844203D177480078012837
:104D70000BD19AA23C210520F4F7F0FA01207149E9
:104D800081F82C030020704908703C210020FDF7B9
:104D900069F900BF00BF002C12DD5C480068844246
:104DA00008D05A48006828B9012213210020FDF7D5
:104DB0003FFA6CE1002213211046FDF739FA66E153
:104DC000604890F82E0389490978884204D14F48F9
:104DD0000068401C002848D15A4890F82E038349A7
:104DE000087008460078012805D181A2142102A884
:104DF00002F0CEFE33E07D480078022805D180A283
:104E0000142102A802F0C4FE29E0784800780428A2
:104E100010D140A14048F0F7A6FE28B97CA2142189
:104E200002A802F0B5FE1AE07DA2142102A802F049
:104E3000AFFE14E06D480078052805D17AA2142150
:104E400002A802F0A5FE0AE068480078062805D10D
:104E500078A2142102A802F09BFE00E018E11123C1
:104E600002AA26210020F4F7EDFA2AA12A48F0F739
:104E70007AFE88BB2022142102A8F0F731FE092215
:104E80006FA102A8F0F71AFE2148006830B911237B
:104E900002AA13210020F4F7D5FAF8E01C480068B4
:104EA000642809D12E208DF81100112302AA1321A4
:104EB0000020F4F7C7FAEAE015480068C8280AD1CC
:104EC0002E208DF811008DF81200112302AA132153
:104ED0000020F4F7B7FADAE0FFE72022142102A855
:104EE000F0F7FEFD59A0016802918188ADF80C1021
:104EF00080798DF80E000648006830B9112302AAA7
:104F000013210020F4F79EFAC1E0A3E05C03002027
:104F100060030020636E000098260020B2CBB5A588
:104F20002020202020202020202020200000000001
:104F30004D656E752020202020202020202020205C
:104F400000000000FC310020C4000020C7EBCFC8E7
:104F5000BDE2CBF8A3A10000506C656173652075BC
:104F60006E6C6F636B000000198C01084803002011
:104F70006C6F676F2E626D700000000050686F6E7E
:104F8000652E626D70000000BFD5CFD0000000001C
:104F900046726565000000004373656E642E626DA5
:104FA00070000000B3040020B1BEBBFAD4DABDB279
:104FB000BBB00000B0B4505454CDCBB3F6534F53F4
:104FC000000000004E6174697665000050726573E0
:104FD000732050545420457869740000437265630F
:104FE000656976652E626D70000000006403002024
:104FF000D5CBBAC5D0C5CFA2B4EDCEF3000000002A
:10500000CEDECDF8C2E7C1ACBDD320200000000049
:10501000C7EBB2E5BFA82020202020200000000020
:105020004E6F204361726400CEDEB7A8C1ACBDD321
:1050300000000000C3BBD3D0B7FECEF100000000DB
:10504000D5FDD4DAB5C7C2BD2E0000004C6F67692C
:105050006E672E0019480068642809D12E208DF84B
:105060000F00112302AA13210020F4F7EBF90EE040
:1050700012480068C8280AD12E208DF80F008DF83C
:105080001000112302AA13210020F4F7DBF900BF5E
:105090000A480068401C09490860B0F5967F01DBAA
:1050A0000020086006480068844204D00448046078
:1050B00000200249086000BF64E500006003002092
:1050C0005C03002070B50446002513A11348F0F7D7
:1050D0004AFD08B9124D00E0124DD4B1F3F7A4FD1A
:1050E0000DA10E48F0F73FFD20B903210EA0FDF7FA
:1050F0001DF803E003210EA0FDF718F80123142288
:105100009F210020F3F7F6FE29460B48F6F772FEC2
:1051100070BD00BFFCE70000636E00009826002011
:105120006803002080030020D6F7B2CBB5A50000AD
:105130004D656E75000000005003002070B50446F8
:10514000002513A11348F0F70EFD08B9124D00E039
:10515000124DD4B1F3F768FD0DA10E48F0F703FD31
:1051600020B903210EA0FCF7E1FF03E003210FA00B
:10517000FCF7DCFF012314229F210020F3F7BAFE85
:1051800029460D48F6F736FE70BD00BFFCE700006B
:10519000636E000098260020B0030020C8030020A2
:1051A000CFB5CDB3C9E8D6C30000000053797374FE
:1051B000656D2053657400009001002070B50546B0
:1051C000002D64D053480078C8B953A15348F0F774
:1051D000CAFC18B952A0FDF787F902E055A0FDF707
:1051E00083F9322402E00120F7F742FE201EA4F1E9
:1051F00001018CB2F7D10120FFF722F970BD4548BB
:1052000090F82B03022802D042488078C8B142A10E
:105210004248F0F7A8FC18B94CA0FDF765F902E088
:105220004DA0FDF761F9322402E00120F7F720FEDE
:10523000201EA4F101018CB2F7D10220FFF700F982
:10524000DCE701210846FDF7C9FC0020464908803B
:10525000F3F7EAFC30A13148F0F785FC20B90321CF
:1052600042A0FCF763FF03E0032143A0FCF75EFFCD
:10527000012314229F210020F3F73CFEF9F71CFBC9
:10528000012368229F210020F3F734FEB6E7364859
:105290000088B8B91F4890F82B03012812D01EA12E
:1052A0001E48F0F760FC30B9012337A26E210020C0
:1052B000F4F7C8F821E0012339A26E210020F4F7A9
:1052C000C1F81AE028480088C82816D1114890F87B
:1052D0002B03012811D010A11048F0F744FC30B97D
:1052E000012334A26E210020F4F7ACF805E001237D
:1052F00036A26E210020F4F7A5F81B480088401C58
:1053000080B219490880B0F5C87F01DB0020088011
:1053100000BF73E7FC310020636E00009826002078
:105320002020C7EBCFC8B5C7C2BC2E2E2E20202010
:105330000000000020506C65617365206C6F676928
:105340006E2066697273742E2E2E0000BDFBD6B9D6
:10535000B2D9D7F7A3A1000043616E277420646F10
:1053600020746861740000003E040020D3C3BBA712
:10537000D1A1D4F100000000557365722053656C13
:10538000656374696F6E00005BC9CF5DD1A1D4F114
:105390002020202020205BCFC25DD1A1D4F10000CD
:1053A0005B55505D2020202020202020205B444F92
:1053B000574E5D005B4D5DB5A5BAF4202020205B03
:1053C000455849545DCDCBB3F60000005B4D5D43BD
:1053D000616C6C2020202020205B455849545D00E2
:1053E00070B50546002D64D04E480078C8B94EA16E
:1053F0004E48F0F7B8FB18B94DA0FDF775F802E07C
:1054000050A0FDF771F8322402E00120F7F730FDDB
:10541000201EA4F101018CB2F7D10120FFF710F892
:1054200070BD404890F82B03022802D03D48807898
:10543000C8B13DA13D48F0F796FB18B947A0FDF76C
:1054400053F802E048A0FDF74FF8322402E00120B3
:10545000F7F70EFD201EA4F101018CB2F7D1022056
:10546000FEF7EEFFDCE701210846FDF7A7FC002070
:1054700041490880F3F7D8FB2BA12C48F0F773FBC8
:1054800020B903213DA0FCF751FE03E003213EA01B
:10549000FCF74CFE012314229F210020F3F72AFD84
:1054A000F9F7B8FA012368229F210020F3F722FDC3
:1054B000B6E73148008890B91BA11C48F0F753FBB0
:1054C00030B9012334A26E210020F3F7BBFF1CE0AA
:1054D000012337A26E210020F3F7B4FF15E0264820
:1054E0000088C82811D110A11048F0F73CFB30B952
:1054F000012334A26E210020F3F7A4FF05E001236D
:1055000036A26E210020F3F79DFF1B480088401C47
:1055100080B219490880B0F5C87F01DB00200880FF
:1055200000BF7DE7FC310020636E0000982600205C
:105530002020C7EBCFC8B5C7C2BC2E2E2E202020FE
:105540000000000020506C65617365206C6F676916
:105550006E2066697273742E2E2E0000BDFBD6B9C4
:10556000B2D9D7F7A3A1000043616E277420646FFE
:10557000207468617400000040040020D3EFD2F46E
:10558000BCC7C2BC00000000766F6963652072650D
:10559000636F7264000000005BC9CF5DD1A1D4F1DC
:1055A0002020202020205BCFC25DD1A1D4F10000BB
:1055B0005B55505D20202020202020205B444F5749
:1055C0004E5D00005B4D5DB2A5B7C5202020205B7D
:1055D000455849545DCDCBB3F60000005B4D5D509E
:1055E0004C41592020202020205B455849545D0023
:1055F00000B504480021016081800120FEF720FFF2
:1056000000BD00004103002010B59AB0F6480078B4
:10561000012804D10020F44908701AB010BDF348E5
:1056200000782E2874D2DFE810F073002E005F009F
:105630007702C00027052A052D057300730073004B
:105640007300730037053A0540053D0573004305B7
:10565000460549054C054F05730052057300550575
:10566000730073005805F5035B0573005E05610563
:10567000640592006D0567056A057005730576057A
:1056800079057C057F05DA480068DA490844D8B115
:10569000B0F5001F1FD0B0F5601F23D1D6480078A9
:1056A000012800D1B9E7D54890F82B0302280AD188
:1056B000D248D3A26421D0F8A43001A802F068FA3D
:1056C00001A8F7F735F80DE00120C849487104201A
:1056D000FEF7B6FE06E00120C44948710320FEF73C
:1056E000AFFE00BF00BF16E2CA48F6F7D7FB04467C
:1056F000C9498C4224D1C7484079052819D2DFE82E
:1057000000F003080C1014000420FEF799FE10E0CE
:10571000A3E30320FEF794FE0BE01520FEF790FEB6
:1057200007E00620FEF78CFE03E00720FEF788FE68
:1057300000BF00BFB7484179B848F8F721FF05E03E
:10574000B748844202D10120FEF77AFECBE7B14888
:10575000F6F7A4FB0446B0498C4225D1AD48407908
:1057600005281BD2DFE800F0030A0E1216001420F1
:10577000FEF766FE0120AB4908610FE02720FEF727
:105780005FFE0BE02520FEF75BFE07E02820FEF71A
:1057900057FE03E02920FEF753FE00BF00BF9D48DF
:1057A00041799E48F8F7ECFE9DE79F48C0880028A5
:1057B00063D18F4800688F49494288425DD10420F7
:1057C0008E4981F830030846B0F9680000280BDDE7
:1057D0000846B0F96800062806DA0020A1F868003B
:1057E000042081F830033BE08448B0F8680060BBD7
:1057F00082488089052190FBF1F201FB120050B92B
:105800007E488089401F00B27C49A1F868000420CE
:1058100081F8300324E079488089052190FBF1F27A
:1058200001FB120075498989081A00B27349A1F871
:10583000680008468089052190FBF1F201FB120007
:10584000401E6E4981F830030AE06C48B0F86800E9
:10585000401F00B26949A1F86800042081F83003B4
:105860006648B0F9681071A002F082F9002108467C
:10587000FDF76AF8F9F776F835E76B48C088401C01
:1058800069498988884252D1594800686F498842DD
:105890004DD10020594981F83003084680890521FF
:1058A00090FBF1F201FB120020B90520534981F869
:1058B000310309E051488089052190FBF1F201FB99
:1058C00012004E4981F831034C4880894B4991F8C8
:1058D0003113401A4949B1F96810884204D10020B7
:1058E0004649A1F8680007E04448B0F86800401D48
:1058F00000B24249A1F868004048B0F968104BA0D6
:1059000002F036F93D48B0F968003C49898988427F
:1059100003DD00203949A1F868000020374981F8EB
:1059200030030121FDF710F8F9F71CF8DBE63E48DB
:10593000F5F7DCF904462E4800683949884214D14D
:1059400000202E4981F8300381F83403274840793C
:10595000012806D10020254948710120FEF770FD7D
:10596000D9E00220FEF76CFDD5E02B488442F7D148
:105970000020224981F830030120354908701F4872
:10598000808900B9D4E31D4890F83403012813D16D
:1059900000201A4981F834032348C08800EB4001F5
:1059A00001EBC0012B4850F821001449C1F838031D
:1059B0001E20FEF745FDAEE01048C16B1A48C088B6
:1059C00000EB400202EBC002224850F82200814264
:1059D0005DD121A12148F0F7C6F820B920A101A886
:1059E00002F0EAF848E043E0C1040020410300204F
:1059F0005C000020F6FB43FFC3000020FC310020C8
:105A000041542B504F433D35343026322625640D0A
:105A10000A000000500300200A04EC0010310020AE
:105A20000A04F400001001400C2F0020737574501C
:105A30006F635374617475732E68616E646C65492D
:105A40006E6465783D3D25640D0A00000A04DC00A3
:105A5000C800002080330020636E000098260020DC
:105A6000D2D1BEADD4DAB4CBC8BAD7E900000000B9
:105A7000FAA101A802F0A0F801A8FCF735FD642006
:105A8000F7F7F6F9F7494878FEF7DAFC50E3F648FD
:105A9000C08800EB400101EBC001F44850F8213010
:105AA000F3A2642101A802F073F801A8F6F740FE02
:105AB000012201A90020FDF733FBAFF26401F04899
:105AC000F0F751F878B9E848C08800EB400101EBE5
:105AD000C001E64800EB8100831DEAA2642101A811
:105AE00002F056F80EE0E048C08800EB400101EB00
:105AF000C001DE4800EB8100831DE4A2642101A8FF
:105B000002F046F801A8FCF7EFFC6420F7F7B0F9C3
:105B10000120FEF795FC0BE3D348C08880BBDE482C
:105B20000068DE4988425FD10420DD4981F83003F6
:105B30000846B0F9680000280BDD0846B0F9680097
:105B4000062806DA0020A1F86800042081F8300356
:105B50003CE0D348B0F8680068BBD14840890521D3
:105B600090FBF1F201FB120058B9CD484089401F6B
:105B700000B2CB49A1F86800042081F8300325E089
:105B800032E0C7484089052190FBF1F201FB120089
:105B9000C3494989081A00B2C149A1F868000846FA
:105BA0004089052190FBF1F201FB1200401EBC4927
:105BB00081F830030AE0BA48B0F86800401F00B22C
:105BC000B749A1F86800042081F83003B448B0F95F
:105BD0006810AFF2A81001F0CBFF00210846FCF7D7
:105BE000FDFFF8F769FEA3E29F48C088401C9E496C
:105BF0008988884254D1A8480068AA4988424FD170
:105C00000020A74981F8300308464089052190FB10
:105C1000F1F201FB120020B90520A14981F83103FE
:105C200009E09F484089052190FBF1F201FB120039
:105C30009B4981F831039A484089994991F8311379
:105C4000401A9749B1F96810884204D1002094495C
:105C5000A1F8680007E09248B0F86800401D00B263
:105C60008F49A1F868008E48B0F96810AFF244205F
:105C700001F07EFF8A48B0F9680089494989884265
:105C800003DD00208649A1F8680001210020FCF70F
:105C9000A5FF0020824981F83003F8F70DFE47E2A6
:105CA0007148F5F723F804467B4800687E4988422E
:105CB00012D16C484079012806D100206949487109
:105CC0000120FEF7BDFB02E00220FEF7B9FB002039
:105CD000734981F830039CE07448844276D10020F7
:105CE0006F4981F830030120714908706C48408980
:105CF00000B91DE26A4801695B48C08800EB4002B8
:105D000002EBC0026648A83050F82200814219D147
:105D1000AFF2BC215A48EFF726FF20B965A101A8D0
:105D200001F04AFF03E067A101A801F045FF01A8C7
:105D3000FCF7DAFBC820F7F79BF84A494878FEF7EA
:105D40007FFBF5E14848C08800EB400101EBC00152
:105D50005348A83050F821305DA2642101A801F019
:105D600017FF4F4801694048C08800EB400202EB32
:105D7000C0024B48A83050F8220081420CD13A486A
:105D8000C08800EB400101EBC0014548A83050F845
:105D900021004349C1F8A40001A8F6F7C9FCAFF2FD
:105DA00048313748EFF7DFFE88B92F48C08800EB4D
:105DB000400101EBC0013A48A83000EB8100431DCF
:105DC00048A2642101A801F0E3FE10E021E026488A
:105DD000C08800EB400101EBC0013148A83000EB66
:105DE0008100431D41A2642101A801F0D1FE1E489B
:105DF000C08800EB400202EBC0022948A83000EB4B
:105E00008200411D26487C30EFF7BBFE2620FEF7BE
:105E100017FB8DE11448C088F0B91F4800681F497E
:105E2000884219D11E48B0F96A00052877DBAFF225
:105E3000D8311348EFF797FE18B92EA0FCF754FBA2
:105E400002E030A0FCF750FB0120DFF8C8C000DF03
:105E500001203149087089E08FE068E1416C72658A
:105E600061647900410300200C2F00208033002062
:105E700041542B504F433D3532392625640D0A00DD
:105E800098260020BDF8C8EB3A257300456E74656E
:105E9000723A2573000000005C0000200A04BC0078
:105EA000FC3100200A04DC000A04F4000A04EC00BF
:105EB000C8000020CEDEB7A8BAF4BDD0D7D4BCBA93
:105EC0000000000043616E27742063616C6C000069
:105ED00041542B504F433D35343026312625640D37
:105EE0000A000000BAF4BDD03A25730043616C6C1F
:105EF0003A257300C3BBD3D0B8FCB6E0BCC7C2BC64
:105F0000000000005265636F72642074686520743D
:105F10006F702100198C010840030020FFE78648BC
:105F2000B0F86A0010BB8448C089052804DD05204C
:105F30008149A1F86A0019E000207F49A1F86A00B0
:105F4000AFF2EC417D48EFF70EFE20B9AFF25C00F6
:105F5000FCF7CAFA03E0AFF25400FCF7C5FA0120DF
:105F6000DFF8DCC100DF0120764908700021084617
:105F7000FCF724FFF8F74EFDDAE07348C088401CB8
:105F80007149898888423DD17048006870498842CB
:105F900038D16948B0F96A0005280BDB6648B0F8CB
:105FA0006A00401F00B26449A1F86A0001206549F7
:105FB000087014E06048B0F86A0080B9AFF2685128
:105FC0005E48EFF7D0FD18B962A0FCF78DFA02E049
:105FD00065A0FCF789FA0120DFF864C100DF5648AC
:105FE000D0F8381365A001F0C3FD01210846FCF785
:105FF000E5FEF8F70FFD5048D0F8381368A001F01F
:10600000B7FD95E05048F4F7C5FE04464F480068D8
:106010006C4988420BD100204A4908706A49487887
:10602000FEF70EFA0120444981F8340323E0674863
:10603000844220D14048C089E8B13F4890F87100BF
:106040004149C988401A401EC0EBC00101EB401114
:106050005F48405C009038485EA26421D0F8383335
:1060600001A801F095FD01A8F6F762FB012201A944
:106070000020FDF755F85BE0F6F74EFA58E0FBF725
:10608000E1FA55E0314800684E49884203D14E4953
:106090004878FEF7D5F94BE0F6F730F948E0F6F727
:1060A00093F945E0F6F7D8F842E0F5F7E1FF3FE075
:1060B000F9F766F93CE0F9F793FA39E0F9F7FEFEF3
:1060C00036E0FAF779FA33E0FAF7CEFF30E0FBF783
:1060D0009FFB2DE0FBF79EFC2AE0FAF729FC27E066
:1060E000FAF7F2F924E0F9F72BFE21E0F9F7F4FAD8
:1060F0001EE0FAF72BFF1BE000F0DCFF18E0F0F7E2
:1061000025FF15E0F1F756F812E0F1F709F80FE076
:10611000F1F7A2F80CE0FBF7E3F909E0F9F706FA6A
:1061200006E0F9F793FB03E0FBF7C4F800E000BFDB
:1061300000BF00BFFFF771BAFC3100209826002095
:10614000198C0108400300200C2F00205C00002067
:106150000A04DC00D2D1BEADCAC7D7EED0C2D2BBD2
:10616000CCF5A3A100000000546865206C61746543
:106170007374207265636F726421000073757450CC
:106180006F635374617475732E7265636F726449C3
:1061900044313131313D3D3D25640D0A00000000A0
:1061A000737574506F635374617475732E72656385
:1061B0006F726449443232323232323D3D3D2564A1
:1061C0000D0A00000A04F400410300200A04EC0058
:1061D0005C34002041542B504F433D353532262549
:1061E000642625640D0A000010B56A48007801286D
:1061F00002D11C20FEF724F96748007866498978A7
:10620000884208D06448007863494870084680781E
:106210000870012400E000245F4800782F2823D272
:10622000DFE800F0B61823272B2F3337B6B6B6B603
:10623000B63B3F4347B64B4F53575BB65F6366B6BB
:106240006A6E72767A7E82868A968E929A9EA2A6CE
:10625000AAAEB2005148F3F709FB2046FEF75AFCFC
:1062600000204D49C870087192E02046FEF72AFFD1
:106270008EE02046FEF7A2FF8AE02046FEF712F9E4
:1062800086E02046FEF700FC82E02046FEF756FF3F
:106290007EE02046FEF730FA7AE02046F6F75AF81C
:1062A00076E02046F6F7E8F872E02046F5F700FFC2
:1062B0006EE02046F5F7EAFF6AE02046F9F7C0F8FD
:1062C00066E02046F9F7D4F962E02046F9F72EFEA1
:1062D0005EE02046FAF7CAF95AE02046FAF74CFF8A
:1062E00056E02046FBF742FB52E0FBF76DFA4FE029
:1062F0002046FBF7E9FB4BE02046F1F783F947E046
:106300002046FAF7B3FB43E02046FFF769F83FE089
:106310002046F9F795FF3BE02046FBF7CFF937E041
:106320002046F9F74BFD33E02046F9F713FA2FE04A
:106330002046FAF78DFD2BE02046FEF791F827E086
:10634000204600F0DBFE23E02046F9F7DDFB1FE0EE
:106350002046F9F703FC1BE02046F9F705FC17E09F
:106360002046F9F731FC13E02046FAF7F3FF0FE07F
:106370002046F8F74BFF0BE02046F9F7D3FA07E089
:106380002046F8F749F803E02046F0F7ABF900BFE4
:1063900000BF10BD1C01002041030020103100206F
:1063A00030B587B00024214890F83C00012804D083
:1063B000022814D003282AD119E01C48406C64211B
:1063C00048431A49096CB0FBF1F0C5B22B4618A23C
:1063D000162101A801F0DCFB601CC4B217E01A4AC8
:1063E000162101A801F0D4FB601CC4B20FE0174ACB
:1063F000162101A801F0CCFBF3F76CF94FF47A7089
:10640000F0F721FBF3F766F9601CC4B200BF00BFD0
:106410002CB1012301AA46210020F3F713F8002034
:10642000024981F83C0007B030BD0000C00E0020DA
:106430002020D2D1CFC2D4D8B0D9B7D6D6AE20255D
:10644000642020200D0A00002D9901085B990108A5
:1064500010B5FDF77DFE10BD10B5FDF703FF10BDB3
:1064600010B5FDF75FFF10BD01F40072B2F5007FBB
:1064700000D100BFCA430280704710B5002200233C
:1064800040F66A14A14200D100BF0A1201249440D0
:10649000A3B2DC43048010BD21B1828942F40052D2
:1064A000828104E082894DF6FF731A408281704731
:1064B00002460020B1F5007F00D100BF13880B40D9
:1064C0000BB1012000E00020704770B502460024A7
:1064D00000230025002040F66A16B14200D100BF1B
:1064E000C1F3421501F01F03012606FA03F3012D43
:1064F00002D19689334006E0022D02D1168A33403C
:1065000001E0968A33400C12012606FA04F416883C
:10651000344013B10CB1012000E0002070BDF0B593
:106520000346002400260025002040F66A17B942E1
:1065300000D100BF1846C1F3421401F01F06012725
:1065400007FA06F5012C01D10C3004E0022C01D130
:10655000103000E014301AB107682F43076002E0E2
:106560000768AF430760F0BD2DE9F04786B00546E8
:106570000E460024A24600BFA1460027B08900B104
:1065800000BF2F462C8A4CF6FF700440F08804436D
:106590002C82AC894EF6F3100440B0883189084350
:1065A000718908430443AC81AC8A4FF6FF40044034
:1065B000B0890443AC8201A8F8F728F81F48874245
:1065C00002D1DDF810A001E0DDF80CA0A88900F4EC
:1065D000004040B10AEBCA0000EB0A1031684900E4
:1065E000B0FBF1F807E00AEBCA0000EB0A103168D3
:1065F0008900B0FBF1F86420B8FBF0F00401200939
:10660000642101FB1089A88900F4004040B13220C8
:1066100000EBC900B0FBF1F000F00700044308E014
:10662000322000EB09106421B0FBF1F000F00F0004
:1066300004432C8106B0BDE8F0870000003801401B
:1066400001468888C0F308007047C1F308028280C1
:106650007047000000B585B0012144F20400F7F74F
:10666000BBFF4FF40070ADF8100018208DF8130038
:1066700003208DF8120004A91C48F1F717F84FF415
:106680008060ADF8100004208DF8130003208DF811
:10669000120004A91548F1F709F84FF416500090BC
:1066A0000020ADF80400ADF80600ADF80800ADF824
:1066B0000C000C20ADF80A0069460D48FFF754FFA6
:1066C00001210B48FFF7E8FE40210948FFF7CCFE07
:1066D000002240F227710648FFF721FF002240F216
:1066E00025510348FFF71BFF05B000BD000801401E
:1066F000003801401FB5044622480078A04202D06D
:1067000020490C7000E01FBDECB14FF41650009012
:106710000020ADF80400ADF80600ADF80800ADF8B3
:106720000C000C20ADF80A0069461748FFF71CFF63
:1067300001211548FFF7B0FE012240F22551124811
:10674000FFF7EDFE1CE04FF4165000900020ADF86E
:106750000400ADF80600ADF80800ADF80C00082004
:10676000ADF80A0069460848FFF7FEFE0121064819
:10677000FFF792FE002240F225510348FFF7CFFEBB
:1067800000BFC0E78E010020003801401FB504465D
:10679000ECB14FF4E13000900020ADF80400ADF80A
:1067A0000600ADF80800ADF80C000C20ADF80A00AA
:1067B00069461648FFF7D8FE01211448FFF76CFE22
:1067C000012240F225511148FFF7A9FE1CE04FF4C9
:1067D000E13000900020ADF80400ADF80600ADF8FF
:1067E0000800ADF80C000820ADF80A00694607481B
:1067F000FFF7BAFE01210548FFF74EFE002240F2E6
:1068000025510248FFF78BFE1FBD000000380140F4
:1068100070B505460E4600240BE0295D0648FFF7DB
:1068200014FF00BF40210448FFF742FE0028F9D0C2
:10683000641CB442F1DB70BD0038014000B585B086
:1068400001210420F7F7C8FE01214804F7F7B4FE40
:106850000820ADF8100048208DF8130003208DF8B3
:10686000120004A92A48F0F721FF0420ADF8100017
:1068700018208DF8130004A92548F0F717FF4FF4EE
:10688000E13000900020ADF80400ADF80600ADF84E
:106890000800ADF80C000C20ADF80A0069461D4850
:1068A000FFF762FE40211B48FFF7DEFD002240F2A9
:1068B00027711848FFF733FE012240F22551154891
:1068C000FFF72DFE002240F224411248FFF727FE79
:1068D000012228210F48FFF722FE012260210D48E6
:1068E000FFF71DFE01210B48FFF7D6FD00200A49E6
:1068F00008800A4908800A4908800A4908800A492C
:1069000008704FF4A0610948EFF7F1F805B000BD39
:10691000000801400044004084010020860100205E
:10692000880100208A0100208C010020022900201B
:106930002DE9F04186B07F48008840F2FE41884250
:106940001ADD002240F225517B48FFF7E8FD0020C8
:106950007A4908807749088079490880012240F205
:1069600025517548FFF7DBFD012276A11046FCF7A3
:10697000D7FB06B0BDE8F0816E480688102E01DA1C
:10698000354600E010256E48078800240CE0714869
:10699000C05D01A90855781C80B20746B0F5A06F0C
:1069A00000DD0027601C84B2AC42F0DBEB21042048
:1069B000F8F7ACFB68A101A8F5F7D1FE002870D06C
:1069C0005F48078800240DE06248C05D0A2800D1B6
:1069D0000AE0781C80B20746B0F5A06F00DB002704
:1069E000601C84B2B442EFDB00BFB4427EDA601CAC
:1069F00085B24FF480710420F8F788FB40F2FE4026
:106A000085424ADA56480580002413E051484C4933
:106A10000988415C5248801C015549480088401C47
:106A200080B247490880B0F5A06F01DB00200880E4
:106A3000601C84B2AC42E9DB00214948801C01554E
:106A4000002240F225513C48FFF769FD3948008893
:106A5000401B38490880012240F225513648FFF793
:106A60005EFD4FF488710420F8F750FB01223C4989
:106A7000891C0020FCF754FB39480088401C384929
:106A8000088008460188801CF6F722F920B101220F
:106A900034A10020FCF744FB6BE73148058000245B
:106AA0001AE044E02B482649098810F8018040F29A
:106AB000FE40844203DA2A48801C00F80480204803
:106AC0000088401C80B21E490880B0F5A06F01DB31
:106AD00000200880601C84B2AC42E3DB0021204827
:106AE00080F80115002240F2255100E01EE0124816
:106AF000FFF715FD0F480088401B0E490880012252
:106B000040F225510C48FFF70AFD4FF49371042021
:106B1000F8F7FCFA12480188801CF6F7D9F820B182
:106B2000012214A10020FCF7FBFA22E721E700BFB5
:106B30001FE700008601002000440040880100207B
:106B40008A0100205B527832427566204F7665726A
:106B50005D000000022900202B544350000000007B
:106B6000D86E00204D51756575652046756C6C3189
:106B7000000000004D51756575652046756C6C32DE
:106B80000000000070B505460E4600240BE0295DAC
:106B90000648FFF75AFD00BF40210448FFF788FC74
:106BA0000028F9D0641CB442F1DB70BD0044004001
:106BB00000B585B001210820F7F70EFD01218804FA
:106BC000F7F7FAFC4FF40060ADF8100048208DF89C
:106BD000130003208DF8120004A91E48F0F766FD8B
:106BE0004FF4165000900020ADF80400ADF80600F8
:106BF000ADF80800ADF80C000420ADF80A006946B5
:106C00001548FFF7B1FC40211348FFF72DFC002287
:106C100040F227711048FFF782FC002240F2255114
:106C20000D48FFF77CFC002240F224410A48FFF7A0
:106C300076FC01210848FFF72FFC00200749088057
:106C4000074908804FF496710648EEF750FF05B0EB
:106C500000BD0000000C0140004800407E01002003
:106C600080010020D62700202DE9F041DFF8C0C0C8
:106C70009CF800C04FEA8C00DFF8B8C01CF8007028
:106C8000E04600F1010C18F80C6000F1020C18F855
:106C90000C50E910B210FB104FEAC12C0CEB421C57
:106CA0009C441FFA8CF4DFF890C0ACF80040DFF889
:106CB0008CC09CF800C04FEA8C00C4461CF80070E1
:106CC00000F1010C18F80C6000F1020C18F80C50DF
:106CD000E910B210FB104FEAC12C0CEB421C9C4493
:106CE0001FFA8CF4DFF858C0ACF80040DFF854C04D
:106CF0009CF800C04FEA8C00C4461CF8007000F1FC
:106D0000010C18F80C6000F1020C18F80C50E91096
:106D1000B210FB104FEAC12C0CEB421C9C441FFA32
:106D20008CF4DFF824C0ACF80040BDE8F08100002E
:106D3000B1040020F4780020BA040020B20400203E
:106D4000BC040020B0040020B804002004480268FD
:106D50000448018804A000F00BFF00BFFEE700001C
:106D6000D8000020D40000200D0A5B5546485D463F
:106D70003D25642C4C3D25640000000010B586B014
:106D80002D4890F83D0308B906B010BD2B48007897
:106D900000B9F9E72A480078012800D1F4E729482A
:106DA0000078FA2843DA27480078401C2549087003
:106DB000084600781E2190FBF1F201FB120000282A
:106DC00038D121480068B0F5A57F33D91F48007835
:106DD00001282FD01C480068B0F5DA7F09D31C4881
:106DE000006864231BA21421009001A800F0D0FECB
:106DF00011E015480068A0F5AA70642148435A21A3
:106E0000B0FBF1F412480068234612A2142100904E
:106E100001A800F0BDFE01A8F5F78AFC012201A936
:106E20000020FCF77DF900200649087002E00020F0
:106E30000449087000BFA7E7FC3100206001002072
:106E4000B701002074010020D00000204C03002076
:106E50004800002041542B504F433D353232262507
:106E6000642625640D0A000070B586B01B4C1C48D2
:106E700090F82D311BA2142101A800F089FE0025F5
:106E800023E0642601A8F5F753FC17E04FF4A06156
:106E9000A01CF5F781FE80B2208058B115A1A01C7E
:106EA000F5F75DFC50B9012214A10020FCF738F978
:106EB00006B070BD0120DFF858C000DF301EA6F11B
:106EC0000101CEB2E2D1681CC5B20A2DD9DB012284
:106ED00010A10020FCF724F900BFE9E7DA730020D5
:106EE000B825002041542B504F433D3630372625DE
:106EF000640D0A003E363037263100005B30335DCA
:106F000053657420566F6C756D65206F6B000000C3
:106F1000198C01085B30335D53657420566F6C75B6
:106F20006D65206661696C656400000010B586B00F
:106F300000F036F810211848F0F797FC0020ADF863
:106F400004004FF48270ADF806000020ADF8080090
:106F50000220ADF80A000120ADF80C004002ADF8A7
:106F60000E000820ADF810000020ADF81200072038
:106F7000ADF8140001A90948F8F7ECF80121074819
:106F8000F8F7CEF84FF47A70EFF76EFD02F08CFA56
:106F90000446012006B010BD000801400030014049
:106FA00008B501210420F7F717FB01210803F7F7C3
:106FB00013FB2020ADF8000003208DF802001820FC
:106FC0008DF8030069460F48F0F770FB8020ADF89C
:106FD000000069460B48F0F769FB4020ADF800005F
:106FE00004208DF8030069460648F0F75FFB102087
:106FF000ADF800008DF8030069460248F0F756FB33
:1070000008BD00000008014070B51C4C00221CA106
:107010001046FCF785F8002527E04FF4FA761CA00F
:10702000F5F786FB1CE04FF4A061A01CF5F7B4FD5A
:1070300080B2208080B118A1A01CF5F790FB20B190
:1070400016A1A01CF5F78BFB50B9012214A100205A
:10705000FCF766F8002070BD0120DFF84CC000DFAF
:10706000301EA6F10106DED16D1C0A2DD5DB0122F2
:107070000EA10020FCF754F80120ECE7DA730020A1
:10708000576169744D6F64656D52756E3A0000000A
:1070900041540D0A00000000524459004F4B0000BB
:1070A00052756E696E670000198C010854696D6530
:1070B0004F75740010B58AB00848046808488442C7
:1070C0000AD1084808A22821D0F8A430684600F068
:1070D0005FFD6846F5F72CFB0AB010BD5C00002090
:1070E0000A04F400FC31002041542B504F433D353D
:1070F000343026322625640D0A00000010B58EB00B
:107100000446002C28D0F1F78FFD14A11448EEF7A7
:107110002AFD30B9134B14A2322101A800F038FD2A
:1071200005E0104B12A2322101A800F031FD01A8A8
:10713000FBF7DAF909A10A48EEF715FD30B901238A
:107140000DA26E210020F2F77DF905E0012310A2C7
:107150006E210020F2F776F90EB010BD636E0000CC
:107160009826002078320020BAF4BDD03A2573006A
:1071700043616C6C3A2573002020202020202020C1
:107180002020202020202020B9D2B6CF00000000EF
:107190002020202020202020202020202048616E38
:1071A0006755700070B5194C002219A11046FBF705
:1071B000B7FF1BA0F5F7BCFA00251EE0322617E04A
:1071C0004FF4A061A01CF5F7E7FC80B2208058B115
:1071D00017A1A01CF5F7C3FA50B9012216A100208F
:1071E000FBF79EFF002070BD0120DFF85CC000DFD0
:1071F000301EA6F10106E3D16D1C642DDEDB0122F9
:1072000012A10020FBF78CFF0120ECE7DA730020CD
:1072100057616974506F63496E69743A00000000E9
:1072200041542B504F433D3630350D0A00000000CD
:107230003E36303526310000506F63496E69742048
:107240004F6B0D0A00000000198C0108506F634954
:107250006E69742054696D654F7574002DE9F047AF
:1072600005460E461746B5F1006F02D32048854209
:1072700001D3BDE8F087C5F3090018B11DA000F0E7
:1072800077FCF6E7EFF730FE3420EFF7BDFD6FF047
:107290007F40EFF735FE4FF00109494619A000F095
:1072A00067FC2846EFF7B6FD8146494619A000F075
:1072B0005FFCB9F1040F06D049461AA000F058FC53
:1072C000EFF7E8FDD5E700240CE0315D601C305C91
:1072D00001EB00201FFA80F828194146EFF7E4FD82
:1072E000A01C84B2BC42F0DBEFF7D4FD00BFC0E7C6
:1072F0000000020861646472202D2D2D6572726F8A
:107300000D0A0000737461747573313D25640D0AB4
:1073100000000000737461747573323D25640D0ABA
:1073200000000000657261736520206572726F2D28
:107330002D2D2D2D25640D0A000000002DE9F047AC
:10734000A4B00546884628783E280AD1002405E0E6
:10735000601C285C23A90855601CC4B2032CF7DB11
:1073600008E0002404E0285D23A90855601CC4B28D
:10737000032CF8DB00208DF88F0023A8EEF719FC12
:1073800087B2892F75D019DC762F73D009DCA7F16D
:107390006F0007286FD2DFE800F051572A5D6E6E4C
:1073A000FA00842F68D004DC772F7CD0812F62D143
:1073B0008FE0862F78D0872FF9D16EE1C92F74D056
:1073C0000CDC972F72D004DC8C2F70D0962FEED16E
:1073D00097E1982F6CD0C82FE9D170E0A7F1CC00CD
:1073E0000528D7D2DFE800F07A7B9BA7F500F948A3
:1073F000A0F20F1191F80E11A0F20F1292F80D21C8
